:020000040800F2
:100000000000012069AE050805AF0508F9330408B2
:100010005D34040805AF050805AF050800000000C1
:1000200000000000000000000000000005AF05080F
:1000300005AF05080000000005AF0508E5DB030873
:1000400005AF050805AF050805AF050805AF0508AC
:1000500005AF050805AF0508BD350408B53504082A
:10006000AD350408A53504089D350408659E0508CE
:10007000559E0508459E0508359E0508219E0508E4
:100080000D9E0508F99D050805AF050805AF050893
:1000900005AF050805AF050805AF05089535040847
:1000A000A18005089981050891800508C18105088E
:1000B000898105087981050869810508E5A1050898
:1000C000F1A10508CDA10508D9A1050805AF0508CE
:1000D00005AF05087DDC03086DDC03085DDC030863
:1000E0008D35040805AF050805AF050881800508B2
:1000F000B180050805AF0508D9800508E59D05080C
:1001000005AF0508057005085981050805AF050804
:100110004DDC03083DDC0308E98005081DDC000810
:10012000D19D0508BD9D0508A99D0508959D05085B
:10013000819D050800000000000000000000000094
:10014000000000000000000000000000B5E0000812
:100150006D9D0508599D0508459D05082DDC030882
:10016000B5A10508C1A1050805AF050805AF05083B
:1001700005AF050805AF05080000000000000000FD
:1001800005AF050805AF050805AF050805AF05086B
:1001900005AF050805AF05080000000005AF05081C
:1001A00000000000000000000000000005AF05088E
:1001B00005AF050805AF05080000000000000000BD
:1001C000000000000000000000000000000000002F
:1001D00000000000000000000000000005AF05085E
:0801E000C0A9050001000000A8
:1001E8000E02010002000000245301208853012060
:1001F80000000000FC3007088453012014020100AD
:10020800050000004C2B0120905301200000000045
:10021800FE3007088C530120031101000A0000007A
:10022800D85201209C53012000000000850F0108CE
:10023800985301202320010010000000A85201203B
:10024800AC53012000000000DD6D0208A853012016
:100258000D1001007000000030520120C053012031
:1002680000000000FD570308BC530120FD010100F8
:1002780024000000B4510120345401200000000083
:10028800B3C3030830540120FB0101000100000042
:10029800705101205C5401200000000079BF04085F
:1002A80058540120FC010100090000003C500120C5
:1002B800645401200000000081BF0408605401203C
:1002C800F7010100060000001050012074540120BD
:1002D800000000000431070870540120F9010100F2
:1002E800040000000050012080540120000000009C
:1002F80021C403087C5401203400010010000000D0
:100308002C4F012088540120000000009575020838
:10031800845401201102010008000000044F01204C
:100328009C540120000000000A310708985401205D
:100338001212010004000000FC4E0120A854012004
:100348000000000012310708A454012018300100F1
:1003580038000000C44E0120B05401200000000005
:10036800E1C70408AC540120000201000B000000A2
:10037800484B0120EC54012000000000BDBF0408D8
:10038800E8540120FF21010005000000EC4A01208B
:10039800FC5401200000000059BF0408F854012053
:1003A8000812040014000000F84A01200855012032
:1003B80000000000E5BF04080455012013020100F5
:1003C80004000000442B01202055012000000000FB
:1003D800163107081C550120FA010100030000002E
:1003E8004C4A01202855012000000000DDBF040808
:1003F800245501202A02010008000000404A01207B
:1004080030550120000000001A3107082C55012042
:100418002052010008000000F84901203C55012045
:1004280000000000B97502083855012006100100C7
:1004380024000000D4490120485501200000000094
:1004480065C00408445501200C02010004000000A6
:1004580070480120705501200000000069BF0408A1
:100468006C550120FE010100140000008C340120AD
:100478007855012000000000C5BF0408745501200C
:100488000B3001001A000000BC8F0120C891012028
:100498000000000024310708C49101201F5001000A
:1004A80024000000808F0120E89101200000000056
:1004B80040310708E4910120050201000400000012
:1004C80030900120109201200000000064310708DC
:1004D8000C9201201B2001000C0000002C9501202B
:1004E800CC9F012000000000FD740108C89F012076
:1004F80021020100F00000005C930120DC9F012034
:1005080000000000A9810108D89F012037100100D0
:1005180030000000E89C0120D0A00120000000006D
:1005280068310708CCA00120161001000600000061
:10053800E896012004A10120000000009831070876
:1005480000A101202F10010022000000A49F01201B
:1005580010A10120000000009E3107080CA1012015
:1005680023220100100000004C96012038A1012030
:1005780000000000C031070834A101201E0001005E
:1005880009000000349601204CA101200000000061
:10059800D031070848A10120052001000C00000007
:1005A800BC9601205CA1012000000000DC31070896
:1005B80058A1012012300100100000001C960120F3
:1005C8006CA1012000000000E831070868A10120A3
:1005D800FD0701007C0000002092012080A101207D
:1005E800000000006D6E01087CA10120F59101005A
:1005F8006C000000E092012000A201200000000031
:10060800CD800108FCA10120261001000E00000089
:1006180080A2012070A2012000000000716C010876
:100628006CA201201400010005000000E4B50120BF
:100638000CB6012000000000F831070808B60120B8
:10064800012001000C000000D0AA012018B60120EA
:1006580000000000FE31070814B601200C40060017
:10066800E400000084A9012028B601200000000051
:1006780045FF020824B601200A900100240000006A
:1006880040A9012010B7012000000000956D020864
:100698000CB701200E300300BC0100007CA701202C
:1006A80038B7012000000000D575020834B70120D2
:1006B800131001000400000070B30120F8B80120F5
:1006C800000000000C320708F4B801200101010005
:1006D80004000000B4A6012000B9012000000000B9
:1006E80000000000FCB80120000101000400000027
:1006F800ACA6012008B9012000000000103207084C
:1007080004B901200201010003000000A8A601208D
:1007180010B901200000000089FF02080CB901206F
:10072800220201001C010000BCB0012018B9012000
:1007380000000000B9C8040814B901200102010032
:100748000B000000C0A6012038BA012000000000FC
:10075800ADBF040834BA0120020201000300000002
:1007680048AB012048BA012000000000000000004A
:1007780044BA01201B0201001000000024AB012034
:1007880050BA01200000000051C004084CBA0120F2
:10079800150010007000000074C7012038C801203F
:1007A800000000000000000034C801202A000800F2
:1007B8006000000084C60120ACC8012000000000D1
:1007C8006D750208A8C801202C0004001000000064
:1007D80020C9012010C90120000000004974020846
:1007E8000CC901202920140078000000FCC3012056
:1007F80034C90120000000000000000030C90120B9
:100808001A0001000E00000020C30120B0C9012019
:100818000000000014320708ACC901202B001200A8
:1008280024000000FCC20120C4C90120000000000F
:100838001D740208C0C9012019020100100000003F
:1008480000C20120ECC90120000000009DBF04087F
:10085800E8C901201C0202001C00000034C001206D
:1008680000CA012000000000C5C50408FCC9012019
:10087800283001001600000050C0012020CA0120C5
:1008880000000000CD7602081CCA01200A020100FF
:1008980014000000B8D40120D4D4012000000000C6
:1008A80011FF0208D0D4012010100100020000003E
:1008B80040CE0120ECD401200000000022320708BD
:1008C800E8D40120F83101000600000048CF0120DB
:1008D800F4D401200000000024320708F0D40120DD
:1008E800030001000100000058CF012000D50120BD
:1008F8000000000000000000FCD4012019000100E5
:1009080005000000F8CD012008D5012000000000F6
:100918002A32070804D50120020001000C0000005B
:1009280020D6012074D8012000000000000000003B
:1009380070D80120F62101000C000000BCD701206E
:1009480084D80120000000003032070880D8012038
:1009580025201E002C0100002CD6012094D801204F
:10096800000000000000000090D8012029020100CA
:10097800400000004CD50120C4D90120000000002F
:100988003C320708C0D901202C02010004000000F5
:100998003CD8012008DA0120000000007C3207085A
:1009A80004DA01202802040004000000C8E1012044
:1009B800A0E70120000000004DC004089CE70120CA
:1009C8002702040004000000C4E10120A8E7012078
:1009D8000000000041C00408A4E701201602150029
:1009E8003F000000B8DA0120B0E701200000000055
:1009F80099BF0408ACE701201A0201003C0000007E
:100A08007CDA0120F4E70120000000003DC804085A
:100A1800F0E70120031201003D000000C8E30120B7
:100A280034E80120000000008032070830E8012087
:100A3800382001000300000048DA012078E801208E
:100A480000000000BE32070874E801200400080016
:100A5800800000003CE90120BCEA01200000000001
:100A6800000000003CEB01200B2201003D000000CB
:100A7800A4EE012098F4012000000000C432070809
:100A880094F401200D1201001400000070F40120FC
:100A9800DCF401200000000004330708D8F401202A
:100AA8001E0201000600000004EF0120F4F40120FA
:100AB8000000000018330708F0F401201D020200AE
:100AC8000600000010F4012000F5012000000000DD
:100AD80000000000FCF401200612040018000000C9
:100AE80018F401200CF501200000000055C6040888
:100AF80008F501201F0208001000000038F5012049
:100B080028F501200000000011BF040824F5012089
:100B1800270001000400000020EF01204CF501200F
:100B2800000000001E33070848F5012010020100EC
:100B380001000000481902204419022000000000AA
:080B48002233070840190220C6
:08280000082800080040000850
:10800000026C03463AB11A6CD20608D50022012050
:1080100083F83C207047426480F83C20F3E71A6CF8
:1080200049494A4811401A6841F00201F0B4196404
:108030004168474D21F44031416041685C6821430B
:1080400041605168186921F48071D3F808C0DF6875
:10805000516054689E6A44EA0024AE4254605468F9
:1080600024F040745460506840EA0C0050609068FE
:1080700020F400609060916841EA0701916054D05B
:108080009068DC6A20F07060906091680E439660A2
:10809000906820F040509060916821439160906812
:1080A0009C6920F002009060916841EA440191606F
:1080B00093F82010002941D05468596A44F40064B0
:1080C000481E5460516821F460415160516841EA92
:1080D00040315160D06A0025DC6920F470005E698F
:1080E000611ED0622846D46A44EA0154D46294687E
:1080F00024F400749460946893F8301044EA4124A6
:108100009460946824F480649460916841EA8621C4
:1081100091605D641A6C22F0030242F001021A645D
:10812000002283F83C20F0BC7047916821F0706118
:108130009160916821F040519160B0E7516821F45D
:1081400000615160C6E700BFFDEEFFFF0023014064
:108150000100000F0129F0B42A4C4FF000062A4D0F
:1081600094BF002701272368EE626662A6626763F8
:10817000676B47EA42076763EE63EC6B002A38D10E
:1081800044F49574EC631C6824F001041C601C68C2
:10819000E407FCD4490289085960D8601968EAB933
:1081A00021F04001196019498B421DD018494FF444
:1081B0007410C860196841F01E011960596941F0D6
:1081C00080015961196841F00101196022B90E4A14
:1081D000D36A43F00803D362F0BC704741F040011A
:1081E00019600A498B42E1D14FF0746041F8500C9C
:1081F000E0E744F01A04EC63EC6A44F00804EC6233
:10820000C1E700BF88190120002C014058640240DA
:108210000064024011480023024611780632032907
:1082200016D00133062BF8D10D49CA6D052A0ED0A0
:1082300002EB4203013200EB4303CA65032040F224
:10824000EB3140F2FF32187059809A8070477047C6
:1082500003EB430300EB4303F0E700BFC019012029
:1082600088190120124B30B41D6E6B6A28B943EA9D
:1082700001430020AB6230BC7047AC6A013803EBAD
:1082800014440BD0002303F14002013305EB8202BA
:10829000DBB25268834204EB1244F4D3403044EA28
:1082A000014405EB80004460002030BC704700BFF3
:1082B00088190120037870B42BB30246C0F1010580
:1082C000531912F8014FDBB2002CF9D101335B00D6
:1082D0000E4C03220B8084F8643484F86524017802
:1082E00079B1022300265A1CE518023354FA82F2AF
:1082F00085F86414DBB282F8646410F8011F002969
:10830000F1D170BC70470223E2E700BF8819012059
:10831000826D136A5B681B78FF2B08D090F8F030F1
:10832000013BDBB280F8F0301BB101207047002028
:108330007047126A0220526813707047F0B40F4BF6
:10834000C40800F0070700221E5D03EBD005BE4005
:10835000F6B2C7F1080300278B4228BF0B46C3F1D2
:1083600008049A40C91A46FA04F415F8016F42EA63
:108370000402EED11046F0BC704700BF2C1F012054
:1083800030B5EFF31181802383F312880A4AD2F8C3
:108390005836D2F85C46D2F85806D2F85C56CAB2C3
:1083A00082F31188013BA84294BF4FF40060002083
:1083B0001B1B184430BD00BF88190120012380F821
:1083C00051307047014BD3F860067047881901207F
:1083D00001207047024BC3F86426C3F86816704743
:1083E00088190120024BC3F86C26C3F87016704739
:1083F0008819012070477047212870B505D02228C0
:1084000029D0202810D0002070BD0029FBD0072AD9
:10841000F9D1184B18791C685A799B79087100209A
:108420000C604A718B7170BD0029ECD0072AEAD12B
:108430001148104B0C680E794D79D0F8682689796F
:108440001C601E715D719971002ADCD02146D0F844
:1084500064069047D7E70029D5D0022AD3D1064A2F
:10846000D2F87036002BCED00988D2F86C06984727
:10847000C9E700BF000001208819012000207047D3
:1084800003460A2201481A80704700BF08000120F5
:108490000346642201481A80704700BF140001207F
:1084A000012901D000207047014BD3F890301847C4
:1084B00000000120012901D008F0BCB9014BD3F81C
:1084C0008C30184700000120014BD3F88830184742
:1084D0000000012010B40B780A46044603F00303A1
:1084E000012B05D0022B0BD000205DF8044B704708
:1084F0008B8843B9204611465DF8044B0CF074BBE1
:108500008B88832BF6D0034B5DF8044BD3F8803077
:10851000184700BF0000012038B5054B04460D4642
:10852000DB6F98472946204608F03EFF002038BD03
:108530000000012038B5054B04460D469B6F984757
:108540002946204608F068FF002038BD00000120C1
:10855000F0B4002452004E1C2746030FB0F1204F08
:108560004FEA001003F1300503F1370334BF0D5516
:108570000B5537550234A242EFD1F0BC704700BF13
:10858000024808B5FFF796FE014808BD9C5C060846
:10859000EC1D0120024808B5FFF78CFE014808BD1C
:1085A000AC5C0608EC1D01200B481A220B4B00683E
:1085B0001B680A80C01801D109487047094B08227E
:1085C000094910B51C68FFF7C3FF0422074920467C
:1085D000FFF7BEFF024810BD107AF01F187AF01F97
:1085E000B0000120147AF01FB2000120C200012067
:1085F000024808B5FFF75EFE014808BDB85C0608F2
:10860000EC1D0120024808B5FFF754FE014808BDE3
:10861000C45C0608EC1D0120042301480B80704750
:10862000CC00012000487047141F0120004870470B
:10863000141F0120034B93F88805032894BF0020E2
:108640000120704788190120034B93F888050328FF
:1086500094BF00200120704788190120034B93F834
:108660008805003818BF0120704700BF8819012015
:10867000034B93F88805003818BF0120704700BFEE
:108680008819012098B182680C4B12B107229A70A8
:10869000704718780421DA6003281A611A750CBF34
:1086A00080224FF480729970C3E901227047034B16
:1086B000012241F2E4715A705A5470478C750120BE
:1086C0000378022B0FD0006908B9012070470E4BC8
:1086D0001B78032B12D080B24FF6F773984294BFE9
:1086E000002001207047084941F6500243688A582B
:1086F000B3EB422F2CBF012000207047034B984260
:1087000094BF0020012070478C750120F7FFFF0FF8
:1087100030B40378022B13D0104A41F64801436865
:1087200041F63C04555802F5C25100692B400968D6
:10873000023812595B0A01FB003030BC104470470C
:10874000064B41F6300441F6340142681859595835
:1087500000EB410030BC00EB522070478C750120CB
:10876000826D0346126A52681278FF2A0AD190F885
:10877000F020002A02F1FF3214BF0120022083F80A
:10878000F02070470020704738B540F48062074CF5
:108790000B4640F2FF55012100F03F00A563A360A6
:1087A000E2604EF081FAA56338BD00BF002C0140A5
:1087B0002DE9F843884600294FD04718461E284C1B
:1087C000802507F1FF39EFF3118185F31288D4F882
:1087D0005826C9B2D4F85C06D4F85836D4F85CC62A
:1087E00081F31188634594BF4FF400630023121A8C
:1087F0001344012B1AD1012035F0EAF9EFF311816E
:1088000085F31288D4F85826C9B2D4F85C06D4F897
:108810005836D4F85C7681F31188BB4294BF4FF48C
:1088200000630023121A1344012BE4D0EFF31182EA
:1088300085F31288D4F85C36D2B216F8011F2344AF
:1088400083F87416D4F85C360133C3F30A03C4F812
:108850005C3682F311884E45B5D14046BDE8F883B9
:1088600088190120F8B5002390F8505080F8503056
:10887000CDB10F4941F2E8028A5C032A15D10D4EB1
:1088800000F13C04B76A29462046FFF791FFB36A1E
:108890002D1A0444DB1B322B01D8002DF3D1B5FA7D
:1088A00085F04009F8BD0120FCE71846FAE700BF53
:1088B00088190120802A0120002280F85120D1E768
:1088C00090F85020531C0244DBB280F8503082F8FC
:1088D0003C1090F851200AB1132B00D9C2E7704721
:1088E000F8B5144641F2E803094A0D46D35C032B60
:1088F0000DD1084EB76A002C09DD21462846FFF746
:1089000057FFB36A241A0544DB1B322BF3D9F8BD99
:1089100088190120802A012010B5074C04F2BC50B0
:108920003BF01EFA0A2035F047F9D4F8C405BDE83B
:10893000104038F0DBB800BF8819012030B50023A3
:108940008DB0124A082102930DF107058DF81430FD
:108950000124099302F2BC508DF828300B9382F861
:1089600054166944CDE90733094BCDE90354069306
:108970003AF0B8FF07483BF0F3F99DF80700A0F183
:10898000FF00B0FA80F040090DB030BD8819012019
:1089900011830008441F0120F0B503798BB0284CE7
:1089A000002B14BF0122002284F8B42503D184F8DF
:1089B00088350BB0F0BD04F2BC56054690F90010A6
:1089C00030463BF095F8AD7875BB01271D4B1E482E
:1089D000C4F85036C4F8C45584F8C8753BF0C6F8DE
:1089E00003464FF47A70A4F8C03535F0F1F8D4F8A6
:1089F000C40538F07BF828226846002154F03EFB7D
:108A00000A236946304602933AF06CFF30463BF049
:108A1000A7F90E4B002284F888759B6A84F87C25A0
:108A2000C4F878350BB0F0BD284637F095FE054602
:108A300008B11E23C3800D21284637F017FFC4E775
:108A400088190120EC1E0120801A0600802A0120CE
:108A500070B5952592B0044640F0400601AA080C76
:108A60008DF809500D0E8DF80810090A00238DF8B5
:108A700005508DF8060006250DF103008DF807104E
:108A800003920121174A8DF8046004938DF8183081
:108A90008DF82C300F938DF84030119305950C9282
:108AA000CDE90733CDE90D33CDE90901FFF746FFE5
:108AB00024B180F0010010F0FF0F10D10A4C082300
:108AC00003A904F2BC5084F854363AF00BFF04F2C8
:108AD000BC503BF045F99DF8030012B070BDFF207B
:108AE00012B070BD618700088819012030B50023DD
:108AF0008DB0104A014602930DF107058DF8143030
:108B00000124099302F2BC508DF828300B9382F8AF
:108B1000541602A9CDE90733074BCDE90354069358
:108B20003AF0E0FE05483BF01BF99DF807000DB058
:108B300030BD00BF8819012061870008441F012053
:108B400070B590B01C4D0024FD220DF103030126E9
:108B500001A905F2BC508DF803200693C5F88445A1
:108B60008DF81040059407948DF824408DF8384016
:108B70000F9403960896CDE90144CDE90A44CDE966
:108B80000C443AF0AFFE05F2BC503BF0E9F8304639
:108B9000FFF7ACFFFF2809D0084A20460923926A54
:108BA00085F88835C5F8782510B070BD04230220FB
:108BB00085F8883510B070BD88190120802A012001
:108BC00070B5064690B008200D46FFF78FFFFF28CE
:108BD00022D0FE2802D0022010B070BD0024022353
:108BE00001A90F48089301948DF8104007948DF85F
:108BF00024408DF838400F94CDE90265CDE9054455
:108C0000CDE90A44CDE90C443AF06CFE04483BF04F
:108C1000A7F8204610B070BD012010B070BD00BF95
:108C2000441F01202DE9F84F484B98420FD003F51F
:108C30006853083398424DD00023454A1846A2F89D
:108C40009430A2F8A030C2E92633BDE8F88F404C3A
:108C5000022300263F4F04F13005DFF80481E36270
:108C6000D7F8D0303146B34206F1010603D0D4F82C
:108C7000B00047F033FE94F8B4302846D4F8B02062
:108C8000414685F82430303545F8102C48F03AF844
:108C9000E36A9E42E4DB002384F8A230E36A012009
:108CA000E16BA28EA56B12FB03F201FB03F3B4F898
:108CB0004060A4F89420C4F89C30E28E264BC4F89F
:108CC000C010C4F89850A4F8A060A4F89620C4F886
:108CD0009030BAE71E4C02224FF0000B1D4F04F1FA
:108CE00030054FF4806A4FF040094FF40068E262AB
:108CF000D7F8D020012659465A45B34403D0D4F8BA
:108D0000B00047F0EBFD4FF00062D4F8B0104FF424
:108D1000003094F8B4C0296285F824C0A5F804A0F6
:108D2000A5F81090A5F80680AE74C5E90202FFF719
:108D300071FA28466E7647F031FFE26A074B934599
:108D400045F8303BD4DB84F8A260A7E71971EF0047
:108D5000802A0120000001209CD3050870D305085B
:108D60001940EF0010B50C4647F0E8FB50B9074B2F
:108D700093F8C430012B4FF012030CBF0448054890
:108D8000238010BD12230448238010BD802A0120B7
:108D9000FC000120E8000120D40001202DE9F84367
:108DA0001C4C05468946904694F888651F46042E5B
:108DB00008D0082E02D00020BDE8F883FFF7C0FEDF
:108DC0000228F8D1D4F8C40537F08AFE94F87E352D
:108DD000B3B969021120FFF73BFEB8B90E4A05236B
:108DE0000120C4F86495926AC4F86855C4F8708587
:108DF000C4F87475C4F8782584F88835BDE8F8831C
:108E000029461120FFF724FE0028E7D0FFF784FD54
:108E1000D1E700BF88190120802A012010B50D4C30
:108E2000002394F85626C4F8843512B10A4AC2F8D1
:108E3000C8304EF045F920B10423022084F888356B
:108E400010BD054A0923926A84F88835C4F878254C
:108E500010BD00BF88190120802A012070B50F4D78
:108E600004460E4695F88835042B0BD0082B07D105
:108E7000D5F8803583420ED0FFF7D0FF022801D00D
:108E8000012070BD08230220C5F88465C5F880451F
:108E900085F8883570BD022070BD00BF881901209B
:108EA00010B509F06FFA104C58B194F88835032BBF
:108EB00013D894F87C350133DBB2072B84F87C356A
:108EC00003D9002384F8883510BD084B01229B6A22
:108ED00084F88825C4F8783510BD05483AF046FE78
:108EE000A4F8C005E5E700BF88190120802A012009
:108EF000801A060070B51F4C06460D4694F888355A
:108F0000042B09D0082B25D1D4F8803583422FD0EB
:108F1000FFF716FE02281DD1D4F8C40537F0E0FD96
:108F200000213720FFF794FD29461720FFF790FD19
:108F3000C0B994F87E357BB971021920FFF788FD1E
:108F400080B908230220C4F88455C4F8806584F8E9
:108F5000883570BD012070BD31461920FFF778FDBE
:108F60000028EED0FFF7D8FCFFF79AFF032070BD72
:108F7000022070BD8819012070B50379234C002BA5
:108F800014BF0123002384F8B43503D1002384F8EF
:108F9000883570BD1E4D0021032095F9CF203AF091
:108FA000B3FB0028F2D0466830463AF0D9FB84F88B
:108FB00055060028EAD095F8CD303046003B18BF62
:108FC000012384F856364DF013FC09F0DBF938B96B
:108FD00094F87C3584F88805013384F87C3570BDBD
:108FE0004EF048F940B194F87C350022013384F802
:108FF000882584F87C3570BDAA6A012384F87C0535
:10900000C4F8782584F8883570BD00BF8819012020
:10901000802A012010B54EF02DF958B10C4C94F86F
:109020007C350133DBB2072B84F87C3503D9002370
:1090300084F8883510BD09F0A5F90028F7D0054B54
:1090400001229B6A84F88825C4F8783510BD00BFDA
:1090500088190120802A01202DE9F84F904C94F8BE
:10906000B455002D00F0028194F8882502278D4E1A
:10907000531E082B3ED8DFE803F03436A73D66497F
:10908000153D05004EF01CF8002840F00181D4F891
:109090007835B26AFA33934229D2FFF7BBFF94F8CE
:1090A0008825E5E74EF00CF80028F0D0D4F8843598
:1090B0000022012B84F87C2540F2EE80D4F8801544
:1090C000013B94F856560131C4F88435C4F8801534
:1090D00015B1744BC3F8C8200823054684F88835B9
:1090E00011E084F888754DF0EBFF00284DD194F81D
:1090F0008825531EDBB2022B3CD9082A18BF042A4C
:109100000CBF012500252846BDE8F88F236B002BF6
:1091100037D1644B0722D4F870559B6A84F88825B0
:10912000C4F87835002DEED0D4F874350120D4F889
:109130006425D4F86815A847D9E7D4F87835B26A19
:10914000643393421DD2D4F82C80B8F1000FF4D1CF
:109150004DF0B6FF0028A2D00423D4F8705584F84F
:109160007C8584F88835002D00F090804046D4F846
:109170007435DCE74B4BD4F878259B6A9B1AC82BD7
:1091800079D800252846BDE8F88F4DF02BFC002843
:10919000ADD196F8D130002BA3F10203B3FA83F3DB
:1091A00014BF022201225B0984F87D2584F87E35F4
:1091B0004DF018FC00287FF470AFD6F8202103236F
:1091C000C4F88C2584F888354DF00CFC00288ED12D
:1091D000344A4FF0040EC4F88405032392F804B116
:1091E000B2F80611D2F8080184F892B5D2F80871E5
:1091F0004FEA106CD2F80861A4F890153F0CD2F831
:1092000008A1360A92F80C9192F80D5192F80D01CE
:10921000D2F8108125FA0EF5B2F816B100F00F0061
:10922000B2F81611B2F81621C1F30B1184F893C5E8
:1092300002F00F0C84F8947541EA1B21724684F801
:10924000956501F00F0184F896A584F8979501F5CE
:10925000FA6184F89C5584F89D05C4F89885A4F8B3
:109260009E1584F8A0C584F888E543E7284684F86D
:109270008855BDE8F88FFFF7CDFE94F88855082D86
:1092800018BF042D0CBF012500253CE705463AE731
:10929000042384F8883536E7FAD1FFF7BFFD26E7C7
:1092A00088190120802A01202DE9F84305468846C7
:1092B00017461E462A4C94F88805042835D00828FD
:1092C00007D1D4F88035AB4206D0FFF739FC02282D
:1092D000F1D00120BDE8F883FC22224BDFF88C900E
:1092E000214883F83021C9F838813AF02BFB002857
:1092F00009F588711C4814BF4FF400734FF4807354
:10930000C9F840313AF0EEFA012206230020C4F8F1
:109310006485C4F86855C4F87075C4F8746584F839
:109320006C2584F88835BDE8F883D4F8C40537F097
:10933000D7FB94F87E3553B969021820FFF788FBF4
:1093400038B994F88835082BC6D0FE22C5E72946DF
:10935000F3E7FFF7E1FAFFF7A3FD0320BAE700BF49
:1093600088190120802A0120441F012000000120CB
:109370002DE9F04FD84C95B094F8B465002E00F06C
:10938000998194F8882504F2BC57DFF8508304F2E1
:10939000A459531E082B00F2A080DFE813F034001C
:1093A0005E0029019E008C00AF001B009E0009009A
:1093B000FFF7C4FA002840F05482D4F87835D8F882
:1093C0002820FA33934280F08580FFF769FD94F8F6
:1093D0008825DEE7FFF7B2FA0028EED0D4F884350E
:1093E0000022012B84F87C2540F26082D4F880258D
:1093F000013B082106460132C4F8843584F88815FB
:10940000C4F8802552E1D4F8C40537F069FB002187
:109410000846FFF71DFB0546FFF77EFA012D59D1DF
:109420004FF0000AD4F8C40584F87DA537F058FB46
:1094300040F2AB110820FFF70BFB052800F09081EC
:10944000012800F05181FFF767FA94F87D35002B71
:1094500000F02882022384F88835D4F8C40537F058
:109460003FFB94F87D3500213720022B0CBF4FF0D5
:1094700080450D46FFF7ECFA29202946FFF7E8FA68
:109480000546FFF749FA2DBB94F87D35022B00F015
:10949000988184F87E55D4F8C40537F021FB00216B
:1094A0000920FFF7D5FA002871D0FFF735FA94F8B4
:1094B0008825531E11E04FF40071D4F86405FFF7BE
:1094C0007FFB012800F03081022800F03581002860
:1094D00000F0618194F88825531EDBB2022B00F264
:1094E000DF807E4BD4F878259B6A9B1AC82B00F24C
:1094F000E7800026304615B0BDE8F08FD4F8BC35C3
:1095000077481D6A3AF01EFA002800F02C81B5FA5F
:1095100085F56D09002DDDD004A800250DF10F03A0
:1095200002224FF0010A05A9059038460792ADF8CE
:10953000105006958DF820508DF834508DF8485015
:109540001395CDE90B3ACDE90955CDE90E55CDE995
:1095500010553AF0C7F938463AF002FC9DF80F3042
:1095600003F01F03052B00F08581FFF799FCD4F869
:1095700070B5BBF1000F00F0F0802A465046D4F8D9
:109580007435D4F86815D84794F8882501E7102178
:109590004846FFF715FB8246002886D101217F202F
:1095A000FEF7CCFE012805467FF47FAF504602212E
:1095B000FEF7C4FE002800F0358101287FF475AF66
:1095C00016213A20FEF7BAFE01308002C4F88C055D
:1095D000FFF7A2F9D4F8C40537F082FA00210A2077
:1095E000FFF736FA002840F01681032384F8883507
:1095F000102105A8FFF7E4FA00287FF46BAF9DF86F
:1096000021309DF822201B019DF815009DF8165071
:1096100002F00F01DBB245EA0025DDF81D0043EA48
:1096200012139DF81C2000BA84F8A01503F5FA6304
:109630009DF81710C4F89805A4F89E3513099DF8F5
:10964000140002F00F0284F89C35069BA4F8905594
:10965000C4F8943584F89D2584F8920584F8931510
:10966000FFF75AF994F87E3573B9D4F8C40537F08A
:1096700037FA4FF400711020FFF7EAF90546FFF7BB
:109680004BF9002D7FF4A1AE16483AF06FFA002294
:109690000423A4F8C005C4F884251A4684F8883544
:1096A000082A18BF042A0CBF01260026304615B030
:1096B000BDE8F08F304684F8886515B0BDE8F08FBE
:1096C000FFF7EEFB94F88865042E18BF082E0CBF38
:1096D00001260026EAE700BF88190120802A012020
:1096E000441F012040787D01042304AA05A977487E
:1096F00007930692CDF814A08DF820A08DF834A021
:10970000CDF838A0CDE909AACDE90BAA3AF0EAF8DC
:109710006E483AF025FB9DF81330AB2B7FF493AEE7
:10972000022384F87D358EE6D4F87835D8F82820E1
:1097300064339342BFF4CEAEFFF7EEF8FFF7B0FB11
:10974000D4F870554DB10022D4F87435D4F86815AA
:109750001046A84794F888251BE694F8882518E653
:1097600084F87D556FE694F86C550246D4F864157C
:109770004FF48073384601EB05213AF0D7FA94F89C
:109780006C250132D2B2A2F1020584F86C25B5FA3B
:1097900085F56D09BEE60190FFF7BEF80423019838
:1097A000D4F8705584F87C0584F88835002D3FF492
:1097B0007DAFD4F87435D4F86425D4F86815A8477B
:1097C00088E6D4F8C40537F08BF929463A20FFF72C
:1097D0003FF904AA0423824605A9384605958DF869
:1097E00020508DF834500E95CDE90955CDE90B5533
:1097F000CDE906233AF076F838463AF0B1FABAF1F4
:10980000000F08D1FFF788F8049B1BBAC3F38073DD
:1098100084F87E353FE6FFF77FF8FFF741FB94F8C9
:109820008825B6E504212C20FEF788FD0321824619
:109830004E20FEF783FD83460C213620FEF77EFD89
:109840000BF1020B421C05FA0AF502FA0BF2A2FB1D
:109850000501420A42EAC152C4F88C25FFF75CF8C0
:10986000B8E60190FFF758F80423019884F888358A
:1098700006461BE7164B0722D4F870659B6A84F8EE
:109880008825C4F87835002E3FF410AFD4F874352D
:109890005046D4F86425D4F86815B04794F8882564
:1098A000531E1AE61E4684F88835FFE608D00423C6
:1098B00084F88835FFF730F894F88825531E0CE6B5
:1098C000FFF73EF902287FF405AEEEE5441F0120C4
:1098D000802A0120154BDB68C3F3022310B4C3F1C7
:1098E00007041A1D042C28BF0424062A4FF0FF3257
:1098F0008CBF033B0023A240002821EA020101FAA9
:1099000003F108DB09010A4BC9B2034483F80013D1
:109910005DF8044B704700F00F000901054BC9B218
:10992000034419765DF8044B704700BF00ED00E07A
:1099300000E100E0FCEC00E030B5264C00222648B7
:1099400041F28731D4F8743183B0244DA0FB030376
:1099500004F59A70C4F83451DB0C013BC4E9501291
:10996000C4E94E320CF098FA1D4B062137201A6CD0
:1099700042F020021A641B6C03F020030193019B48
:10998000FFF7A8FFD4F834314FF400001549164A08
:109990004860D96841F00101D96099680A40062AF7
:1099A00006D0B2F5803F03D01A6842F001021A6077
:1099B0000E4B41F2041200200D499A5803F27464D0
:1099C000C3F87006C2F81002C3F86806C2E9811431
:1099D00003B030BD802A012083DE1B430014004009
:1099E0000038024000E100E0070001008819012072
:1099F000F82B012038B50F4B0F4AD3F87431A2FB76
:109A000003239B09013BB3F1807F10D20B4A002452
:109A1000F0200B490725536081F82300214694600C
:109A20004FF0FF301560FFF755FF204638BD01208D
:109A300038BD00BF802A0120D34D621010E000E045
:109A400000ED00E04309012200F01F0084B0013B5B
:109A500002FA00F0032B0BD8DFE803F015021E0C0E
:109A6000124B5A6C02435A645A6C10400090009B8F
:109A700004B070470D4B1A6B02431A631A6B104007
:109A80000390039BF4E7094B5A6B02435A635A6BEA
:109A900010400290029BEBE7044B1A6C02431A64DD
:109AA0001A6C10400190019BE2E700BF00380240B1
:109AB0002DE9F041D0F800E00C46DFF8588084B082
:109AC000DEF804501746DFF850C0194605EA0805CD
:109AD000DDF82880064603932C43424644EA0C0CEA
:109AE000CEF804C00AF098F978B931680246039BB1
:109AF00030468F624021CDF800800AF0BDF9003871
:109B000018BF012004B0BDE8F081012004B0BDE819
:109B1000F08100BF009800FC00200180F8B5134FD1
:109B200004460D460AE09B69DB0602D50AF034F9CB
:109B3000D0B9D7F878395B1B0A2B08D823682A4696
:109B40000A2120469E69B606EDD50020F8BD636C5B
:109B50002021002201200B4384F84020636484F814
:109B6000411084F84220F8BD0120F8BD802A012070
:109B70002DE9F04788B0884615461F46064639F05D
:109B8000FBFC041E30DB224BDFF890901A19B188E1
:109B900009EB840492F858A0C4F87C895EB14FF0B8
:109BA0000042B1FA81F0C24005D01A48046824EAA4
:109BB00002040460426103EB870305F0030230688E
:109BC000C5F341149B6E0026C5F38105D1441343B0
:109BD000039103A907960695CDE9043408F0D6FD54
:109BE00099F8BC39F02B02D808B0BDE8F0870A4AD2
:109BF000F023032112F90A0089F8BC390190FFF71C
:109C000069FE01980CF020F808B0BDE8F08700BFAD
:109C100070D30508003C01402C5D0608802A012015
:109C200010B4B8B10D4CD4F8C439102B05D10521AE
:109C300000205DF8044B39F06FBC03EB4302224473
:109C400082F8C919012182F8C8090B4482F8CA199F
:109C5000C4F8C4395DF8044B704700BF802A012066
:109C600020218078DCE700BF2DE9F04FC14C0023B4
:109C700087B004F6F81894F80C2AC4F8F839C8E943
:109C80000133C8E903331AB194F80D3A84F8F8396E
:109C900094F80E3A1BB194F80F3A84F8073A94F806
:109CA000123A1BB194F8133A84F8023A94F8103A35
:109CB0001BB194F8113A84F8FD3994F8143A013B39
:109CC0005FB2DBB2019702933B46013300F04F8154
:109CD000A94EB0220023A94802FB076106F5217AAC
:109CE000A0F128050093743106F53F7953F054F93B
:109CF0000122009B2E4602FA07FB1F46307890B3E4
:109D00009F494FF0300C03E089452CD011F808CF63
:109D10006045F9D14A7812EA0B0FF5D036F01CFDF8
:109D2000FB1DDBB210B100218371C171032136F03C
:109D30009DFD30780023302101E01AF8331088426D
:109D400000F0B2810133102BF7D14FF0000C009AD4
:109D50000121072086F801C0531CB270F170DBB2FC
:109D6000307100930B4601370536042FC6D194F8A5
:109D7000240A01270393FFF765FE4FF44031814E1B
:109D80000022009BC4F82C1A3046D4F8201AC4F8DC
:109D9000443AC4F8407AC4F8387A84F8587AC4F857
:109DA000302AC4F8502AC4F8542AC4F8342A84F853
:109DB000482AC4F84C2AC4F83C2AC4F8281AFEF7EA
:109DC0001FF9019B002B40F0EF80039B002B00F05C
:109DD000EB80A6F1080050F059FA012308F11408AD
:109DE0004FF0000A9B46EA78002A40F017810535BB
:109DF0004545F8D1019B02200299234493F91C2A7E
:109E000039F082FC0546002800F0B180406839F046
:109E1000A7FC0022062139F0B3FC002800F0A7803F
:109E20006868002739F09CFCDFF874814FF078FFF8
:109E3000009B6A68012B4FF40063A8684FF400553B
:109E40008CBF4FF480613946C4F8702A4FF4003259
:109E5000C4F8801A4FF48071C4F8843A0323C4F81C
:109E6000740A4046C4F8983AC4F8787AC4F87C7A00
:109E7000C4F8947AC4F89C7AC4F8A07AC4F8885AD2
:109E8000C4F88C1AC4F8902A09F064FB94F8643A78
:109E9000C4F8608A012B0597C4F8A86A67D001232B
:109EA000D4F8285A84F8643AAB68DE0713D4D4F89F
:109EB00074313549AA68B3FBF1F342F0010203EBB8
:109EC0004303AA600593059B2BB1059B013B0593BA
:109ED000059B002BF9D1AB68D80748D5D4F8682A80
:109EE0002A4B134043F48073C4F8683A6B685905F1
:109EF00007D5D4F8683A23F4405343F48053C4F8A8
:109F0000683AD4F8683A13F4805300F03881D4F8F2
:109F10006C3A23F00603C4F86C3A1D4800231D492F
:109F20006FF02202C4F8B00A1B4884F8643AC4F8FF
:109F3000AC1A05F14C01C4F8BC0A2A606E68009B9B
:109F400046F08066154A16486E60AE6846F4807624
:109F5000AE6009F073FA134B5A68D20640F0F880ED
:109F6000D4F8283A9A6812F0405F00F0038107B0F5
:109F7000BDE8F08F802A012070D30508A0340120AD
:109F8000F4D50508A834012040420F00FEF8FFFF79
:109F9000B90C0108BD0C0108A90C0108E40100205E
:109FA000F034012000230140B02200217B484827E3
:109FB00053F064F8B0220021784853F05FF8784BF2
:109FC000384684F8D47AC4F8D03AFFF73BFD4FF412
:109FD000403000230121D4F8D02AC4F8DC0A7148AB
:109FE000C4F8F01AC4F8E81A84F8081BC4F8E03A78
:109FF000C4F8003BC4F8043BC4F8E43AC4F8F43AAB
:10A0000084F8F83AC4F8FC3AC4F8EC3AC4F8D82A10
:10A01000FDF7F6FF614850F039F9DEE694F8640A7E
:10A020005A1C69780128D2B22F79CDF810A039D006
:10A03000092984F864BA52D94FF0030E6FF01D005D
:10A04000D4F828CA4FF007091EFB0100DCF80CE029
:10A0500009FA00F907FA00F02EEA0907CCF80C70AB
:10A06000DCF80C703843CCF80C00062B4FF00500E0
:10A0700020D86FF0040710FB0373D4F8287A1F2050
:10A0800000FA03FC786B01FA03F320EA0C00786312
:10A09000786B03437B63D4F8283A4148834234D039
:10A0A00084F864AA1346A2E63F4A02EBC30393F87E
:10A0B00088C24CE60C2B32D86FF0220710FB0373DA
:10A0C000D4F8280A1F2707FA03FC076B01FA03F3E9
:10A0D00027EA0C070763076B3B430363DBE7D4F80E
:10A0E000280A01EB41094FF0070ED0F810C007FA1B
:10A0F00009F70EFA09FE2CEA0E0CC0F810C0D0F8D1
:10A1000010C047EA0C070761AFE712291AD01129DE
:10A11000C6D126494B6843F400034B60C0E76FF09B
:10A12000400710FB0373D4F8280A1F2707FA03FC23
:10A13000C76A01FA03F327EA0C07C762C76A3B4301
:10A14000C362A8E719494B6843F480034B60A7E753
:10A15000D4F8282A12498A4214D05B68DB063FF5FE
:10A1600006AF134B9A427FF402AF9A6812F0405F39
:10A170007FF4FDAE9A6842F080429A60F7E6C4F838
:10A180006C3ACAE6936813F0405F03D1936843F0DA
:10A1900080439360054B5B68E9E600BF50350120C2
:10A1A000002001405835012070D3050800230140EC
:10A1B000002201402DE9F041D0F800E00C46DFF824
:10A1C000588084B0DEF804501746DFF850C01946B6
:10A1D00005EA0805DDF82880064603932C4342462D
:10A1E00044EA0C0CCEF804C009F016FE78B93168C8
:10A1F0000246039B30468F628021CDF8008009F033
:10A200003BFE003818BF012004B0BDE8F0810120FA
:10A2100004B0BDE8F08100BF009800FC002001817F
:10A22000034690F83C00012800F03E810220F0B483
:10A23000012483F83D0083F83C40142A45D8DFE828
:10A2400012F04D004400440044007B0044004400F0
:10A250004400DA00440044004400AA0044004400E2
:10A260004400060144004400440015001A688E684A
:10A27000156A0F6825F48015AB4C1562106A556895
:10A2800020F40010D2F854C040EA0650A74E0CEA61
:10A290000404B24244EA072400F0088106F580660F
:10A2A000B24200F003814E6855605465D665106275
:10A2B000506D0C6940F400605065506D20F4806072
:10A2C0005065516D41EA042151650022012110467B
:10A2D00083F83D1083F83C20F0BC70471A68D1F831
:10A2E00008C0156A0F6825F00105914C1562106AC7
:10A2F0005668956920F002002C408C4D40EA0C0015
:10A30000AA4244EA070400F0DD8005F58065AA4210
:10A3100000F0D8804D685660946155631062906972
:10A320000C6940F008009061906920F00400906191
:10A33000916921439161C8E71A68D1F808C0156A8C
:10A340000F6825F010057B4C1562106A56689569F8
:10A3500020F020002C40754D40EA0C10AA4244EA3F
:10A36000072400F0C38005F58065AA4200F0BE8096
:10A370004D68566094619563106290690C6940F471
:10A3800000609061906920F480609061916941EA79
:10A390000421916199E71A688E68156A0F6825F49F
:10A3A0008055644C1562106A556820F40050D2F84C
:10A3B0001CC040EA06305D4E0CEA0404B24244EA96
:10A3C000072400F08D8006F58066B24200F0888098
:10A3D0004E685560D46116641062D0690C6940F40F
:10A3E0000060D061D06920F48060D061D16941EA19
:10A3F0000421D16169E71A68D1F808C0156A0F68AD
:10A4000025F480754A4C1562106A5668D56920F4A7
:10A4100000702C40454D40EA0C20AA4244EA070453
:10A4200073D005F58065AA426FD04D685660D4613F
:10A43000D5631062D0690C6940F00800D061D06922
:10A4400020F00400D061D1692143D1613DE71A6851
:10A450008E68156A0F6825F48035374C1562106ACE
:10A46000556820F40030D2F854C040EA06402F4E20
:10A470000CEA0404B24244EA07041DD006F58066E3
:10A48000B24219D04E685560546596651062506DA1
:10A490000C6940F008005065506D20F004005065D4
:10A4A000516D2143516510E70220704725F4802546
:10A4B0004E6945EA8625F6E625F480354E6945EA7B
:10A4C0000625DFE726F4407C20F008008E69CF687F
:10A4D0004D693843354320F0040045EA0C0619E77E
:10A4E00025F480454E6945EA861571E726F4406CEF
:10A4F00020F080008E69CF684D6940EA071035432F
:10A5000020F040004CEA850632E726F4405C20F457
:10A5100000608E69CF684D6940EA0720354320F41A
:10A5200080604CEA051680E7FF8FFFFE00000140C7
:10A530008CFFFEFFFF8CFFFE8FFFFEFFF8B53D4E48
:10A5400096F8804B04EB4403670006EBC30393F8D3
:10A55000843B032B44D8DFE803F0461B0F023C4446
:10A5600006EBC404D4F8883B002B58D0013B0025EF
:10A57000C4F8883B2846F8BD3B1906EBC303D3F863
:10A58000882B7AB1013A0025C3F8882B2846F8BDFC
:10A590003B1906EBC303D3F8882B002AF2D1022221
:10A5A00083F8842B3C4406EBC40494F8903B013BB5
:10A5B000DBB284F8903B4BBB0323D4F88C0B84F8BC
:10A5C000843B52F0B1FEC4F8880B064652F088FE78
:10A5D00080F00100002E0CBF002500F0010525BB16
:10A5E00001252846F8BD3AF0A3FE05460028F7D01D
:10A5F0003C44012342F2107006EBC40484F8843B0F
:10A6000052F092FEC4F8880B2846F8BD01254FF49D
:10A610007A7052F089FEC4F8880B2846F8BD52F0D3
:10A620006BFE80F00100C5B2B0E7013EC4F8886B54
:10A63000ACE700BF802A012003689B0AA3F58013C2
:10A64000522B00D970470E4A134470B593F8044357
:10A6500084B00D2C12D800294FF0000309494FF0A7
:10A66000010514BF1E460226427901EB841069469B
:10A67000CDE90065CDE902330BF00EFB04B070BDEF
:10A6800070D305086436012033492DE9F84F91F85D
:10A69000D1101C46012507460229DFF8C4A0104648
:10A6A00019464FF00002DFF8BC9018BF7F02CAF8CD
:10A6B0002C50FDF74FFD294A630240F2FF5BC9F8B9
:10A6C00024204FF40075C9F828304FF48A62D9F875
:10A6D0002C30012110205E4643F09303C9F82C3042
:10A6E000C9F838B0C9F808504D46C9F80C204CF0EC
:10A6F000DBFA012CC9F838B04FF00A048CBF4FF0D8
:10A7000052084FF051084FF0000939464046FEF715
:10A710003BF8013C034640F2774201213720E4B286
:10A7200023B91846CAF82830BDE8F88FAE63C5F8DB
:10A730000890EA604CF0B8FAAE63034608B1002C0A
:10A74000E3D1002BEDD000221846CAF82C20CAF81D
:10A750002830BDE8F88F00BF802A012000E1F50510
:10A7600088190120002C01402DE9F843DFF874809E
:10A7700004460F46914698F888551E46042D08D089
:10A78000082D02D00020BDE8F883FEF747FB022821
:10A79000F8D101233A4620460021FFF775FF68B142
:10A7A000FEF738FCD8F87045002CEBD00022D8F822
:10A7B0007435D8F868151046A047E3E7084A052322
:10A7C0000120C8F86475926AC8F86845C8F87095A1
:10A7D000C8F87465C8F8782588F88835BDE8F88326
:10A7E000802A0120881901202A492DE9F04F91F88B
:10A7F000D1100124DFF8A8B00746022983B0CBF8B6
:10A8000030409A4618BF4702012B4FF00A04224DF0
:10A8100040F2FF568CBF4FF059084FF058084FF0E8
:10A820000009009239464046FDF7AEFF013C034661
:10A8300040F2774201213720E4B2BBB9009851467B
:10A8400001220193154CFDF785FC13494FEA4A227A
:10A850000020019B4C628A62CA6A42F09102CA627D
:10A86000CBF82800184603B0BDE8F08FAE63C5F8FA
:10A870000890EA604CF018FAAE63034608B1002C69
:10A88000D0D1002BDAD000221846CBF8302003B00C
:10A89000BDE8F08F802A0120002C014000E1F50581
:10A8A000881901202DE9F84F05460E4690461F46AF
:10A8B000394C94F8880504280CD0082807D1D4F81E
:10A8C0008035AB4206D0FEF7A9FA0228F1D001206C
:10A8D000BDE8F88FDFF8C8A0C4F86465DAF8C8905E
:10A8E000C4F86855C9F34F234FEA59220F2B2BD8D0
:10A8F000D4F884B5BBF1000F26D094F8561619B3DE
:10A90000B9F5005F41D025484FF400723146484404
:10A9100052F042FB09F50072C2F34F23CAF8C82077
:10A92000520A102B31D0BBF1010F2ED0D4F8802564
:10A930000BF1FF33042102200132C4F8843584F87E
:10A940008815C4F88025C3E701234FF00109284684
:10A95000062532460021C4F87085C4F8747584F861
:10A960006C9584F88855FFF73FFF0028B0D0FEF7BC
:10A9700051FBD4F870556DB14846D4F87435D4F80D
:10A9800068150022A8470320A2E792B2034E013ABD
:10A99000AD1ADAE703209BE7881901208C550120C6
:10A9A000802A012070B50D4C1346D4F8A45F2A7894
:10A9B000022A07D00A46014604F6A470BDE870409A
:10A9C0003AF030B82A6A0AB1002070BD0A46014642
:10A9D00004F6A47039F02AF9012070BD802A012004
:10A9E00003681878012801D00020704793F90430DB
:10A9F000074A03EB430302EB431313F8332C202ADB
:10AA0000F3D153F8743C9869C0F3C030704700BF6D
:10AA1000783B0120036801221B78022B01D03AF019
:10AA20002BBA39F05BB910B50B4CD4F8A43F1B78A6
:10AA3000022B10D1D4F8AC0F36F058F8D4F8AC0F84
:10AA400008B12123C380012135F010FF034839F0FC
:10AA50008DF8A4F8A80F10BD802A012080969800D8
:10AA600038B505460A460C460648294639F00EF91F
:10AA700045F08001034839F08DF8231A58425841B7
:10AA800038BD00BF243A012030B5044683B001230D
:10AA90000D460DF107020848214639F0C3FF9DF825
:10AAA000072035EA020304D02A43214602483AF03F
:10AAB00097FA03B030BD00BF243A012013B53A4CD9
:10AAC0000023D4F804218DF80730137803F0FD013A
:10AAD000012905D194F8081111B90C2184F8081145
:10AAE000022B1ED0032B2ED001220B212F484BF01E
:10AAF00055FD042033F06CF801230DF1070200210D
:10AB00002A484BF06DFD002839D09DF80730482BBE
:10AB100035D1274BC4F8F830264BC4F8FC3002B0CE
:10AB200010BDD4F80C0135F0E1FFD4F80C0108B1E8
:10AB30003523C380012135F099FE1F4839F016F8FE
:10AB4000A4F80801D0E7D4F8B43546F2A81150684B
:10AB5000122219610023372180F888304BF0F1FC74
:10AB6000D4F804310D22242158684BF0EAFCD4F8C3
:10AB7000043130226A2158684BF0E3FCB4E7D4F882
:10AB800004311A78022A03D0032A07D00020C6E72E
:10AB9000D4F80C0138F086FE0020C0E710223721DF
:10ABA00058684BF0CEFCF1E7783B01207C3C01205B
:10ABB0003F660508C166050880969800F8B55E4CAA
:10ABC00000234FF4F07206460F4604F63810202199
:10ABD00084F8343984F8353952F050FA4FF4F07271
:10ABE000202104F6183052F049FA322032F0F0FFFA
:10ABF00094F8F93C002B00F0948094F8FA1C04F6C9
:10AC0000FC4038F075FF002800F08B8094F8F90CB8
:10AC100035F0A2FD0546C4F8040D35F069FE0028A4
:10AC20007FD00DB12323EB800D21284635F01EFE89
:10AC3000D4F8040D35F05AFF404838F097FF03462A
:10AC4000FF213F48A4F8003D39F052F88C213C48E0
:10AC500038F0A0FF1B2867D10122D4F8043D84F806
:10AC600034290BB12322DA8040220A21344839F0FA
:10AC70000DF88A21324838F08DFF94F8F83CC0F383
:10AC8000801584F8945D002B44D0022B3BD12D48D5
:10AC900038F06CFF0346A4F8960D94F8982D182A06
:10ACA00011D1294A2949D2F87421A4F89C7D52086F
:10ACB000A4F89E5DA4F8A03DB2FBF3F2A1FB021242
:10ACC000520BA4F8A22D1E4802220021A4F8003D38
:10ACD00038F0DCFFC8201A4D32F06EFF8021284684
:10ACE00038F058FF10F00200F8D17278B37831785C
:10ACF000C2F12002C3F1100384F8A52D84F8A63D0B
:10AD000084F8A41DF8BD124838F030FF0346A4F8BB
:10AD1000960DC2E7094838F029FF0346A4F8960DBE
:10AD2000BBE76FF00100F8BDD4F8040D202135F029
:10AD30009DFD4FF0FF30F8BD783B0120404B4C00AB
:10AD400074480120002D3101802A01205917B7D104
:10AD5000809698000146014838F01CBF2049012028
:10AD600030B40023314D32494CF25034C5F8583ECE
:10AD7000304AD1F8780904E0D1F878391B1AA34297
:10AD80000FD8D368DB03F7D4D16811F4F9710BD174
:10AD9000D06810F0010002D001230846D36030BC17
:10ADA0007047032030BC7047D3689B0705D5D5F8A2
:10ADB000583E43F02003C5F8583E1E4BDB68DC06C6
:10ADC00005D5D5F8583E43F01003C5F8583E194B49
:10ADD000DB68980605D5D5F8583E43F00803C5F85A
:10ADE000583E144BDB68590605D5D5F8583E43F05C
:10ADF0000403C5F8583E0F4BDB681A0605D5D5F895
:10AE0000583E43F00203C5F8583E0A4BDB68DB05A9
:10AE100005D5D5F8583E43F04003C5F8583E054BDC
:10AE20004FF4F9720120DA6030BC7047783B0120A2
:10AE3000802A0120003C0240014488420ED0034693
:10AE4000074810B4074C13F8012B04FB00F099429B
:10AE500080EA0200F7D15DF8044B70470048704764
:10AE6000C59D1C8193010001094B93F85E3E042BA4
:10AE700008D9053B032B08D801231A4600B10370FB
:10AE80001046704700230122F8E700231A46F5E731
:10AE9000783B01202DE9F04FDFF8DC81DFF8DC9111
:10AEA000D8ED037A08F5B06399F8802EF8EE677A4A
:10AEB0002DED028BC3ED007A83B0002A4ED1614E96
:10AEC000C8F8882598F88C153278D9B1B9F8863E3B
:10AED0000024DFED5D5A07EE103ADFED5C6A5C4B53
:10AEE000B8EE477A67EEA66A03EBC10085EE876A83
:10AEF00036EE266A86EE867A1C60083303ED017A08
:10AF00009842F9D199F87E3E9FED525A06EE103ADA
:10AF100096F8583B9FED507A1A44B8EEC66A27EE71
:10AF2000877ADFED4E6A12FB01F14D4AC5EE065AF3
:10AF3000C9B207EE901AF8EEE77AE7EE876AF7EE05
:10AF4000667AFCEEE77AC2ED005A17EE903A88F87E
:10AF5000DC3603B0BDEC028BBDE8F08FFCEEE77A87
:10AF60009FED404A99F8811EB9F8843EF8EE674A91
:10AF700006EE101A002107EE103A324EB8EE466A7D
:10AF8000C4EE245A0191B9F8821E01239FED365A6E
:10AF900006EE901AC6ED057A98F88C15B8EEC77AC9
:10AFA0009FED328AF8EE666AC8F88865327067EEFF
:10AFB000057A86ED016A88F88435C6ED036AC6ED28
:10AFC000047AC6ED025A89B3294B4FF0000B019960
:10AFD00003EB010A12B3AAF118045746002507EE45
:10AFE000905A01223846B0EE481AB8EEE70AD6ED7C
:10AFF000017AD6ED040A15447169283720EE270A34
:10B00000283452F0A5F984ED028A84ED018A84ED9A
:10B01000048A84ED038A32789542E0DB0BF1010B60
:10B0200098F88C150AF1780A8B45D3DB019B03F560
:10B030007073B3F5346F0193C5D10E4BD3ED007A25
:10B0400043E700BFD034002083F9223EBD37863568
:10B05000004A0120555555406E12833A48E1FA3EA8
:10B06000BC0800200060EA480AD7233C000000002A
:10B07000E834002064070020E4010020783B012030
:10B0800007EE900ADFEDAF5AAF4B0022B8EE677AB9
:10B09000DFEDAE4AB3F8C81E85EE874A06EE101AF9
:10B0A000B3F8CC1EDFEDAA5A07EE901AB3F8CA1E09
:10B0B000B8EE466A06EE901AF8EEE77AF8EEE66A1F
:10B0C00036EE065A67EEA47A2DE9F04FC6FE856A81
:10B0D000A04D2DED048BB4EEE54A05F5DC6993F83F
:10B0E000CE4E85B0C5F83007F1EE10FA89ED016A51
:10B0F000C5F8EC46C5F8F026C9ED026AC9ED007A3C
:10B1000002D51446C5F8EC26F6EE004A9FED925A99
:10B11000F7EE003A914927EE055A9FED912A64EE29
:10B12000247A0B46F0EE002A9FED8E3A143381ED1F
:10B13000045A87EEA67A01F5A677039301F12C064F
:10B1400091ED055A884A12F8542C87FE237ABDEEF9
:10B15000C77AF8EEC77A17EE103A012BC5F88C398A
:10B16000C4EE275AB8BF0123029383EEA74A65EEC7
:10B17000825A86EE257AA1EC014AC1ED005AC6EE4C
:10B18000A57A37EE247A87FE227ABDEEC77A77EE6B
:10B19000A47A17EE101AC7FEC37AFDEEE77A01F122
:10B1A000FF38C5F8981917EE901AB8F1230F01F17E
:10B1B0000100A8BF4FF02308C5F89C192328834637
:10B1C00028EAE878A8BF4FF0230B5B468045C8BF4C
:10B1D00043460093A3EB0803019362BB624B934683
:10B1E000DFED629AA3F1500A9FED619A07EE90BAE3
:10B1F0000BF1010B0AF1080AF8EEE78A68EEA98A5A
:10B20000B0EE680A44F036FFB0EE408AB0EE680A4D
:10B2100045F04EF9B0EE680A45F04AF928EE098A81
:10B2200020EE090ABBF1240F0AED028A0AED010A99
:10B23000DCD19FED505A019A00234F489446029A60
:10B240009FED4E7A9CFBF2FA0AF10101A2461446E8
:10B250008E460099324646F80C1C46E9053846E908
:10B2600002E4A2EC017A9742FBD13A4606F5107B44
:10B27000D0EDD67AD0F85CC3C2ED007A083242F83D
:10B2800004CC5A45F8D106F515763D4A07F51577F1
:10B290009642DFD1039BB6EE008A5446012283ED2D
:10B2A000005A4FF0000A374B4FF0000800932E4B26
:10B2B00003F8542C002C35DD09EB0A06DDF800B04C
:10B2C000002707EE907AD9ED016A99ED027A06EE31
:10B2D000104AF8EEE77A012237EE667AD5F8301791
:10B2E000B8EEC66A06F1540077EE887A1744B7EED6
:10B2F000001A283667EE877A87EE860A30EE260A2D
:10B30000ABEC010AD9ED000A52F022F8D5F8EC4670
:10B31000C6F84480BC42C6F84080C6F84C80C6F8E7
:10B320004880CEDC009B0AF1C80A1433BAF5167FB8
:10B33000009302D0D5F8EC46BCE705B0BDEC048B19
:10B34000BDE8F08F00247449783B01200AD7233CE4
:10B350000000FA44E40100209C534937740B00209C
:10B36000398E633C00000C42DC120020C3B8B23DB1
:10B3700072F97F3FBC297E3F70D3050800000000B2
:10B380009C120020D80800200848002302461178AB
:10B390000632022904D00133062BF8D10020704771
:10B3A00003EB430300EB4300704700BFC0190120CB
:10B3B0000021094B00B5084683B0C3F8D01E2AF01F
:10B3C00027F80422054B06200DEB020101932AF019
:10B3D00013F803B05DF804FB783B01205475C52ACF
:10B3E00070B5461E00F13105344614F8011F601E89
:10B3F000FF29A0EB060002D0C0B22AF009F8AC4247
:10B40000F3D1A02040F2E93446F02AF801210220CD
:10B4100029F0FEFF01E0013C04D04220FFF79AFC36
:10B420000028F8D16220FFF795FC1321242029F091
:10B43000EFFF2520092129F0EBFFA020BDE8704097
:10B4400046F00EB830B54CF205028DB0002304462C
:10B450000321ADF8002001AD01228DF802300B93DD
:10B460008DF814208DF82820CDF808D0CDE90633CA
:10B47000CDE90833CDE9035138F072FC204602A92A
:10B4800038F030FA204638F06BFC9DF806000DB01D
:10B4900030BD00BF2DE9F043734E83B0734C2422BE
:10B4A000002106F1380051F0E9FD002394F8D55E43
:10B4B000F365002D37D16E4FD7F8903043B39B6AB8
:10B4C00033B36C489847836813B3038800246A4FEA
:10B4D000013BBC4639469BB20878063103281BD095
:10B4E0000134062CF8D1002239780637022900F001
:10B4F0009D800132062AF7D1F16D052908D002FBA3
:10B5000001C20131F1650220002193801070518049
:10B51000284603B0BDE8F083062303FB0464638F71
:10B52000013B9BB2DFE704F6DC6794F8D40EC4F865
:10B53000D87E10B900254E4FBEE735F00DF9C4F89E
:10B54000E40E35F0D5F90028F4D02946384638F015
:10B55000CFFA05460028EDD0D4F8D83E454A986881
:10B56000C3F8942008B12023C3800D21404F35F04B
:10B570007DF9D4F8D83E4FF00109986835F0B6FA55
:10B580003E4838F0F3FAD4F8D83E024632209A808A
:10B59000C7F8B03087F8B49032F01AFB04234FF0AC
:10B5A000000C9F21D4F8D80E0DEB0302CDF804C097
:10B5B00038F03CFB9DF805809DF8043007F19000C1
:10B5C0004FEA08289DF8061048EA034848EA0108AF
:10B5D000414645F097FB00287FF46EAF4046FDF7EB
:10B5E00021FB034600287FF467AF9DF806009DF815
:10B5F000052000029DF8071040EA0240204A084357
:10B60000904217D0A7F89430A7F8A030C7E92633A6
:10B61000FDF708FB034600287FF44EAF94F8D40EE4
:10B620001D4635F099F838F03DF945E7062101FB54
:10B6300002C268E7134B4FF400314FF0006287F805
:10B64000A290C7F894304023C7E92612A7F8A0308B
:10B65000FCF7E0FD07F1900087F8A99045F09EFA0D
:10B66000094BC7F8903027E788190120783B012063
:10B67000802A0120102B0120C0190120404B4C00D2
:10B6800021AAEF000004000870D305082DE9F04F4F
:10B690000423BE4C402141F21C1504F6746704F1EA
:10B6A00060064FF0A042636661670023022194F8B0
:10B6B0001D048BB0C4F8607466512266C4F89030E3
:10B6C0002367C4F88C30C4F88430A167E166C4E90C
:10B6D0001F33002800F0628103211F46164684F8BC
:10B6E0001D14936823F001039360F368304643F020
:10B6F0004003F36008F090F9B36B012F054643F463
:10B700008033B36317D005B3022384F81D34A04BF4
:10B7100093F8C450012D00F0FD80236E802101209C
:10B7200059625A6A42F480029A62FCF79BFD00203B
:10B730000BB0BDE8F08FB36843F00603B360B368A5
:10B7400043F02003B360002DDED1236E3220DA688F
:10B7500022F0C042DA60DA6842F08042DA600AF031
:10B7600081FA606E50B32A4601272946C2EBC20314
:10B77000561C04EB830383F89C20A3F8A220F2B2AA
:10B7800083F89D70824283F89F10C3F8B010C3E91C
:10B790002911EBD300221146C2EBC203561C04EB65
:10B7A000830383F85C22F2B283F85D12824283F84D
:10B7B0005F12C3F87012C3E99911EDD30022236E12
:10B7C000D4F86CC01646D4F87080D4F88CE0D4E974
:10B7D0001E71019102F14001013203EB81010F2A38
:10B7E0004E60F7D19A6BBEF1000F40F0438122F416
:10B7F00000129A631A6842F040021A601A6842F016
:10B8000080021A600022012F03F50066C3F8002EA3
:10B81000D3F80028C3F80028D3F8002800F02181CD
:10B82000032F00F01E8142F00302C3F800284FF4FA
:10B830008461584A196102E0013A00F032811969C5
:10B840008F06F9D41021534A196102E0013A00F041
:10B8500026811969C906F9D4002131617161F1614C
:10B86000E0B103F510624FF0904A4FF0006B0F46C5
:10B870004FF67F399C4607E0176001311761C2F827
:10B8800008902032814261D01368002BF4DA11B1A4
:10B89000C2F800A0F1E7C2F800B0EEE73269B8F1F3
:10B8A000010F22F48072326100F0ED8000216FF010
:10B8B000804299615A61B8F1000F03D19A6942F050
:10B8C00010029A619969344A0A439A61019A1AB13D
:10B8D0009A6942F008029A61BEF1010F00F0CE8031
:10B8E000002D7FF411AF0121D4F8842084F8985002
:10B8F0008A4284F81D1400F0D6807368032043F058
:10B90000020373600AF0AEF9214B93F8C450012D85
:10B910007FF403AF44F012FE00287FF4FEAE236EE6
:10B920008022284640215A625A6A42F400129A62E2
:10B93000FCF798FC20210220FCF794FC4021032016
:10B94000FCF790FC00200BB0BDE8F08F00216346AF
:10B950000CF530624FF0904A4FF0006B0F464FF6F7
:10B960007F39844607E0176001311761C2F80890FB
:10B970002032614592D010680028F4DA11B1C2F883
:10B9800000A0F1E7C2F800B0EEE700BF881901207F
:10B99000802A0120400D030000383C8000F0FF05A4
:10B9A0004C4B03204FF4C05684F81C541A6B42F0E1
:10B9B00001021A630A221B6B069105A903F0010319
:10B9C000089045480493049B07950596099206F054
:10B9D000DDFED4F88C30012B72D03E4B0621432083
:10B9E0005A6B42F080025A635A6B02F08002029254
:10B9F000029A5A6C42F480425A645B6C03F48043AE
:10BA00000393039BFDF766FF266E0323334A082149
:10BA1000916084F81D34A26FB368012A276F23F068
:10BA20000103B3607FF461AEB26B2D4B22F4803220
:10BA3000D4F89410B2630129F26803EA0203F360B8
:10BA4000F36823F44013F36003D1F36843F48013E5
:10BA5000F360304607F0E0FF012F05467FF453AE58
:10BA600069E6BCF1000F3FF4E0AE42F00102C3F81A
:10BA70000028DCE642F400129A63C3E69969194A89
:10BA80000A439A612CE718490020184A31636FF085
:10BA90008041376B3A4332639861596112E701255F
:10BAA000DAE60125CEE684F854549969C4F85C249A
:10BAB00041F000610E4A9961596D0A435A651CE7CD
:10BAC0004FF4007305A904480593CDE9065506F027
:10BAD0005DFE82E7003802400000024000E100E025
:10BAE000BFFFBDFF04000040000180000300010013
:10BAF0000300001010B51A4C94F8750FC0B9194B1B
:10BB000083F8B505C3F8B80594F8783F012B05D044
:10BB1000022B21D0D4F87C3F1BB910BD124BC4F8C6
:10BB20007C3F12495B68A1F10C00BDE8104018474A
:10BB300034F012FE94F8772F0A49003AC1F8B8059C
:10BB400018BF012281F8B5250028DDD01F22202151
:10BB5000C28034F08BFED7E7054BC4F87C3FE0E7AA
:10BB6000783B01208819012084010120F84A012036
:10BB70006001012099B10A6B824216D9154BD3F8A6
:10BB8000C42F914221D34C3991421ED30B6B984262
:10BB9000F9D38B6B9842F6D80B46184670470D4B7D
:10BBA000D3F8C41F0A6B904212D30B680BB9F4E7A9
:10BBB0000A6B90420B4602D38A6B9042EDD951F842
:10BBC0004C3F002BF4D118467047002318467047AD
:10BBD0000A46D8E7783B01202DE9F047CC0143D154
:10BBE000034622494FF0FF32022443F8081B7E2609
:10BBF00042601846DFF878802644051D6FF07047D4
:10BC0000D8F8C89F4FF0010A013E494608E0A34218
:10BC10001CD0631C45F8043C321B1C460435CAB1D9
:10BC20000B6BA34202D88B6BA34204D22046FFF7D2
:10BC3000A1FF014690B10A794B6B002AE7D1A342DC
:10BC400004D0E6D2631C45F8042CE5E7631C45F8F4
:10BC5000047CE1E7C8F8C81FBDE8F087321B631C0D
:10BC6000494645F804ACD8E78026C3E7F8FFFF0F44
:10BC7000783B01200A44914219D0013910B4541E76
:10BC800011F8012F0823504002E0013BD0B209D047
:10BC900010F0800F4FEA4002F7D082F0D500013B50
:10BCA000C0B2F5D1A142EBD15DF8044B70477047AB
:10BCB000194A00232DE9F04702F6DC7484B00546EA
:10BCC00092F9D58F1F46461804F5287A4FF0B60929
:10BCD000D4F800C0204600226946E034BCF1000FD1
:10BCE00014D09CF838C0BCF1140F0FD018F1020F1B
:10BCF00001D0C4450AD1CDE90277CDE90056ADF8AF
:10BD000008908DF80D702AF0CDFA0346A245DFD1D8
:10BD1000184604B0BDE8F087783B01202DE9F047D4
:10BD20009AB004460D4617469846DDF89090DDE936
:10BD3000226A02E0206831F0BDFF206831F0C2FFC6
:10BD40000028F7D10146642201A851F097F9264B4B
:10BD50008DF80450CDF85CA00293002D3FD0AB1EAF
:10BD6000012B3ED9042D14BF002303231F4A8DF855
:10BD700005300123926A039616448DF85B30CDE9B5
:10BD80000594049637B14246394607A851F004F9A4
:10BD90008DF85A80164E002396F8C6911893B9F183
:10BDA000000F19D196F8C501642201A902FB0060B9
:10BDB00000F5E47051F0F0F8012386F8C59186F89B
:10BDC000C631236843B143463A46294620461AB055
:10BDD000BDE8F04717F080B81AB0BDE8F08705233A
:10BDE000C4E70223C2E700BFF44D0120802A0120EE
:10BDF000704C01200C480D4BD0F8481210B48A1E2C
:10BE00000B4C2231C0F83832B0F866321B01A4FB6B
:10BE100003C3DB08A3F5B06322F8023F9142F3D1DC
:10BE20005DF8044B704700BF704C01201D70020884
:10BE3000CDCCCCCC70B5084C251D2E4614F8010B8A
:10BE40002AF004FC28B10378B44205F8013BF5D18F
:10BE500070BDFF23F8E700BFFC4E01202DE9F0473D
:10BE60001C4F01264FF03C094FF0000807F1080570
:10BE7000B24617F8010B34F06FFC044690B180F81D
:10BE80000690C671FB7803F07F02012A17D013F0E9
:10BE9000800F20460CD185F8048034F021FE85F80F
:10BEA00005802C6001360835052EE2D1BDE8F0870B
:10BEB00085F804A034F01AFE85F805A0F1E71B060A
:10BEC00005D40121204634F0D1FCFB78DFE734F0C3
:10BED0000DFEF6E7044F01202DE9F047204E82B019
:10BEE00000244FF00409DFF87C8006F10C05A6F56C
:10BEF000307716F801AB5046BAF1000F2CD034F071
:10BF00002BFC0134034604215046E4B26B6113B1AB
:10BF100083F80690DC71224631F0EEFB0221824666
:10BF2000D0B168699AF8082034F068FCB7F8BE32DE
:10BF3000B7F8BCC2002051460A4A01902846CDF805
:10BF400000C01835B8FBF3F39BB229F07BFA01234C
:10BF5000082C05F8073CCCD102B0BDE8F08700BF43
:10BF6000304F012040420F002DE9F041204C0023CA
:10BF70004FF0050894F8932304F5647704F565758C
:10BF800084F88C2317F8010B5E1C20BB2860032E5D
:10BF900005F104053346F5D194F88C13D4F89403D5
:10BFA000C94301F0010134F055FE94F88C13D4F824
:10BFB000980381F00201C1F3400134F04BFE94F884
:10BFC0008C13D4F89C0381F00401BDE8F041C1F367
:10BFD000800134F03FBE34F0BFFB0121F3B2286092
:10BFE00010B180F80680C371286834F03FFCCEE7BA
:10BFF000704C0120F0B5294C83B0B4F8A453A4F8D8
:10C00000A653EDB994F8A00334F0A6FB94F8A1234D
:10C01000C4F8A803003A18BF012284F8AC2348B141
:10C0200094F8A2132B220029C28014BF11210121F0
:10C0300034F01CFC002003B0BDE8F04034F012BE28
:10C0400094F8A07300222B21384631F055FB0646A8
:10C05000384634F081FB00B10EB903B0F0BD2B229D
:10C06000C4F8C40302210027C280327A34F0C6FB30
:10C070000B4AA4F8C853314604F56C700197B2FB23
:10C08000F5F3C3F34F059BB2009529F0DBF9D4F823
:10C09000B0331F6084F8C173DFE700BF704C01202C
:10C0A00040420F002DE9F84F264B002693F8D42389
:10C0B00003F2CB3703F57A7483F8CA235FFA86FB61
:10C0C0004FF0010917F8010F01360BEB090A494639
:10C0D0004FF000085FFA8AFA524631F00DFB054630
:10C0E00048B3387804F80E8C04F80D8C04F80FBCB3
:10C0F00004F8109C44F8045C34F02EFB022118B1C3
:10C1000080F8069080F807A02A7A34F077FB0E4A70
:10C11000002128464CF090F90C4B221D214623604B
:10C1200028460B4BC4E901384CF052F84246697975
:10C13000286829F0D5F8082E04F11C04BED1BDE80A
:10C14000F88F00BF704C012040420F009553030848
:10C15000D1FB020870B52C4C00222C4B022194F824
:10C160000005C4F8F834C4F8B824C4F8BC24C4F8F2
:10C17000C024C4F8F424A4F8FC2431F0BDFA00284B
:10C1800041D0234B0546026803F1C000597C11B130
:10C1900059688A422CD018338342F7D1002394F88F
:10C1A0000005C4F8E45384F8D83334F0D5FA08B164
:10C1B0000223C38000262A7A022134F01FFB314675
:10C1C0002846144A4CF038F9134B144A2846C4F850
:10C1D000E833134B111FC4F8F063C4F8EC334BF091
:10C1E000F7FF324669792868BDE8704029F078B8D1
:10C1F000926A0C4801320C49D0F87431B3FBF2F367
:10C2000081F8A831CAE770BD704C012000FFFF0023
:10C21000AC13002040420F00F9FB02085C500120E3
:10C2200095FD0208802A0120000001202DE9F04F31
:10C23000DFF878B180460B46DFF874A10BF1D0002F
:10C24000C02200212DED068B97B0CDE9023850F0C9
:10C2500015FF9AF80185B8F1000F00F095829AF861
:10C2600002350893002B00F0CE82DFF8489199F850
:10C270006C3E012B00F0ED82022B00F0E5820BF505
:10C28000FC73444D99F8626E1C460F930FCD0FC49A
:10C290000FCD0FC4311E404A99F85E3E18BF0121F0
:10C2A000CBF81022072B8BF8301295E8070084E8B2
:10C2B000070000F25D83042B0ED999F8613E374ADE
:10C2C000012BCBF8382205D09A1E53425341002E41
:10C2D00018BF00238BF83C320023DFF8DCA0039367
:10C2E0002F4B04932F4B0593DDE90232934240F329
:10C2F000B081059B032113F8015B059309EB05034E
:10C30000013593F8636EEDB230462A4631F0F4F908
:10C310000446002800F02283304634F01DFA049BC6
:10C32000586110B10323C571837199F85E2E99F895
:10C330005F3EE77906920BB187F00107204637F0A0
:10C34000A7F90346002800F006839BF83C220792D9
:10C35000002A40F01883D0F80480B8F1000F00F0F4
:10C36000FD829B6840460B9337F0FAF92A46032179
:10C370000A9037F005FA002800F0F0829BF840623E
:10C3800025680948CAF89480002E00F0278300230E
:10C39000024617E020D80508398E05086D410408CB
:10C3A000AC130020E649012020150020DC120020FB
:10C3B000704C0120783B0120A02600200133B342BD
:10C3C00000F00C831168B8328D42F7D1DEB2B82389
:10C3D0009BF84022039906FB0303013A8AF81110E7
:10C3E000CAF898302079099234F0B6F907F00101C3
:10C3F0009BF8303201310BB187F001074901CAF8CF
:10C40000084041F00E01CAF81410227A34F0F6F90F
:10C41000099B9E4200F01E84069B063B0C93002362
:10C4200060220AF16401CAF8803008EE101ACAF8D6
:10C430006420CAE91A33CAE91C33CAE91E3317F06B
:10C4400002034FEA47070D9300F0E082012307F053
:10C450000207CAF86C30CAF87870002702234FF43C
:10C4600080310A22CAF87070CAF88420CAF8903065
:10C47000CAE9221763790C2B00F2BE82CB4A9BF8E3
:10C480003C1202EB8302D2F80874CAF854700029F7
:10C4900000F0F982DAF89830C3F8A880CAF89480DE
:10C4A000079B002B00F073830AF118000E9007F031
:10C4B000F1F89BF83C320E98002B00F08E83BC49BB
:10C4C0004FF4907322684FF0030C03FB0613DAF865
:10C4D00098104C32C1F8B030CAF81C300B9BCAF827
:10C4E0001820CAF83C30CAF848C0069B40214FF4D7
:10C4F000806C082B4FF00403CAF820104FF48051D1
:10C50000CAF844304FF000030CBF06221222CAE9D9
:10C510001333CAE909334FF40033CAF838204FF413
:10C520008042CAF84030079BCAF83420CAE90BC1E0
:10C53000002B00F040839DF83030CAF89480022B25
:10C5400000F25582994A9B4902EB8303069AD3F87D
:10C55000FC33082AB1FBF3F308BF5F2203F1230386
:10C5600018BF1322CAF85C30DAF8983050469A8027
:10C570004CF0D2FB9BF83C32002B00F02782079B4B
:10C58000002B00F0238218EE102A3946284605F0C9
:10C590002FFF012F00F0EC82042F00F05383102FA7
:10C5A00000F08682402F00F0AB83B7F5807F00F06B
:10C5B000B583B7F5806F00F0B983B7F5805F00F001
:10C5C000BD83B7F5803F00F0C1836A6D05F11800A7
:10C5D000082342F400626A6577490422DFF800C24A
:10C5E000C95C1CF803C00B5802FA0CF223EA0203E0
:10C5F0000B502B6843F001032B600D9B002B00F0C8
:10C60000B3822B6A43EA87072F62099B9E420BD1B4
:10C610006B6C43F400436B642B6843F080032B6026
:10C620002B6843F001032B609BF83032002B40F065
:10C63000A782039A012304990AF1A00A01320AF899
:10C64000913C4B7401F11803082A039204937FF480
:10C650004BAE0F9B89E1DFED598A594AB0EE688AEB
:10C66000584BCBF8AC210022CBF8A831564BCDF873
:10C670001080039238EE887ADFED547AF5EE006A86
:10C68000534C28EE278ADFF85CA1B0EE67AA00279A
:10C69000C6EE879A9FED4F9ACBF8B431CDF814804F
:10C6A000029BBB426DD01AF8015B032109EB050325
:10C6B000013593F8638EEDB240462A4631F01CF8FE
:10C6C0000646002800F0B782404634F045F8606125
:10C6D00010B10323C5718371327A022134F08EF8D0
:10C6E000049B002B00F0EE81B9F85C3E4FF6FF7121
:10C6F00007EE903A384BF8EEE77AD3F87421FCEE67
:10C70000E77A17EE903AB2FBF3F00144090CB2FB62
:10C71000F1F2B2FBF3F399F85E1E042900F0E48114
:10C7200007EE902AF8EE676A26EE887A69EE477A75
:10C7300099F85F0E03999BB201902046E6EEA87A25
:10C740000091314684ED027AC4ED037A28F07AFE36
:10C75000002F40F3B58161681D4B02E09C4200F060
:10C76000AF815A6818338A42F8D1059B013783F0AC
:10C77000010301221834082F04F8083C04F8072CA0
:10C780008ED1164ECBF82C62DBF82C3263B300222C
:10C790000121029883F82D1083F82C001A6383F886
:10C7A0002E2017B0BDEC068BBDE8F08F70D30508C6
:10C7B000E01A002000D0121368D80508000000001D
:10C7C000A50203080DC4030801C403086F12833ACD
:10C7D000AC13002000007A44802A01206C14002051
:10C7E0005CD80508E6490120C54DC64C0FCD0FC4E5
:10C7F0000FCD0FC495E80700A4F1200384E80700DB
:10C80000CBF82C32CDE7C04D0BF5C874DFF854934C
:10C810000FCD0FC40FCD0FC495E8070099F85E3E09
:10C8200099F8606E84E80700042B00F23C8101A2B5
:10C8300052F823F051CA0008A7CA000847CA0008E6
:10C8400025CA000857C6000899F85E3E082B00F07C
:10C850000281029B0026AD4DCBF83432AC4C99F8E6
:10C860005E7E8AF804658AF83C750FCD0FC40FCD43
:10C870000FC499F8623EA4F58A729B1B049295E856
:10C88000070018BF0123354684E8070031464FF4FE
:10C890004C72A0488BF8303250F0F0FB9E4BDDF824
:10C8A00010809E4E0393CDF810900AE034F018F9F2
:10C8B000F368082D06F1200608F1180848F8043C32
:10C8C0005DD0DBF83432AB4259DD039A12F8013BFC
:10C8D0000392049A134493F8637E384630F094FF31
:10C8E0000446384633F038FF049A8146E77992F8D7
:10C8F0005F2E0AB187F0010707F001049BF8302290
:10C9000001348AF803450AB187F00107484633F03D
:10C91000EFFF002800F084814846013536F02CFEF8
:10C92000C6F80C9061017060EAB2377441F0010101
:10C930007161B9F1000F05D04FF0030389F80720AA
:10C9400089F80630484633F091FFF9074846ADD4E0
:10C9500034F0CCF8ACE79BF83C32A3B97049002323
:10C96000704ACBF81412CBF81C22CBF82C320BE710
:10C97000082B7FF4B1AC6C4BCBF83832ACE4644894
:10C98000CBF82C0200E7D4F81480B8F1000FE5D002
:10C99000A36940460B9336F0E3FE644B2422451E08
:10C9A0000A9002FB053595F8C831392B00F02C812F
:10C9B00020684BF0AFFD024639210A98D2B236F01A
:10C9C000DFFE0028CAD000230793D7E40A989022FC
:10C9D0009AF8113056494DF07DF9D4E5B823721C10
:10C9E00003FB06B38BF84022C3F84452EFE48D23D7
:10C9F0001322CAF85C30B7E59BF83C32CAF8547091
:10CA0000002B7FF447AD1F461A4641E001224FF448
:10CA1000807307F00207CAF86820CAF87C30CAF8A9
:10CA200074701AE59FED438ADFED438A002E3D4A7C
:10CA3000424B16BF414600211346414A04914149E9
:10CA4000CBE96A2116E69FED408AF0EE488AEDE7D1
:10CA5000DFED3E8A01E60BF5FC733D4D99F8626E01
:10CA60001C460F93003E0FCD0FC40FCD18BF0126FB
:10CA70000FC4384B8BF83062CBF8103295E80700C2
:10CA800084E8070077E7344A02EB4303B3F83C2419
:10CA9000DAF89810AAF80C20B1F8B43023EA0203AF
:10CAA000A1F8B430FCE49FED2D8AF0EE488ABDE792
:10CAB000AA6905F11800022342F40062AA618BE51D
:10CAC000002353E6FAFE697AFCEEE77A244B17EE70
:10CAD000901AD3F874214FF6FF73B2FBF1F11944A9
:10CAE000090CB2FBF1F216E607EE903AB8EE677A5F
:10CAF00007EE902AF8EE676A27EE0A7A16E600BF7C
:10CB0000C8D7050878510120D0D60508F4D7050804
:10CB1000A0140020A02B0020E6490120D02E0020E8
:10CB200009C4030801C403083941040800000120B6
:10CB300095370000ACC5A737ACC5A73601FE020883
:10CB40000DC40308A5020308282930386F12833A60
:10CB500020D80508398E050870D305086F120339EF
:10CB6000802A0120783B01202B6A1F432F624CE56D
:10CB7000AA6905F11800002342F00802AA612BE51A
:10CB800023684FF6FF7162793433995051E5D8F834
:10CB900000205FFA88F3182128F0FF0022F001023C
:10CBA000103BC8F80020B3FBF1F106F0CBFD0A986A
:10CBB0004DF0B6F878E45FFA88F31821024628F0C1
:10CBC000FF00103BB3FBF1F106F076FDD8F8003022
:10CBD00043F01003C8F80030ADE40B9A5821DFF899
:10CBE000A0C1CAF83C20039A01FB02C12268CAF81E
:10CBF0004830CAF89C1002F13403CAF81C1062795C
:10CC00001344CAF8183070E420684BF083FC95F8A0
:10CC1000C93183427FF4CCAE089B0793FFF7AEBBCC
:10CC20004E4B01224E498AF80425CBE977314D4B12
:10CC3000CBF8E831A4E64C4A4A4BCBF8AC21CBF810
:10CC4000B4319FE5AA6905F11800012342F00802FA
:10CC5000AA61C1E400224FF0FF311346ADF8442031
:10CC6000129214928DF854201391404A52F83320B6
:10CC700095424DD001330E2BF7D10020069B9A1F11
:10CC80000C92FCF7DFFE2B6839499DF8302023F029
:10CC90000103D1ED5D7A022A2B60F8EE677A22D883
:10CCA0003449DFED356A01EB820292EDFF7AB8EE8E
:10CCB000477A87EE870A30EE260A4EF0FBFE069B87
:10CCC0000138082BADF8440014BF13225F22002363
:10CCD00011A92846139214938DF85430129305F03D
:10CCE000D9FCFFF79CBB9FED257A9FED230AA7EEA9
:10CCF000870A4EF0DFFE01381322ADF84400E6E764
:10CD0000AA6905F11800032342F00802AA6163E44E
:10CD1000184A02EBC30393F89003AFE7EA6905F101
:10CD20001800042342F00802EA6155E4EA6905F1BB
:10CD30001800052342F00802EA614DE4EA6905F1B2
:10CD40001800062342F40062EA6145E46A6D05F1C9
:10CD50001800072342F008026A653DE40DC4030889
:10CD600009C4030801C403080DFF0208FCD6050826
:10CD7000802A012070D305080AD7233CFCF4B23482
:10CD8000E023002070B5524E96F8600233F0E4FCC8
:10CD900096F8615260B12D2304462021C38033F000
:10CDA00065FD0A2030F008FF204636F0DBFB18B99D
:10CDB000D6F84035DA0000D570BD013D092DFBD80D
:10CDC00096F85F42CCB940202BF052FA0028F3D0FD
:10CDD00090F9043096F83112092BC8BF143B0A2988
:10CDE000334493F8444566D093F8503596F85E2264
:10CDF000002A08BF1C46002CDED0204633F0ACFCD5
:10CE0000054608B12D23C3800121284633F02EFDAD
:10CE10000121084633F068FF0121284633F01AFF4C
:10CE20003C2030F0D5FE0021012033F05DFF96F864
:10CE300061321BB3002400210134084633F054FF53
:10CE40000021022033F050FF0021284633F002FF7A
:10CE5000782030F0B1FE0121002033F045FF0121A0
:10CE6000022033F041FF0121284633F0F3FE782001
:10CE700030F0A2FE96F861329C42DCDB96F85F321D
:10CE80008BB9D6F8603203F0FF13B3F5803F93D12E
:10CE9000D6F8403513F080538ED186F86132BDE864
:10CEA000704043F02FBA322030F092FE2846002125
:10CEB00033F0DCFCE5E7D6F868355B057FF57CAF41
:10CEC0000EF072FC00287FF477AF002C95D173E749
:10CED000704C012030B40438043A0C1F01F10805ED
:10CEE00054F8043F52F8041FAC42A3EB010340F88E
:10CEF000043FF5D130BC704738B5041E0D4611DB38
:10CF0000092C1FDC0846134B0021134AA3FB04C362
:10CF10004170DB0803EB8303A4EB4303D35C037092
:10CF2000284638BD64422D230846092C00F8013BF1
:10CF3000E9D9084B01460A22A3FB0430C00842F09D
:10CF400009F9E0E703480A22A0FB0430C00842F0D8
:10CF500001F9D8E7CDCCCCCCDC5C0608344870B401
:10CF600090F86C35A3F13001092958D800F26C54BF
:10CF700000F27B50224612F8015FA5F13001092929
:10CF800004D88242F7D1002070BC7047141B022CD9
:10CF90004BDD2848002101E010F8013B01EB810145
:10CFA000161A044603EB4103022EA3F1300303F0EB
:10CFB000FF01F1DC204B03FB01F1A2424FF0000323
:10CFC0000ED903EB830314F8016B5B00A242A3F1BB
:10CFD0003003334403F0FF03F3D1184800FB03F39D
:10CFE0002E2D06D01648A0FB032370BC01EB930046
:10CFF000704701320425002404EB84041078013DBD
:10D00000303864000928A4B2204401D8013284B227
:10D0100015F0FF05F0D1642202FB0433E2E70021A2
:10D020001D4600F26C520B46DAE70021054CC4E7BE
:10D03000704C0120DD5101208096980040420F0085
:10D04000ABAAAAAADC51012038B50D460446FF213F
:10D0500000682A4650F012F822682A44226038BD3F
:10D060000C461646054683B529F07CFB204629F080
:10D0700079FB0021204B0846002E08BF1E4633F0E6
:10D0800033FE0021012033F02FFE284630F01AFE37
:10D09000B0B10121002033F027FE284630F00AFE0F
:10D0A0000746204630F00AFE0028FAD039462046CE
:10D0B00030F02EFE3846B0470021084633F014FE0B
:10D0C000204630F0FFFD0028DFD00121002033F0A2
:10D0D0000BFE204630F0EEFD01462846019130F06F
:10D0E000EDFD01990028F8D0284630F011FE00210E
:10D0F000084633F0F9FDC8E7B5570308F0B500223C
:10D1000089B0234E04AF13460A61BC46C1E9002230
:10D11000C1E902220268C2F3855040FA03F4654671
:10D12000E40703D59C5D05F8014BAC460133062BA3
:10D13000F3D1184DC2F303240023C2F305302C5D54
:10D140000DF119068CF80030DFF850C08DF818404A
:10D1500040FA03F43546E40704D513F80C4005F80B
:10D16000014B2E460133062BF2D10023C2F3834537
:10D1700006AC0846337002F00F030749C2F30312EE
:10D180000097CDE9014542F0E9FD09B0F0BD00BFCF
:10D19000245D06081C5D0608045D0608145D06088B
:10D1A00070B5094C0546D4F87C2562B100260136DD
:10D1B0002D21D4F87C0538F02FF8AE42F7DBBDE81E
:10D1C000704038F0D3BA70BD704C012038B50546B8
:10D1D000084641F06DFE041E0D4B0FDB93F88C25C5
:10D1E000944205DA21460B4839F0F0FD204638BD5F
:10D1F000FF2C03D1084839F0E9FDF7E793F88C25B7
:10D20000284606494FF0FF34013A38F075FAEDE749
:10D21000E4010020345D0608455D0608585D0608F7
:10D2200030B583B04D1C0093002304688572C27230
:10D23000A469A04703B030BD03685B6C0BB1022149
:10D240001847704770B5104ED6F82C3293F82E2040
:10D25000CAB19B699847B0B1D6F82C3293F82C200C
:10D260006AB10A4D0024DB69E0B2B5EC010A013471
:10D270009847D6F82C3293F82C209442F3DB5B6A63
:10D28000BDE87040184770BDDC12002060300020FF
:10D2900038B51E4C0968D4F884550068491B1C4DEC
:10D2A000DFED1C6A00EE901AD4F88015D5EDFB7AFC
:10D2B0001C46F8EEE00A401A60EEA70A07EE900A54
:10D2C000F8EEE77A20EEA07AB1EE670AA7EEA77A29
:10D2D000F1EEC77A67EEA67AFCEEE77AC2ED007A45
:10D2E00042F06AFE9FED0C7ADFED0C7AE0EE077AF1
:10D2F000FDEEE77A17EE902A002A02DBC4ED007AF1
:10D3000038BD48F6A0431344236038BD704C01205B
:10D31000000001202C7D8E3FA00CB34500A00C46E0
:10D3200038B50F4C034694F89F1504F5B36084F8A4
:10D330009B3501F03F0101F10A058B1C083184F88F
:10D340009A55254484F89D351FF0C4FC85F8960550
:10D3500094F89A35000A1C4484F8970538BD00BF3C
:10D36000704C012038B50A4C00250122802120464E
:10D370002AF06AFF30B194F904002AF099FF08B14D
:10D38000006838BD01350C34092DEED10020F8E7D6
:10D390003052012038B5041F00F1080554F8043F4D
:10D3A000D81780EA430018F065FCA542F6D138BDD5
:10D3B000074B4FF6FF70002103F6AC4210B4002477
:10D3C000C3F8280D5167C3F8244D5DF8044B70472E
:10D3D000D4230020F8B5794CDFED797AD4F8302DDC
:10D3E00094F8103D07EE102AB4F8127D2DED028B53
:10D3F000B8EE478A28EE278A002B68D1D4F81C6D36
:10D4000094F82D1D304626F097FC0F2894F8113D16
:10D41000B8BF0F2085B2A4F8125D002B00F0BB80CE
:10D42000AF4258D094F8AC6CB4F8143D07EE905A63
:10D43000DFED645A002206EE103AF8EE677A624990
:10D440000020B8EE466AC5EEA76A0B4685EE867ADE
:10D4500076EE886AC8EE267A37EE087AC8EE076A52
:10D4600096BB58609860D860C3ED047A01321033DF
:10D47000032AF5D1002E34D094F8163DB4F8185D87
:10D48000C1ED106AC1ED147AC1ED187A002B7CD180
:10D4900094F82D1DD4F81C0D26F04EFC0F28B8BFB3
:10D4A0000F2080B28542A4F8180D6ED000286CD0F1
:10D4B00007EE900ADFED436A444BF8EE677A86EE9A
:10D4C000A77AD3ED006A56E0C3ED047ACEE794F86C
:10D4D000113D002B5CD094F8AC6C002E66D13D461B
:10D4E000A2E7002394F8162DB4F8185DC1ED106A78
:10D4F000C1ED147AC1ED187A4B638B63CB634B6437
:10D500008B64CB644B658B65CB6562B994F82D1D3C
:10D51000D4F81C0D26F010FC0F28B8BF0F2080B2E5
:10D520000546A4F8180D41F26D0394F82C2DE25431
:10D530005DB307EE905A254BDFED226A0022F8EE2C
:10D54000677A41F26C010120C3F80823C3F80C2369
:10D5500086EEA77AD3ED006AC3F81023C3F8182328
:10D56000C3F81C23C3F82023C3F82823C3F82C23B3
:10D57000C3F83023605437EE267AC6EE877AC3EDBF
:10D58000C57AC3EDC97AC3EDCD7ABDEC028BF8BD87
:10D59000D4F81C6D3D46304694F82E1D26F0CCFB89
:10D5A0000F28B8BF0F20A4F8140D39E794F8163DE2
:10D5B000B4F8185D002B3FF46BAFE6E7D4230020EE
:10D5C000BD3786354E2DA63D803000200831002025
:10D5D000012817D0304A41F29303D35C012B2DD0A0
:10D5E0002E4BF6EE006ABEEE007ADFED2D7A03EBED
:10D5F000800090ED000A80FE660A80FE070A20EE99
:10D60000270A7047274A41F294032349F6EE006A3D
:10D6100002F5C960BEEE007ADFED217A90ED010AD5
:10D62000CB5C80FE660A80FE070A20EE270A23B143
:10D63000B5EEC00AF1EE10FA03DC70479FED1A0A4E
:10D64000704707EE903AB2F93216B2F94636DFED7E
:10D65000176AF8EEE77ACB1A07EE103AB8EEC77AF7
:10D6600027EE267AB4EEE77AF1EE10FAE6DA77EEF4
:10D67000C77AB2EE047AF4EEC77AF1EE10FADCD88B
:10D68000B1EE047A67EEA67A30EE470AA7EE807A0A
:10D69000B0EE470A704700BFD4230020B8520120E3
:10D6A00000004843704C012000000000CDCCCC3D70
:10D6B000F8B5744B40F60301B3F854260A402DED3B
:10D6C000048BB0EE408A04D0B0EE480ABDEC048B67
:10D6D000F8BD03EB4003B5EEC00ADFED6B7A00F155
:10D6E000D40EB3F93016B3F94436F1EE10FA674DA3
:10D6F000A1EB030305EB8E0CC8BF012600EE103A28
:10D70000D8BF4FF0FF36DCF8344D05F63457B8EE8D
:10D71000C00A20EE270AB5EEC00AF0EEC07AF1EE9C
:10D7200010FACCBF01214FF0FF31A31B18BF01231A
:10D73000002C08BF0023002B49D197EDCF7AF4EEDF
:10D74000C77AF1EE10FA07DD8E4208BF002C0CBF3D
:10D750000123002300F08180002C42D007EE901AB4
:10D76000B0EE408AD7EDD25AF8EEE77A9FED486ADC
:10D77000DFED486ADFED488A97EE878A28EE258A32
:10D7800088FE468A88FE268A002B58D141F278030B
:10D79000EB5C984298D1414D95F8983D262B93D15A
:10D7A000B2EE049A20EE090A4EF084F9B0EE480A6F
:10D7B000A5F89E4DA5F89C0D4EF07CF928EE890A3F
:10D7C000A5F8A00D4EF076F9A5F8A20D7CE797ED2F
:10D7D000CF7ACCF8342DF4EEC77AF1EE10FA3ADCB9
:10D7E00013462F4A9FED2F6A02EB8002D2ED097A91
:10D7F000F0EEE76AF4EEC66AF1EE10FA28DC9FED6F
:10D800002A6A66EE866A97EDD06AF0EE408A67EE85
:10D81000867AE6EEA78AF5EEC08AF0EEE87AF1EEB7
:10D8200010FAF4EE477ACCBF01224FF0FF32F1EE4E
:10D8300010FA01DD964217D00024002BA6D01B4A17
:10D8400000EB8003002102EB830343F8341C9DE7C7
:10D85000F7EE006AD7E78E42C2D105EB8E0E0C467A
:10D860000123CEF8341D77E707EE902AB0EE688AE0
:10D87000D7EDD26A0024F8EEE77A97EE878A28EE91
:10D88000268ADCE7704C0120CDCCCC3DD42300208F
:10D8900000007A4400007AC400000000783B0120B8
:10D8A000E4010020FFFFF9436F12033BCC3400205A
:10D8B00070B504466F4EC0B22DED048BF0EE408A79
:10D8C0000D7820F07FFB6C4A06EB8403694207EE7B
:10D8D000905AD3F8583607EE101AF8EEE76A82FB32
:10D8E0000312DB17B8EEC77AC3EB621307EE903A68
:10D8F000F8EEE77AE6EE807AF4EEC77AF1EE10FA07
:10D9000005D407EE105AB8EE477A87FE677A06EB21
:10D910004404DFED5A9A40F60100B6F85426B4F9F3
:10D920003036B4F944161040A3EB010307EE903AE9
:10D93000F8EEE77AA7EEE97AB0EE478A07D0504BC7
:10D94000BDEC048B93ED7C0A27EE000A70BD20F03D
:10D9500039FB0120B0EE409A20F034FBB6F93036A6
:10D96000B0EEC00AB6F93216002B464AB0EEC99A9C
:10D97000B8BF5B42002992F8380FB8BF49429BB24A
:10D9800089FE009A89B28B42B8BF0B4607EE903AE7
:10D9900002F63453F8EEE77A67EEA97A50BBF7EE59
:10D9A000006A93ED807AB4EEE67AF1EE10FA50D484
:10D9B00093ED7E7ADFED347AB4EEE77AF1EE10FA89
:10D9C00044D9DFED325AB7EE006AC5EE876AB0EE91
:10D9D000467AA9EE667AC7FE466AC6FEA76AD3ED06
:10D9E0007D7AB0EE680A68EE277ABDEC048BA7EE6C
:10D9F000A60A70BD9FED246A93ED7E7AB4EEC67AD6
:10DA0000F1EE10FA1FDDD3ED7F5AF4EEC65AF1EEB7
:10DA100010FA18DDDFED1E6A75EEE77AB7EE005AF0
:10DA200029EE269AC7EEA56AC9EE077AC6FEC56A30
:10DA3000C6FE866A77EE857A66EEA76AC6FEC56A76
:10DA4000C6FE866ACBE7F0EE466AC8E7F0EE676A84
:10DA5000C5E776EEC76A9FED0F5A9FED0F6AD3EDCB
:10DA60007E5A66EE856A76EE677AA6EEA77A27EE8C
:10DA7000257A9FE7704C01201F85EB51CDCCCC3D22
:10DA800008310020D4230020000000000000C8421C
:10DA90000000C8C2610BB63B000034431C4991F83A
:10DAA0006C259AB3F0B40026054633463046374617
:10DAB0001BB991F86C452D2C22D02E2A18D0CA18EB
:10DAC00000EB800092F86C454000A4F13002092A76
:10DAD00002D8A0F13002A0180E2B14D80133CA18B6
:10DAE00092F86C25002AE3D106B14042F0BC7047A1
:10DAF0000133002DF8D0CA182A4482F86C75DEE78D
:10DB000001231E46EBE70020F0BC70470020704761
:10DB1000704C01202DE9F041A02301240B4F182562
:10DB2000E6B2FF2B0BDCC5F11B0103F10108324605
:10DB3000DBB2C9B2D7F86006FFF772FB4346013D7E
:10DB4000EFD10134052CEAD1BDE8F081704C012001
:10DB50001FB503AC8DF80C30002300948DF80D3008
:10DB60000EF0F0FC04B010BDF8B50546262023F0F9
:10DB7000F3FF144C014608BBD4F8640690F8383023
:10DB80001E3B012B02D894F871360BB130F0C0F86F
:10DB90000D4F0026AE4209DBB4F892360133A4F8EB
:10DBA00092360A4B9B6AC4F8A436F8BD17F8011BDD
:10DBB0000136D4F8640630F0ABF8EBE7002384F8C4
:10DBC000A036EEE7704C0120E2520120802A0120AD
:10DBD00010B51C2032F0C0FD0446112132F046FE83
:10DBE000204632F07DFFC8202FF0F2FF2046BDE82E
:10DBF000104032F07BBF00BF08B5002032F0ACFD12
:10DC0000054BC3F8A80608B12A23C3804021BDE80C
:10DC1000084032F02BBE00BF704C0120F8B56A4CB2
:10DC2000D4F834110B699E0702D5CB689D074BD4FD
:10DC30000B69580702D5CB685A073DD40B691B07FF
:10DC400002D5CB681F072FD40B69DE0602D5CB683F
:10DC5000DD0621D40B69D80702D5CB68DA073FD49B
:10DC60000B691B0603D5CB681F0600F191800B6979
:10DC7000DE0503D5CB681D0600F18E800B695C06BE
:10DC800003D5CB68580600F18B800B699A0602D544
:10DC9000CB689B0620D4F8BD6FF0100200230A6108
:10DCA000CA6984F85031D5E76FF0080200230A6191
:10DCB000CA6984F85031C7E76FF0040200230A6193
:10DCC0008A6984F85031B9E76FF0020200230A61D3
:10DCD0008A6984F85031ABE76FF020030B61F8BD1F
:10DCE0003A4B6FF0010299420A61B9D141F2041333
:10DCF0003748C558D5F81432002BB1D1354FD7F875
:10DD0000AC2692B1D0F858C602F03F066244C0F883
:10DD10005826D0F85826B2F5006F01D1C0F8583611
:10DD20000023C7F8AC36002E44D0D0F85826D0F8DF
:10DD30005C369A4294D0D0F85826D0F85C369A4295
:10DD400032D9D0F85866C6F50066D0F858C6B6F590
:10DD5000007F214A28BF4FF40076D5F81432624480
:10DD6000C5F81062C5F80822002B7FF479AF0123B3
:10DD700041F21C11C0F8A46EC5F814323346405865
:10DD8000812106F035F9D4F83411C7F8AC6667E79D
:10DD90006FF080030B616AE76FF480730B616DE7CE
:10DDA0006FF040030B6170E7D0F85C66D0F858362E
:10DDB000F61ACAE7D0F85826074BC5F81062134484
:10DDC000C5F808324CE700BF802A0120001400404B
:10DDD00088190120704C0120FC1F012070B5D0F87B
:10DDE000A852C1EBC1000C46002605EB80001C21A7
:10DDF000C0F80822C0F8103280F8FC41C0F8146264
:10DE000080F8FD612B6901FB0451012B01F5FE71C6
:10DE100008BFC0F80C22DAB228681CB905F042FE2F
:10DE2000002070BD05F0CAFE002070BD0E4841F212
:10DE30000413C35810B5A3B190F8844E00F6746073
:10DE4000D3F8042234B1002440230121FFF7C6FF98
:10DE5000204610BD4FF400730121FFF7BFFF20469D
:10DE600010BD0224204610BD8819012010B50C4CAD
:10DE7000D4F8603663B10B49013BD1F8B026C4F841
:10DE8000603612F8014BC1F8B026047013B10123BB
:10DE9000184610BDFFF7CAFF0123184610BD00BF8A
:10DEA00088190120704C012013B5074CD4F8B03606
:10DEB00003B9FEE701A8FFF7D9FF0028F6D09DF8C7
:10DEC000040002B010BD00BF704C012010B50B68FB
:10DED000064C074AC4F86036C2F8B0060BB1002001
:10DEE00010BDFFF7A3FF002010BD00BF881901205F
:10DEF000704C012038B5D0F8A84201F00F036268D9
:10DF000093422BD80A062BD41C25C1EBC10200205A
:10DF100005FB014104EB820201F5FE7182F8FD016F
:10DF200001220B708A7094F8BC03904216D084F8DA
:10DF3000BC234A782068012A09781DD000F5306298
:10DF400002EB41121568002D00DBF1B9116841F4B4
:10DF5000001111601BB3002384F8BC33002038BDCE
:10DF60001C21C3EBC302012001FB034104EB82022D
:10DF70003C3182F83D00D3E700F5106202EB41121C
:10DF800015680029E2D0002DE0DB116821F0804106
:10DF90001160116841F400111160002BDBD104F510
:10DFA0007172217C05F052FDD5E700BF10B5044623
:10DFB0008021FFF79FFF00212046BDE8104099E730
:10DFC00011F0800F01F00F01F0B4D0F8A8424FF02B
:10DFD0001C0042D1C1EBC10500FB0140002604EB4F
:10DFE000850500F5FE7085F8FD6145780170836058
:10DFF000C27005B1C180022A01D10023037194F8D7
:10E00000BC33012B1AD00122236884F8BC23417849
:10E01000057891422CD003F5006605F00F0103F559
:10E0200030638A40F16903EB451341EA0242F26131
:10E030001A68120405D5002384F8BC330020F0BC14
:10E04000704782681D68C2F30A02C07818492A43E3
:10E0500042EA804211431960EDE7C1EBC105012698
:10E0600000FB014004EB85053C3085F83D60BCE7D2
:10E0700005F00F06D3F81CC803F5106203F500671E
:10E08000B14002EB451241EA0C01F9611368190431
:10E09000D1D483681668C3F30A03C07804493343B4
:10E0A00043EA804343EA855319431160C3E700BF45
:10E0B000008000102DE9F04F854D83B02C6E636910
:10E0C00013F0010B02D003B0BDE8F08F6269A369C1
:10E0D0001A42F8D06369A26913409E0703D56369A9
:10E0E00003F0020363616369A2691340180379D4E2
:10E0F0002046436982691340590300F1D480426984
:10E1000083691A4200F1B9804369826913401A0594
:10E1100008D5D4F80838DB0700F15383436903F4CA
:10E12000006343614369826913401F0110D543694D
:10E1300003F00063436195F85434002B40F04A82A9
:10E14000012385F85434436DC3F38303C5F8583471
:10E15000436982691340DE0400F1D3814369826917
:10E1600013409A0400F17681436982691340DB060B
:10E1700012D5836923F010038361236AC3F34342FA
:10E1800003F00F01022A00F0E582062A00F05E8209
:10E19000836943F0100383614369826913401F0759
:10E1A00000F10D82436982691340DE0200F10282B0
:10E1B0004369826913409C0200F1F78143698269D7
:10E1C0001340590000F1EC814369826913405A07FA
:10E1D0007FF579AF4468630700F1E78243681C4329
:10E1E000446070E7D4F81868D4F81C381E40360C28
:10E1F0003FF47EAF374B20460027CDF800B099465C
:10E2000006E0760807F1010709F11C0900F03282E7
:10E21000F107F6D5F9B200F5306A0AEB41129268BF
:10E22000D0F8143802EA030818F0010F40F02882F1
:10E2300018F0080F40F05C8218F0100F05D004F5BC
:10E240003063102203EB47139A6018F0200F09D0B7
:10E25000296F012900F0568304F53063202203EB77
:10E2600047139A6018F4005FCBD004F530634FF485
:10E27000005203EB47139A60C3E7D4F8043823F045
:10E280000103C4F8043895F85434012B00F0B78129
:10E29000D5F8603493F8752283F87422436903F04B
:10E2A0000043436130E7D0F81838D0F81C2803EA5F
:10E2B00002081FFA88F8B8F1000F3FF420AF054EAE
:10E2C0004FF0000A04F51067CDE9004B0CE000BFE9
:10E2D00088190120E81901205FEA58080AF1010AAB
:10E2E00006F11C0600F0C98118F0010FF4D05FFAA6
:10E2F0008AF9D0F81028D0F8344800F5106309F0F6
:10E300000F0103EB4913CC409B68E401E4B21443D2
:10E310001C40E20732D54FF0010E009B0AF00F0CB3
:10E3200007EB4A12D3F834180EFA0CFC21EA0C0160
:10E33000D5F870C0F445C3F83418C2F808E003D12A
:10E34000D6E911231344B364D5F860B4B9F1000FD2
:10E3500040F0E681DBF86C32022B00F0D88233F01B
:10E36000040300F01A839BF87832012B02D10023BA
:10E370008BF87832BCF1010F00F0F182230703D54E
:10E3800007EB4A1308229A60E10603D507EB4A130C
:10E3900010229A60620603D507EB4A1340229A6066
:10E3A000A30703D507EB4A1302229A60210693D5EF
:10E3B000D6E91441A1428FD8621A736C00EB4A1C53
:10E3C00093420CF5106C28BF1346DCF81820033379
:10E3D00092B2B2EB930F2ED309F10109864600EBFE
:10E3E00009393CB3A14280F0C682621A736C95F879
:10E3F00070009A4228BF1A46B36C02F1030B4FEA31
:10E400009B0B70B990B2033080080AD003EB8001F7
:10E4100053F8040B8B42C9F80000F9D1B36CD6E96C
:10E420001441DCF818001344114480B2B3647165E0
:10E430008345D6D97046A142FFF44EAF0AF00F01D2
:10E440000124D0F8342804FA01F122EA0102C0F8CC
:10E45000342841E7D0F8001900F50063B84A0A40B3
:10E46000C0F800299A6802F00602042A00F0CB8066
:10E470005A6842F480725A609B6813F0060340F0B9
:10E48000AA81C268EB6622F47052C260C36843F48A
:10E490001053C3604FF00009D5F860644FF0400896
:10E4A00000220127434630461146FFF789FD4346C7
:10E4B000002230468021C6F84471C6F85081FFF72B
:10E4C0007FFD0023D6F8A022B761C6F8248086F825
:10E4D0007472C6F86C327360C6F87C32002A00F0A1
:10E4E000EC81D6F88C32304600215B689847D5F82D
:10E4F0006034286E83F81090436903F4005343613D
:10E5000032E6D4F804284FF4846104F500678D4B9B
:10E5100022F001027A60016101E0013B02D0026950
:10E520009106FAD4D5F864C0BCF1000F16D004F5FA
:10E5300010634FF67F3199600BF1010B1A6820339D
:10E54000E34522F4001243F8202CC3F8E811D3F875
:10E55000E02122F40012C3F8E021ECD1FB69D5F8E8
:10E56000902043F00113FB61002A3DD17A6942F209
:10E570002B0313437B613B6943F00B033B61D4F8EE
:10E58000003895F8701023F4FE636F4AC4F8003821
:10E5900005F05CFA286E436903F480534361DDE5BE
:10E5A000436903F0804343610EE6436903F40013BB
:10E5B000436103E6436903F480134361F8E5D5F84A
:10E5C000603493F87422032A37D0436903F00803B8
:10E5D0004361E7E5D5F86034042193F8742283F8A9
:10E5E000741283F87522B3E5D7F8843043F00B0337
:10E5F000C7F884307B6C43F00B037B64BFE70023D8
:10E6000085F854344AE6D0F8002942F00302C0F8F5
:10E6100000295A6842F480725A609B6813F006031E
:10E6200040F0D980C368002223F47053EA66C360C7
:10E63000C36843F41053C3602CE7D3F88C22D2692B
:10E64000002AC2D018469047286EBEE7C1EBC10130
:10E6500004F58054C3F30A1305EB81022668D2F84F
:10E660007412C5F824640B442168C2F87432C5F8EA
:10E6700028148DE5DDF800B03BE5DDE9004B3EE513
:10E6800004F530634FF0010C2A6F0AEB471A03EBD5
:10E69000471B6245CBF808C0D0F840E0DAF80830F4
:10E6A00000F01681294A964540F0FB801A0440F19B
:10E6B000F3804FF4004218F0080FCAF808203FF426
:10E6C000BBAD026CDAF80800204B9A4200F0D08013
:10E6D0001D49D5F86004019206F080FB1C4B019A9D
:10E6E0009A4200F2D0800822286ECBF80820A3E5D9
:10E6F0007B01296F026C03F5306A012904F5306152
:10E70000824401EB030BDAF80800DDD1104B9A428A
:10E7100000F2AE800C49D5F8600406F05FFBE2E73A
:10E72000DBF88C325B69002B3FF428AE9BF8742237
:10E73000032A7FF423AE584649469847286E1DE6C3
:10E7400000F8FFFF400D0300AC1D01200A31544FBB
:10E750000A30544F47F6F07213423FF419ADC3F339
:10E760000A16C1EBC1024FEAC10C3346033605EB72
:10E770008202B608D2F8682208D004F5805402EB71
:10E780008607266842F8046BBA42FAD1ACEB010264
:10E7900005EB8202D2F86842D2F874121C440B4492
:10E7A000C2F86842C2F87432F2E4D5F8600401227B
:10E7B000D0F88C3280F8742201795B689847286E13
:10E7C0000CE5D5F86034042193F8742283F87412B0
:10E7D00083F87522A2E423F00403002B3FF422AF58
:10E7E000A74A0326A74BD2F87421A7491344EE6623
:10E7F0008B4240F2C280A54BA54913448B4240F2A4
:10E80000D480A44BA44913448B4240F2F380A34B21
:10E81000A34913448B42C0F02481A24BA249134464
:10E820008B4240F22181A14BA14913448B42C0F09D
:10E830001E81A04BA04913448B42C0F01E819F4B08
:10E840009F4913448B42C0F015819E4B9E4913444F
:10E850008B4234BF4FF4E0534FF4C053C2684FF0C3
:10E86000010922F47052C260C2681343C36013E608
:10E87000000403D54FF40042CAF808209349D5F8A4
:10E88000600406F0ABFA296F01297FF42CAF8F4AA0
:10E89000286E05F0DBF826E79B0602D52023CAF890
:10E8A0000830C1EBC103D5F8600405EB8303D3F84E
:10E8B000682206F07FF8286EBAE4D6F89032002B72
:10E8C0007FF40FAED6F89832002B7FF40AAE0EE636
:10E8D0001A0755D57E4A964505D9190403D54FF434
:10E8E0000043CAF808307949D5F8600406F076FA92
:10E8F000764A0121286E05F0A9F80823286ECAF887
:10E90000083095E4714A05F0A1F8286EA4E4DBE92B
:10E9100008239A4259D8DBF81C10B1FBF3F203FB31
:10E9200012120AB98B4268D9DBF88C32DB682BB142
:10E930009BF87422032A01D15846984780215846F3
:10E94000FFF7D8FA0023052258461946CBF86C2267
:10E950001A46FFF743FAD5F870C0286E03E5D5F8DC
:10E96000B0305AEA03037FF409AD6146574A05F017
:10E970006DF8286E02E5704660E54FF470536DE760
:10E980009A0615D52022CAF8082018F0080F3FF47F
:10E9900053AC026CDAF80800B8E680215846FFF75D
:10E9A000A9FAD5F870C0286EDDE44FF4605355E73E
:10E9B00013F0280FE9D1464A96452CD91B042AD5D5
:10E9C0004FF40042CAF80820DFE7D31A4946D5F8C9
:10E9D000A820DBF8A802CBF820309BB205F008FB9A
:10E9E0004B464A4649465846FFF7F8F9D5F870C0F5
:10E9F000286EB8E44FF4505330E7DBF87032994298
:10EA000092D24B464A464946DBF8A80205F0F0FA96
:10EA1000CBF87092E4E7DAF81020C1EBC100D9F826
:10EA20000432C2F3120CD9F8082205EB80001A4414
:10EA3000A3EB0C03C9F80822D0F86822D5F86004CB
:10EA4000C9F8143205F0B6FFD5F870323B437FF4B5
:10EA500032AF1E4A0121286E04F0F8FF286EFFF73E
:10EA6000E7BB4FF44053F9E64FF43053F6E64FF46A
:10EA70002053F3E64FF40053F0E64FF41053EDE665
:10EA8000802A0120405327FFFF340C00401E1BFF4B
:10EA90003F420F0000DC0BFF7F4F1200808CF9FE1D
:10EAA00020D6130060B6E5FE5FE3160000D3CEFE6D
:10EAB00040771B00C05BB3FEC091210000CA91FEED
:10EAC00020753800E05459FEE09C4100AC1D012047
:10EAD0000A30544F2DE9F0414FF0FF35324A002300
:10EAE00032482C4603E0013310320B2B14D0917ABC
:10EAF0000429F8D103F5B17100EB0111C979CF07F1
:10EB0000F1D4661C116801D0A942ECD21C46013335
:10EB10000D4610320B2BEAD1631C02D10120BDE857
:10EB2000F081224D04F5B17705EB07139988E9B917
:10EB30002601DFF88480AA19D8F87C3F41F21860DA
:10EB40001B491E690023105801EB4421194AB047A4
:10EB5000E0B1022817D141F2CC6205EB0717012181
:10EB60000020AB58B971013BAB50D8E7DFF84880C3
:10EB700005EB041241F218602601D8F87C3F1058CA
:10EB8000DB689847D7E70020BDE8F08141F2CC620E
:10EB9000032405EB071741F2D061AB58BC71012487
:10EBA000013B6C54AB50BAE7A88B01208C75012057
:10EBB000A4750120D5EB0008783B0120044B41F2FD
:10EBC000E472995C09B90121995401225A70704785
:10EBD0008C75012070B50024164D41F2D066164B9D
:10EBE0002046AC5503E0013010330B2814D053F805
:10EBF0000E4C8C42F7D11C78032CF4D16AB10F4B28
:10EC000003EB40239A4201D0FFF7D8FF00F5B17023
:10EC1000012305EB0010837170BD41F2CC6100F55A
:10EC2000B17304206A5805EB0313013298716A50DE
:10EC300070BD00BF8C750120B28B0120A47501202E
:10EC400038B50020114B9C7B14B11D688D4204D057
:10EC5000013010330B28F6D138BD82B10C4B03EBD9
:10EC600040239A4201D1022C01D0FFF7A7FF00F503
:10EC7000B170084B012203EB0010827138BD00F522
:10EC8000B170044B03EB0010827138BDA48B0120DE
:10EC9000A47501208C7501202DE9F04F83B002F09E
:10ECA000020C019310B9BCF1000F60D1844C41F605
:10ECB00038056559002D61D14FF0FF36814F002591
:10ECC000B146B046B2463B68984200F0BE8097F825
:10ECD0000EE0BEF1000F62D0BEF1010F15D105F5B7
:10ECE000B17E04EB0E1E9EF807E01EF0010F0CD162
:10ECF0001EF07E0F09D15FEADE1340F0B080D7F836
:10ED000008E0F24501D9F246A946013510370B2D2E
:10ED1000D9D1751C04D1B8F1FF3F00F0A780464659
:10ED200041F2C86806F5B17704EB061E41F21C6A91
:10ED300054F808504FEA071941F2186B01354EF8A4
:10ED40000B0044F8085004EB07184EF80A5044F83A
:10ED500009500025C8F8045004EB0715AD79042DBF
:10ED600000F2A980DFE805F02139163955000225A7
:10ED7000FFF724FF284603B0BDE8F08F04F5C25723
:10ED800041F63C063F68A65907FB0565A84293D3A8
:10ED9000FFF714FF0025284603B0BDE8F08F2E468C
:10EDA000013510370B2D8ED1B3E712F0010E6FD164
:10EDB00004EB0710019BD51090F80780032B65F337
:10EDC000C71880F8078061D94FF6FF70834228BFCB
:10EDD00003469BB204EB07108380BCF1000F18D0F0
:10EDE00004EB061041F218630344987B042810D00A
:10EDF00041F2C86C41F2CC654FF0040E54F80C009F
:10EE0000013044F80C00586083F80EE06359013378
:10EE10006351500705D504EB0710C37943F0010394
:10EE2000C371D30608D504EB0714E379C3F3450295
:10EE3000013262F34603E371234B012503EB4626BF
:10EE400028460E6003B0BDE8F08F05F5B17704EBFE
:10EE500007164FEA071EB6796EB92E4660E7A84638
:10EE6000013510370B2D7FF42EAF52E7B9F1FF3F7C
:10EE700090D04E4654E741F2C8682E4654F80850E8
:10EE8000013544F8085044F80E5065E77346A1E791
:10EE90000E4A00230C49D2F87CCF01EB46210C4AE4
:10EEA000DCF80860B04700283FF474AF04EB0714A7
:10EEB0000223A3715EE70225FFF780FE5AE700BF39
:10EEC0008C750120A48B0120A4750120783B0120C2
:10EED00041EC0008F0B5154D83B00E462B78022B9F
:10EEE0000FD14FEA102CC4B241F6300700230122A3
:10EEF00001A9E8596044FFF7CFFE012806D003B00E
:10EF0000F0BDC0F3D41C00F07F04EDE72B78022B9A
:10EF1000019B04D133F81430336003B0F0BD53F8D3
:10EF2000243023F07043336003B0F0BD8C750120B2
:10EF300010B5144602070B4610D50B4941F2C472B6
:10EF4000581C8B58834204D305D100230120236031
:10EF500010BDFFF733FE2060012010BD214618468A
:10EF6000BDE81040B6E700BF8C7501202DE9F041E7
:10EF70000D46416882B00446C1F308032B44B3F543
:10EF8000007F58D390F91A30591C0AD0304A03F543
:10EF9000B173FF2102EB0313DA796FF30002DA7128
:10EFA000817694F91B305A1C0FD0294A03F5B173AE
:10EFB000FF2002EB0313DA79C2F34501013921EA9C
:10EFC000E17161F34602DA71E0762378022B38D0E2
:10EFD0001F4A02F5C2531B68B5EB432F4FEA432883
:10EFE00025DC41F648036768D6583E407242AA4283
:10EFF0001DDCAB19434512D301AA2169207EFFF71E
:10F0000097FF012813D16768A5EB0805206908EB75
:10F010000703019A354460619F1B226167602046A7
:10F02000F9F74EFB20B93D440120656000E0002067
:10F0300002B0BDE8F08129440120616002B0BDE862
:10F04000F081616801202944616002B0BDE8F0816F
:10F050008C75012070B5154604460E46FFF786FFF5
:10F0600050B994F8280028B90223C4E90B5684F853
:10F07000283070BD022070BD1DB12046A847012078
:10F0800070BD012070BD00BFD0E9011310B48B42E8
:10F0900090F91A2038BF0B46511C83600AD0144BDC
:10F0A00002F5B172FF2103EB0212D3796FF3000373
:10F0B000D371817690F91B305A1C0FD00C4A03F59E
:10F0C000B173FF2402EB0313DA79C2F3450101396E
:10F0D00021EAE17161F34602DA71C4760022436AE3
:10F0E0005DF8044B1146426142600361B2E700BF24
:10F0F0008C75012070B544220021114841F60204AC
:10F100004DF0BCFF0F4B032141F64C001A784FF62F
:10F11000FF761D5803F5C050022A1E5341F2E876CF
:10F1200041F60C0418BF0A4600F8181941F601010F
:10F130001D519A5510225A54FFF7A6FF012070BDA9
:10F14000748D01208C750120B1F904300F2B2DE94D
:10F15000F0410C4682B01646054633D02846F9F7F2
:10F16000D7FA95F91B800746B8F1FF3F34D02D4BF5
:10F1700041F2186203EB08118A58904212D11833F9
:10F1800003EB4823A1882846013109B203EB411360
:10F19000A1803360F9F7BCFA03460120236002B076
:10F1A000BDE8F081FFF70AFD2846F9F789FA28B192
:10F1B00000230120336002B0BDE8F081002002B0DE
:10F1C000BDE8F0814FF40071FFF7D0FE0028F5D0C4
:10F1D0004FF6FF73A380C1E72846F9F771FA0028BC
:10F1E000E2D10FB9FFF7EAFC38460023112201A94A
:10F1F000FFF752FD0128D7D1019B0B4A9A1A48BF4D
:10F2000002F2FF12B2F5B05F4FEA622106D24FFA66
:10F2100081F885F81B80002BB4D1C5E7FFF7CEFC41
:10F22000019BF6E78C750120A475012030B50446DA
:10F23000C06983B010B9012003B030BD0D46002372
:10F24000032201A9FFF728FD0128F5D1B4F92030E8
:10F25000002B03DAFFF7B2FC0220EDE7019A012D43
:10F260004FEA431102EB431303D0022D12D1E525DF
:10F270005554A268DA612278032A04D100221A7751
:10F280005A779A77DA77626AC2F30F415A83998282
:10F2900003B030BDE268DA61EDE700BF10B5037876
:10F2A0000446023B012B037E02D913F0060F5AD10C
:10F2B00098063AD494F91A30591C0AD02D4A03F50D
:10F2C000B173FF2102EB0313DA796FF30002DA71F5
:10F2D000A17694F91B305A1C0FD0264A03F5B1735E
:10F2E000FF2002EB0313DA79C2F34501013921EA69
:10F2F000E17161F34602DA71E076237E1B070BD5DC
:10F300001C4841F2C873C35C072B01D0FFF756FCC1
:10F3100041F2C8730022C2540023E26A237084F8C9
:10F320002830FAB1BDE81040104700231249E069C7
:10F330001A018A58904206D001330B2BBAD01A0119
:10F340008A589042F8D10B4A03F5B17302EB0313CC
:10F35000DA79C2F34501013921EAE17161F346022C
:10F36000DA71A7E710BD0121FFF760FF0128F9D18D
:10F37000237E9DE78C750120A48B0120B8B138B5A0
:10F38000027822B190F828201AB1002038BD01205F
:10F3900038BD826803244568C162AA4280F82840CB
:10F3A00038BF2A468260FFF779FF012038BD01206F
:10F3B000704700BF2DE9F04FDFF84C91174683B03E
:10F3C0008A4699F800300A68022B7BD1D6B241F602
:10F3D00030044FF48071A6EB020859F80450B84489
:10F3E00005EB12258844BA4208F1FF38B8FBF1F862
:10F3F00064D200F0010BA844032B06EB0704A8EB32
:10F4000005030CBF80214FF48071A41A8C4228BFE1
:10F410000C460EB98C4235D20B2201A92846FFF7C3
:10F420003BFC012802D003B0BDE8F08F99F8001032
:10F43000DAF80020022902F1010325D0A64210D2F9
:10F44000019A6FF04040111F304401EB840102EB40
:10F45000800242F8043F914203F10103F9D1DAF846
:10F460000020A61B3244BA42CAF8002002D1BBF1E8
:10F47000000F39D1BA4205F101051FD299F80030C9
:10F480000026B9E70A22C8E7A642EAD201996FF03E
:10F49000004C881EB44400EB440001EB4C0121F801
:10F4A000023F884203F10103F9D1DAE76FF000432C
:10F4B000019A4FF6FF71234422F81310012003B084
:10F4C000BDE8F08F41F6300102F07F06032BC2F356
:10F4D000D41559F80140A6EB020814BF4FF480710F
:10F4E0008021B84425447DE799F80030022BDDD017
:10F4F0006FF04043019A4FF0FF31234442F823104C
:10F50000DAF80020B6E700BF8C750120F8B590F856
:10F5100038300446032B4ED8DFE803F0023039447C
:10F520002B4B41F2A87EC56841F2C47C187803F5E4
:10F53000C25153F80C2041F2AC770328096853F804
:10F540000E000CBF80264FF48076226101FB06F18D
:10F5500005EB4125A0EB4120E560951943F80E002D
:10F56000D85943F80C50A0EB4121E06AD951C4E9C5
:10F570000C2548BB6262012384F83830002115480D
:10F58000FFF754FE012811D1022384F83830626B52
:10F5900004F130010120FFF70DFF012806D10323FC
:10F5A00084F8383000212046FFF740FE431EDBB2CE
:10F5B000012B01D9F8BD022094F82830062BF9D18F
:10F5C000002384F82830F8BD921B2263D3E700BFE4
:10F5D0008C7501202C8D01202DE9F04FDFF824815E
:10F5E000012887B00C4698F800608CBF00230123E7
:10F5F0001546032E02930B6839D0022E62D14FF4C8
:10F6000080724FEA1329DFB201920138012823D812
:10F61000012203929D421AD9384E06F1880A06F15A
:10F620001C0B32681AB1DBF8001099424ED0DAF8A0
:10F6300000000023092205A94844FFF72DFB0128FB
:10F640001FD002280FD020B123689D42E9D80320A3
:10F65000256007B0BDE8F08F87B1FFF7AFFA022051
:10F6600007B0BDE8F08F022007B0BDE8F08F802220
:10F670000192C3F3D41903F07F07C6E7019A0392FE
:10F68000C8E7059ADDF804E0DDE902C198F800302A
:10F69000022B14D0032BE6D152F8273023F070430D
:10F6A000B3FA83F30F445B096345236823D00B440B
:10F6B00077452360EAD309F101090027C5E732F84D
:10F6C0001730EDE74FF480720192D2E70C49013A0E
:10F6D000096802EB41224902B2FBF1F2039913449B
:10F6E000B3FBF1F201FB12320AB10B449B1A9D42AB
:10F6F000236096D8ABE7AB42ABD3A8E7348D0120AB
:10F70000CC8D01208C750120F0B5114D83B00E46D3
:10F710002B78022B17D14FEA102CC4B241F63007D8
:10F720000023032201A9E8596044FFF7B5FA012834
:10F7300007D12B78022B019B0CBF23F8146043F8F0
:10F74000246003B0F0BDC0F3D41C00F07F04E5E7F3
:10F750008C7501202DE9F043002990F83C3083B0EE
:10F76000044614BF02210021042B7BD8DFE803F0FC
:10F77000030C3C476900FFF759FD012870D1626B0B
:10F78000002A75D184F83C00404E4FF6F777DFF839
:10F7900004813F4D1BE0B94594BF4FF000094FF085
:10F7A000010901A9B9F1000F48D1FFF793FB012826
:10F7B000494652D1206BFFF7A7FF01284DD1019A8E
:10F7C0002B68511E22638B4228BF0B462B60337877
:10F7D000206B032B1FFA80F9DDD1404594BF4FF019
:10F7E00000094FF00109DCE7426B04F13001002011
:10F7F000FFF7E0FD012833D1032384F83C30234B8D
:10F8000041F2C470E16A41F2A8771A5803F5C25573
:10F81000195041F2AC76511A2A68D85902FB01F20C
:10F82000995900EB422503F5BD5001EB422200211E
:10F83000DD519A51FFF7FAFC012811D1042384F815
:10F840003C3094F82830042B02D1002384F828306F
:10F85000A36B8BB120469847012003B0BDE8F0832D
:10F860000228FAD194F82830042B09D00220F4E7BA
:10F87000022384F83C30B8E7012003B0BDE8F083F0
:10F880000023022084F82830E7E700BF8C750120B0
:10F89000D08D0120F7FFFF0F38B590F834300446C3
:10F8A000052B42D8DFE803F01E033B0F1868006BFE
:10F8B0004FF0FF31FFF728FF012836D1E06AB0BBD7
:10F8C000032384F8343000212046FFF7AFFC0128E1
:10F8D0002BD1042384F8343094F82830082B2AD014
:10F8E000012038BD41F63803244D00F130010120DC
:10F8F000EA580232FFF770FE01282AD00238C0B25F
:10F90000012812D8052384F8343094F82830082BC5
:10F9100016D041F2E57301220220EA5438BDC06AD4
:10F92000216BFFF7F1FE0128CAD0002038BD022369
:10F9300084F83430F4E70023012084F8283038BDFF
:10F9400000230122022084F8283041F2E573EA54B2
:10F95000E4E705F5C252E368206B41F64401126802
:10F96000685003EB4223E26AC4E9033002B96062E3
:10F97000012384F834309BE7004DC6E78C750120E5
:10F9800043682DE9F04F164683B0C3F30808002AF8
:10F9900000F0DF80704B054689464FF0000AA3F166
:10F9A000180BC8F5007495F91A702846B44228BFA0
:10F9B0003446791C2ED0F8F7ABFE41F218620BEBFF
:10F9C00007139B58984205D0FFF7F8F8504603B04C
:10F9D000BDE8F08F604B03EB472022464946404488
:10F9E000A2444DF0D9FA002221462846FFF732FB07
:10F9F0000028EBD02B7E1B0706D5584B2A691B68C5
:10FA00009A4201D3FFF7DAF8361BA1444FF0000801
:10FA1000C7D1DBE7F8F754FE002846D12846F8F7AF
:10FA200077FE6968C1F308031BBB4D4AAB680A4007
:10FA300002F500729A422CBF062207222B7E03F0A9
:10FA40000C030C2B1BD0002301A9FFF725F901287B
:10FA5000BCD10198404BC31A48BF03F2FF13B3F562
:10FA6000B05F4FEA63224CD257B2AF760028B4D1D0
:10FA7000ACE72B7E072203F00C030C2BE3D19BF8A1
:10FA800000C0384BBCF1030F1B680CBF4FF0800C5B
:10FA90004FF4807C03FB0CF34FEA432C0CF1FF3C4A
:10FAA0000CEA0101A3EB5123CEE72B7E1A072CD5DC
:10FAB0009BF800202B4B032A95F828201B680CBFCD
:10FAC00080214FF48071062A03FB01F34FEA4323A0
:10FAD0003FF47CAF24490868834231D891F83D3027
:10FAE000002B7FF473AF002A7FF470AF06216B699F
:10FAF000284685F8382085F82810EB62FFF706FDC8
:10FB00001AE0FFF75BF80198AFE795F82830002B73
:10FB10007FF45CAF154B1A78002A7FF457AF0821A9
:10FB200085F834206A69284685F82810D3F85F30B4
:10FB3000C5E90B23FFF7B0FE01283FF46FAF45E79F
:10FB400041F2E573012250460BF8032003B0BDE8F3
:10FB5000F08F92463AE700BFA4750120508D012036
:10FB600000FEFFFFCC8D0120348D0120718D01201E
:10FB70002DE9F04790F8384082B00546032C00F29A
:10FB80009980DFE804F00218600BFFF785FE01287A
:10FB90000FD0022809D1032385F8383000202B6CC0
:10FBA000022485F8280003B19847204602B0BDE83A
:10FBB000F08785F838002B78022B50D03E4941F66B
:10FBC00048026B688A5803EA0208C8F34F2828469F
:10FBD000DFF8E890F8F79CFD0646A8EB0008022243
:10FBE00001A930460023FFF757F808EB0607012864
:10FBF0004FF40072BFB24FF00001044606F1010657
:10FC0000D3D101984DF03AFAEB694FF400712846D0
:10FC10000BB16B684BB3D9F80030013B9F4206D261
:10FC2000FFF7A4F90028DAD1FEF7C8FFD7E7C3EB46
:10FC3000C35328465902FFF799F908B9FEF7BEFFEA
:10FC4000022385F8383000222B6C85F8282053B128
:10FC5000012428469847204602B0BDE8F0876B682B
:10FC6000C3F34F28B3E701249FE7019B4FF02032F5
:10FC70002E244FF0100C1A605A601C70C3F8072035
:10FC8000D5F824E01A625A62CEF30F4A83F8204076
:10FC900083F82140C3F8272083F80BC0EA6BA3F850
:10FCA0001AE0C2F30F44A3F814A05A879C8683F885
:10FCB0002BC0B0E7002478E78C750120CC8D0120A3
:10FCC0002DE9F04F90F8303089B00446042B00F253
:10FCD000A780DFE813F0A800B10005008900E70065
:10FCE000B54D41F61003EB5C002B40F09980B34F0B
:10FCF00004F11C0901AEB84607F1380BBA4632468A
:10FD000049464046FFF720FA012840F01681019845
:10FD1000002800F0F98003780BB1E52BEFD1A84A59
:10FD2000821A48BF02F2FF12B2F5B05F4FEA6223B7
:10FD300080F03B811B01A34A13449A7B042A0CD018
:10FD400041F2C86641F2CC610427AA590132AA5196
:10FD50005A609F736B5801336B5041F60202AB56E9
:10FD60005E1C09D003F5B173FF2105EB0313A95401
:10FD7000DA796FF30002DA7141F603016B565A1C0F
:10FD80000ED003F5B173FF2605EB0313DA796E5439
:10FD9000C2F34501013921EAE17161F34602DA71EA
:10FDA000202200214DF06AF92346019A05A853F854
:10FDB000315F59681560516019899B7A118193727E
:10FDC000019B627EDA723FF013FABDF81430002B0B
:10FDD00040F02E8144F28172019903200A82CB8186
:10FDE0000A83CB8284F83000237E980600F1A88035
:10FDF0002046FFF749F92369002B00F0AD80237EF0
:10FE000003F0F70213F00403227640F0B380122AC5
:10FE100000F0B9800022E36A204684F82820984741
:10FE200009B0BDE8F08F6548FFF72EF94FF6FF7275
:10FE30000123228484F8303004F11C0801AE5F4FA6
:10FE400004F13109324641463846FFF77DF9012871
:10FE50002FD00228E4D1584D41F60202AB56591C6E
:10FE600009D003F5B173FF2105EB0313A954DA7927
:10FE70006FF30002DA7141F603016B565F1C0ED07E
:10FE800003F5B173FF2005EB0313DA796854C2F36D
:10FE90004501013921EAE17161F34602DA71042377
:10FEA00084F830300020E36A2070984709B0BDE83C
:10FEB000F08F019D0B2249462846002D00F08680D8
:10FEC0002B78002B00F0828095F80BA01AF0080F19
:10FED000B8D14DF0B9F90028B4D1637E8AEA0303A2
:10FEE000DB0640F1C680344D41F60202AB565F1C82
:10FEF000C1D003F5B173FF2105EB0313A954DA79DF
:10FF000060F30002DA71B6E73B78092250462E49C9
:10FF1000022BC4D00B78002BC1D10A708BF80030B3
:10FF20004A6B0B73C1E9053351F8143CC1E9013246
:10FF3000FFF71EFE01283FF4E2AE0228AFD06FE7C4
:10FF40000023112205A9E069FEF7A6FE01283FF46F
:10FF50004FAF09B0BDE8F08F237E19077FF55AAF88
:10FF6000154A41F2C873D15C00297FF459AF0721CB
:10FF7000D1544FE70023E26AA168204684F8283074
:10FF8000FFF768F84CE7E56A0421626A204684F8C6
:10FF90003C306363A56384F828106362C4E90233CC
:10FFA000C4E90B22FFF770F83AE7FEF707FE019865
:10FFB0006FF00F03BFE600BF8C750120748D012028
:10FFC000A4750120A48B01209C8D0120474D41F692
:10FFD0000202AB565E1C09D003F5B173FF2105EB9D
:10FFE0000313A954DA796FF30002DA7141F60301C1
:10FFF0006B56581C0ED003F5B173FF2005EB0313AD
:020000040801F1
:10000000DA796854C2F34501013921EAE17161F3FB
:100010004602DA71237EDA067FF541AF3448FFF7F6
:1000200033F84FF6FF720223228484F8303058E60A
:10003000304B05A902A8B3F9B4263FF0F9F89DF8B2
:100040000C309DF80D00DB029DF80A509DF80B2046
:10005000BDF8081043EA401342EA45129DF80E002D
:10006000A1F2BC7143EA500342EA41229BB292B230
:10007000B2E6A98A6A8B204B42EA01421B6862629F
:100080005A02EB69B3FBF2F102FB1131A36009B133
:1000900013445B1A154D41F60202E36084F819A07F
:1000A000AB565E1C09D003F5B173FF2105EB0313BA
:1000B000A954DA796FF30002DA7141F603016B5645
:1000C000581C0ED003F5B173FF2005EB0313DA794A
:1000D0006854C2F34501013921EAE17161F3460236
:1000E000DA71032384F830307EE600BF8C7501207E
:1000F000748D0120704C0120CC8D01202DE9F04140
:1001000090F8283084B00446013B082B41D8DFE842
:1001100003F048054D525865406A4300394B41F69B
:10012000480241689F5803F5C253056B0F401B6896
:10013000EA194FEA4328B2EB432F16D258E021695F
:10014000207EFEF7F5FE012823D1256B6168A5EB23
:10015000080522694144039B3D446261C91B236138
:10016000A84537466160256342D82046F8F7A8FACB
:1001700003AA06460028E2D06168A3680020E26A6C
:10018000994284F8280038BF1946A1600AB1204678
:10019000904704B0BDE8F081FFF7EAFC04B0BDE889
:1001A000F081FFF78DFD04B0BDE8F081FFF776F830
:1001B00004B0BDE8F0810021FFF7CCFA04B0BDE83F
:1001C000F0810121FFF7C6FA0128E2D10023216C5A
:1001D000204684F82830FFF7D1F8DAE7FFF796F9E0
:1001E00004B0BDE8F081FFF757FB04B0BDE8F08133
:1001F00020460191F8F764FA01990028BDD12944FD
:100200006160BAE78C7501202DE9F04782B00546A0
:1002100018461C4602AF0E4690464AF03DFC083098
:10022000013C20F00700ADEB000D0DF1080AD146AE
:1002300014F8013F5BB94246314689F80030284640
:10024000CDF800A033F0E2FABD46BDE8F0871846CD
:100250003EF07AFDC3B2A3F120023F2A88BF2023DB
:1002600009F8013BE4E700BF2DE9F0470D46904651
:100270000021442204461E46089F4CF0FFFE012345
:100280004FF6FF722676628384F828302B782E2B67
:1002900042D004F1310A04F139092E463278202384
:1002A00010462AB12E2A03D03EF04EFD0136C3B2CD
:1002B0000AF8013BCA45F1D130782E2801D1707877
:1002C000013604F1380904F13B0A202318B13EF04D
:1002D0003BFD0136C3B209F8013FD14507D0307864
:1002E00020230028F3D109F8013FD145F7D118F0B8
:1002F000100F84F81980E76214BF032301232370D1
:100300002B782E2B24D00023204684F83030FFF7A2
:10031000D7FC2046BDE8F0876B78002BB9D1124B93
:1003200041F60C0041F2F47141F2F0721E589A58F5
:10033000585841F601016662C4E9022041F2E872B0
:10034000595C61769B5CE76223702B782E2BDAD1A7
:100350006B78002BD7D10323204684F83030FFF789
:10036000AFFC2046BDE8F0878C75012001210320F9
:1003700008B549F07BF872B640F0FEF82DE9F04F71
:10038000CF4C8DB04FF00008DFF84893CD4D009072
:1003900054F80B0C002800F0FE802DF093FC06466C
:1003A000002800F0DC81D9F82830E026A4F10B0BFE
:1003B000C54F44F8073C002306FB08F604F8033C4D
:1003C00054F80B0C2DF07EFC002800F0E48054F86B
:1003D0000B0C2DF06FFC14F8023C82465A1E0B2ABF
:1003E0000DD8DFE812F01F003A00460053008300EA
:1003F0009B00E20016013601410179019101242898
:100400000CD0009A3AB995F82E26824240F08281AB
:10041000012204F8032C0D2BD2D186E0012304F82D
:10042000023CCDE700234D28C4F8C53084F8CD3018
:1004300084F8CE3004D0582808D004F8023CBFE736
:10044000022284F8C43004F8022CB9E7032304F82C
:10045000023C022384F8C430B2E704233C2804F8A9
:10046000023C0BD0BAF13E0F0CD0002304F8023C42
:10047000A6E70A233C2804F8023CF3D1002304F841
:10048000013C9DE7012304F8013C99E7D4F8C5003D
:10049000BB19421C0344C4F8C520022A83F8E7AF05
:1004A00094F8CD008AEA000184F8CD1088D1237831
:1004B000C02BDAD86278FF2A08D1052BD5D90123C1
:1004C00084F8C430072304F8023C79E7A4F8C1207B
:1004D0000022C4F8C930934284F8C320C4F8C52070
:1004E00014BF0523062304F8023C69E7D4F8C500CD
:1004F000BB19421C0344C4F8C52083F8E7AF94F845
:10050000CD00D4F8C9308AEA00019A4284F8CD10AF
:100510007FF456AF062304F8023C51E794F8CD303F
:100520008342A2D10D2304F8023C14F8017C002F71
:1005300040F0F780654B04AE0894ADF82A7003973D
:100540000FCB86E80F00D4F8C930324608A9D4F89A
:10055000D10023440993B4F8C130ADF8283094F8A1
:10056000C3308DF82C3001238DF82D3003AB28F0EB
:10057000B7FB48B1049B314694F8C4205846059314
:10058000534B049325F08EFE0023039E04F8023C97
:10059000002E40F0DC8008F10108E034B8F1030FD0
:1005A0007FF4F6AE0DB0BDE8F08FD4F8C500BA19EF
:1005B0005146431C0244C4F8C53082F8E7AF94F8B2
:1005C000CD2094F8CE008AEA0202019384F8CD206F
:1005D000D5223EF077FE019B84F8CE00072B7FF4F6
:1005E000EFAEB4F80530C02B3FF63FAFB4F80320B0
:1005F000C4F8C930A4F8C120A27884F8C32000222E
:100600009342C4F8C52014BF0823092304F8023C10
:10061000D6E6D522014694F8CE003EF053FE94F87B
:10062000CD3084F8CE008AEA0303D4F8C50084F8FC
:10063000CD30BB19421C0344C4F8C52083F8E7AF92
:10064000D4F8C9309A427FF4BBAE092304F8023CC7
:10065000B6E694F8CD30434084F8CD3094F8CE30EF
:1006600083427FF402AF55E7D4F8C500BA1951466A
:10067000431C0244C4F8C53082F8E7AFD52294F891
:10068000CE0001933EF01EFE019B84F8CE00052BA8
:100690007FF496AEB4F80120B4F80330A4F8C1207A
:1006A0002278C4F8C93084F8C32000229342C4F8E9
:1006B000C52014BF0B230C2304F8023C80E600BFC6
:1006C0005F4B0120704C0120783B01204CD805087D
:1006D00050190220802A0120D522014694F8CE002C
:1006E0003EF0F0FDBB1984F8CE00D4F8C500421CE2
:1006F0000344C4F8C52083F8E7AFD4F8C9309A4260
:100700007FF45EAE0C2398E694F8CE3083427FF4FB
:10071000ACAE07E723287FF47EAE022204F8032C58
:1007200079E6012F4FF0000602D004F8026C32E7A0
:10073000D4F8C93008A8089423440993B4F8C13008
:10074000CDE90A66ADF8283025F074FAEDE754F8E3
:100750000B0C26F007F854F80B0CB0471BE714F805
:10076000033C002B3FF417AFD9F8282054F8071C9E
:10077000521A632A7FF60FAF012B29D0022B7FF488
:100780000AAF54F80B3C012285F8C906C5F8B83603
:10079000C5F8BC36C5F8C436402385F8B62685F8BA
:1007A000C8360C4A0C4B0D48C5F8C026C5F87C3538
:1007B000C5F80C3734F0DEFF4FF4005028F0EEF8A7
:1007C000074834F0CDFF85F8106785F81167E2E639
:1007D000FFF7CCFD0DDD0308305301207E5D0608D8
:1007E000B45D060803460A2201481A80704700BF1C
:1007F000F00301200346202201481A80704700BF01
:10080000FC0301200346202201481A80704700BFE4
:100810001C0401200346202201481A80704700BFB3
:100820003C04012003460A2201481A80704700BF99
:100830005C0401200023D0F89822184613737047F7
:100840000346222201481A80704700BF6804012035
:100850000346222201481A80704700BF8C04012001
:100860000346222201481A80704700BFB0040120CD
:1008700003460A2201481A80704700BFD4040120B1
:100880000346432201481A80704700BFE00401205C
:100890000346432201481A80704700BF2405012007
:1008A0000346432201481A80704700BF68050120B3
:1008B000D0F8943283B110B5D0F8904294F8000289
:1008C000FF2807D09B68214694F801229847FF2310
:1008D00084F80032002010BD0020704701F00F01A5
:1008E000D0F8A822C1EBC10102EB810238B5D0F8E3
:1008F0009032D0F89452D2F8144203F50371EA68AA
:10090000D3F80402C3F80C429047002038BD00BF62
:1009100008B5D0F88C325B689847002008BD00BF4E
:1009200008B5D0F88C321BB11B68984700B908BDD8
:10093000022008BD0022836BA3F85A20A3F852209E
:10094000704700BF836B1A6810B45C6F986F916832
:10095000090601D5212C1AD09168490601D5222813
:1009600006D0DA6F5DF8044B42F01002DA67704788
:1009700000202024A3F85A00116821F4907111601E
:10098000916821F00101916018669C67E9E70021F8
:100990002024A3F85210116821F0C00111605C6797
:1009A000DAE700BF704700BF704700BFC369B3F507
:1009B000807F12D0826B002120201368A2F85A1089
:1009C000196821F480711960996821F0010199601A
:1009D000996821F04001996090677047C369B3F549
:1009E000807F0CD0826B00211368A2F852109A68A5
:1009F00022F080029A601A6842F040021A60704742
:100A000011F0010307D090F8413003F02803282BA0
:100A10000CBF4223F2238A0709D590F8412002F047
:100A20002802282A0CBF43F0440343F0F4034A078A
:100A3000016848BF43F0B8030A6822EA03030B6069
:100A4000704700BFC16838B5022903689A699C697C
:100A50009A68DD680DD1C2F3C21282EA144212F024
:100A6000060206D1816C01318164816C022907D0B4
:100A700038BD0421FFF7C4FF002380F8403038BDA3
:100A800008218264D96180F8402038BD836B002240
:100A9000D3E90E0102650A6593F84120602A02D16C
:100AA000202283F8412070470023202210B5134CE8
:100AB0004363C462036380F8412080F842304B07EF
:100AC00012D50268436A526A1A70436A028D013372
:100AD00043624AB1438D013A013B02859BB2438593
:100AE000436C43F0040343640721FFF789FF10219F
:100AF00002680023D16180F8403010BD0000FFFF84
:100B000038B5002580F8425090F84130292B04D0A8
:100B100090F841302A2B0BD038BD28222123012107
:100B200080F841200363FFF76BFF80F8405038BD29
:100B300028222223022180F841200363FFF760FF6F
:100B400080F8405038BD00BF38B50025202280F81D
:100B5000425090F8413080F84120212B0BBF1123E7
:100B60001223012102210CBF456345630363FFF794
:100B700047FF80F8405038BD90F8BC33012B29D096
:100B8000012380F8BC330B060ED402681021124BEF
:100B9000116101E0013B02D01169C906FAD40023BA
:100BA00080F8BC331846704701F00F010A4B8901E9
:100BB00010B441F020010468216101E0013B02D042
:100BC00022699206FAD4002380F8BC3318465DF8F7
:100BD000044B704702207047400D030011F0800F56
:100BE0004FF01C0301F00F0170B432D103FB01037D
:100BF000C1EBC102002400EB820203F5FE7382F810
:100C0000FD41197090F8BC23012A31D001210268FE
:100C100080F8BC135C781D7802F500638C422AD002
:100C200005F00F04DE6B02F53062A1401C4C02EBB4
:100C3000451226EA0146DE63DD6925EA0141D961F4
:100C400013681C401460002380F8BC33184670BC45
:100C5000704703FB0103C1EBC102012400EB8202D8
:100C60003C3382F83D40197090F8BC23012ACDD165
:100C7000022070BC704705F00F01DE6B02F51062B8
:100C80008C40084902EB451226EA0406DE63DD6962
:100C900025EA0404DC61136819401160D3E700BF42
:100CA0000078F3EF007833EC836B40221A645A6CBF
:100CB00042F004025A647047704700BF836B1A6C9D
:100CC00012F0500F1A6C20D142F4007219681A64A5
:100CD0008A6812F0405F1AD19A69C2B9CA6A12F4DE
:100CE000700F02D08A68500511D44A6822F02002A1
:100CF0004A601A6C22F480721A641A6CD10406D409
:100D00001A6C42F001021A647047D20600D570478F
:100D10009B6BDB6C184700BF836B0121002283F8BB
:100D20003D101A77704700BF0122836B83F83D2086
:100D3000704700207047114A1068A8B153689BB1F2
:100D400088420FD88B4234BF00230123DBB243B16A
:100D5000D368916099421FBF094B1420D16083F87A
:100D6000BB0170470023F1E7A1F59C53083BB3F5A5
:100D70007A7F2CBF00230123E9E700BFE08D01202B
:100D8000F0030120054B5A7C19748A421FBF044AA4
:100D90001420597482F8BB01704700BFE08D012018
:100DA000F0030120704728B1034B987C012894BFC1
:100DB00000200120704700BFE08D012008B5FFF73B
:100DC000F2FF50B1054AD37C127C5B0003F00203B2
:100DD000002A18BF43F001030B6008BDE08D01201D
:100DE00008B5FFF7E0FF10B1014B5B690B8008BD50
:100DF000E08D012070B5FFF7D6FF50B10A4A158B80
:100E000035B1D6690023B3421C4603DB002000E065
:100E10000D7070BD02EB44040133248CDBB2AC4294
:100E2000F1D10B70F5E700BFE08D012008B5FFF7A9
:100E3000BAFF10B100230B70137008BD0420704777
:100E400028B1034B93F9BC01003818BF012070474B
:100E5000F003012008B5FFF7F3FF50B1054B93F9FC
:100E6000BC21012AC9BF93F8BF310020C3F340035E
:100E70000B6008BDF003012008B5FFF7E1FF18B1D2
:100E8000024B93F8BE310B7008BD00BFF003012088
:100E900070B5FFF7D5FF38B10E4C94F8BF31DB07C2
:100EA00003D500230B70137070BD0B4D94F9BD3149
:100EB00095F8306093FBF6F301330B7094F9BD4164
:100EC00095F8301094FBF1F301FB134301331370D9
:100ED000EAE700BFF0030120E08D01200320704706
:100EE0000A4A70B592F8343006255E1CB6FBF5F45C
:100EF00005FB146492F83550AC421EBF02EBC303ED
:100F000082F83440C3E90E0170BD00BFE08D0120BE
:100F1000002230B504461046914200DC30BDA35C8F
:100F20000825584010F0800F4FEA400318BF83F0A7
:100F3000D503013DD8B2F5D10132EDE710B5D9B1F5
:100F40000E4B986E814217DCB2B11B6B9A4213DCD8
:100F5000013A01390A4C03FB012104F5E37084F8DE
:100F6000CA110521FFF7D4FF062184F8CB0104F54F
:100F7000E370BDE81040B3E710BD00BFE08D012075
:100F8000F00301200023038083708380C3800381EA
:100F9000704700BF074A084992F86C30097801335E
:100FA000DBB2994282F86C3004BF002382F86C30C7
:100FB000704700BFE08D012070070020F8B5774C26
:100FC000236F83B1764B1B6893F82E305BB1754B62
:100FD00094F87420A3FB0013012A4FEA93132FD037
:100FE000022A08D002B1F8BD6F4B9842FBD9012309
:100FF00084F87430F8BDA26F64329A423DD894F8F8
:101000006C3004EB031393F88C20FF2A06D00132D6
:101010006649012083F88C2081F8CC01FFF7BAFFE4
:10102000634B01221B7884F87420092BDBD1B4F8C0
:101030000E31604A01339BB2A4F80E315380F8BDE3
:1010400094F86C1004F180055B48002701EB8106E1
:10105000A367E567022500EB461355480A2684F886
:101060008A7000789A70092884F88B6084F874502C
:10107000B9D101314F4B1980F8BD94F88A2094F80A
:101080008B309A42AFD104F17F0004F18805002330
:1010900010F8011F08224B4013F0800F4FEA430164
:1010A0000B4616BF81F00703CBB2DBB2013AF3D196
:1010B0008542EDD194F88910994238D1B4F8836013
:1010C000012794F86C5076BA94F887C004EB0511A8
:1010D000B4F88500B6B294F8883040BA81F88C2014
:1010E00043EA0C23C1F8906094F881C080B294F870
:1010F00082601BB2C1F89400032D46EA0C2294F9D9
:101100008000A1F89830A1F88E20284A81F88D003F
:1011100082F8CC7108D8264A12780C2A29D00D2AD8
:1011200002D1244B23F81500FFF734FF5FE794F852
:101130006C3004EB031393F88C20FF2A06D00132A5
:101140001A49012083F88C2081F8CC01FFF722FF97
:10115000174B01221B7884F87420092B7FF443AFCE
:10116000B4F80C31134A01339BB2A4F80C319380CC
:10117000F8BD03EB83031149114A03EB830391F894
:1011800022100C48F9409B0093FBF1F382FB031201
:10119000DB17C3EBA20320F81530C5E7E08D012073
:1011A00008150020D34D62103F4B4C00F003012086
:1011B0001049012014490120A0260020D449012013
:1011C000676666660A4B93F88A1093F88B20914203
:1011D0000DD0C0B210B493F88A20DC6F511CD2B28B
:1011E000C9B283F88A10A0545DF8044B7047704769
:1011F000E08D01200F4B104AD3F81031B2F90000F6
:101200005B0707D400EB8000400080B200F5C87097
:1012100080B27047094B0A4AD3F8C430323382FB9C
:101220000312D817C0EBA20080B200F5C87080B2DC
:10123000704700BFE08D0120844B0020243A01203C
:101240006766666680F08003042B70B520D941285C
:101250001ED0FD2806D0F0281DD0EF281FD0022474
:10126000204670BD0B2004260F4D2E44002401356E
:10127000FFF7E8FF2044AE42C4B2F1D015F8010BED
:10128000FFF7E0FF2044AE42C4B2F7D1204670BD64
:101290000424204670BD03200526044DE5E70C20FC
:1012A0000626034DE1E700BF085E0608005E06085B
:1012B000F85D060870B5D0F8A052044695F81832CB
:1012C00013B9D5F814323BB981212046FCF712FE40
:1012D0006B7A022B07D070BD6B7A002BF4D1012101
:1012E000FCF708FEF0E705F5037220461F230121F5
:1012F000BDE87040FCF772BD70B5037C0446012563
:101300007BBB4FF4007302222946FCF759FE4FF4D1
:101310000073C4F85851174E812102222046FCF771
:101320004FFE321DE5620025D4F8A432C4F8A02295
:101330002846B581A6F860521B6898470121D4F869
:10134000A802FFF719FC8121D4F8A802FFF714FCCA
:1013500006F5047220461F230121FCF73FFD2846B5
:1013600070BD402302222946FCF72AFE4023C4F820
:101370005851D0E7844B002038B5044600250121A0
:10138000D0F8A802FFF72AFC8121D4F8A802C4F8FB
:101390005851FFF723FCD4F8A002E5624BF03EFE63
:1013A0002846C4F8A05238BD38B504468321D0F889
:1013B000A8020025FFF712FCD4F89802656518B161
:1013C0004BF02CFEC4F89852002038BD38B50446C6
:1013D00000258121D0F8A802FFF700FC0121D4F8F4
:1013E000A802E562FFF7FAFBD4F8A8028221C4F84C
:1013F0005851FFF7F3FBD4F8903225644BB1D4F881
:1014000094325B689847D4F890024BF007FEC4F81A
:101410009052002038BD00BF10B50823032283215D
:101420000446FCF7CDFD0123102063654BF0EEFD73
:10143000C4F8980218B103460020187310BD0220AA
:1014400010BD00BF2DE9F041037C04460125BBBB64
:101450004FF4007302228121FCF7B2FD29464FF4BC
:10146000007302222046E562FCF7AAFDC4F8585139
:101470004FF001080823032282212046FCF7A0FD3B
:101480004FF40770C4F840804BF0C0FD0546C4F827
:10149000900258B3D4F8943200271B689847267CF2
:1014A000C5F814724146D5F804222046C5F81872D2
:1014B000AEB140233E46FCF791FC3046BDE8F081DA
:1014C000402302228121FCF77BFD29464023022292
:1014D0002046E562FCF774FDC4F85851C8E74FF4A4
:1014E0000073FCF77BFC3046BDE8F0814646E4E73C
:1014F00007B50DF1060212F06BFA68B1084BBDF8A2
:101500000620B3F814111A8391421FBF0549142015
:10151000A3F8142181F8BB0103B05DF804FB00BF00
:10152000E08D0120F003012013B50446FFF788FC8D
:1015300000B300230DF106022046ADF8063012F08C
:1015400047FAB8B10C4C9DF8062094F9BC1184F808
:10155000D121032909484FF0050104BF62F07F0241
:1015600084F8D121FFF7D4FC062184F8D201034886
:10157000FFF7B6FC02B010BDF0030120BD0501204D
:101580002DE9FF47002304461E200193ADF80C30DF
:101590001D4B93F8009093F801A09D78B3F8048058
:1015A000DF881E7A20F0D8FA28B1002F1EBFB84677
:1015B00001254FF00009154A92F81631D9070AD4CF
:1015C00092F81B213AB9012E1BD0022E03D113F041
:1015D000020F08BF012501AB8DF80C608DF8049057
:1015E0008DF805A08DF80650ADF80880ADF80A70AA
:1015F00003CB1B88206020466160238104B0BDE8D6
:10160000F0873546E7E700BFD8520120E08D012082
:10161000144B30B4D3F8404114B383F84611090A8F
:1016200000220F2583F8450103F5A27083F84711C6
:101630000121C3F84821C3F84C21C3F8502183F895
:10164000445110F8015F01312A440E29D2B2F8D179
:1016500083F8522120461022034930BC2CF036BBBF
:1016600030BC7047E08D0120248F0120034B002106
:1016700083F85411C3F85811CAE700BFE08D012068
:1016800013B504462620019120F066FA019920B98D
:10169000204602B0BDE81040BAE702B010BD2DE907
:1016A000F743B74C0D46D4F840314BB14FF0020828
:1016B00000264FF00109D4F840012CF003FB58B983
:1016C0000027A37C042B00F25781DFE813F08F0082
:1016D000E400F7003D014601D4F840012CF0EAFA9D
:1016E000D4F858315A1C234483F85C0194F85431DF
:1016F000C4F85821012B0AD0022B11D0002B70D135
:101700000F280CBF84F85491C4F85831D3E7A0F1E6
:101710007203012B01D9762863D184F85481CAE77A
:10172000102AC8D197490023012211F8010F013274
:1017300003440E2ADBB2F8D194F86A2184F854618C
:101740009A42C4F85861B6D194F86B31002BB2D1EB
:1017500094F85D71732F37D0762F0DD0722FAAD1E8
:1017600094F85F2194F85E3153EA0223A3D02360FA
:10177000B4F860316360A4E794F85F2194F85E31B7
:1017800053EA022397D094F8611194F8602194F8F9
:10179000650142EA012294F862116361E17494F8F0
:1017A0006311A4F86C2184F86E1194F8641141EA75
:1017B0000021A4F87011A16801B9A360238B002B4C
:1017C0007FF47FAF22837CE794F8632194F8623141
:1017D00043EA02231AB2002B3FF46DAFA4F8722142
:1017E0006FE784F85461C4F8586164E7722F44D1FC
:1017F00001230022A374644B1B78402B2FD1634E2E
:10180000A37C94F86EC1208B33804FEA0C33050221
:10181000B4F86CE103F44053217C05F470657780E3
:101820006769704514BF042000202B434FEA0E1552
:1018300043EA8133614514BF02210021EDB22B43FD
:10184000A5681BB2BD4214BF0825002513432B43D6
:1018500018434F4B014393F8BB31B180F380A36E23
:101860001BB1E369002B40F09D801F2249494A4883
:1018700003B0BDE8F0434BF0F9BCD4F87431474AEB
:10188000EB1A934201DC0022B5E77220FFF7EEFE6F
:10189000C4F87451F7E7762F03D102230022A37412
:1018A000A9E7D4F874313D4AEB1A9342EBDD762078
:1018B000FFF7DCFE0022C4F874519CE7344ED4F8E4
:1018C000743196F8BB21EB1A82B3344A934230DD6F
:1018D000E27CD2071BD4A168626991420ED089B222
:1018E0004620FFF7CDFE96F8BB310122C4F87451B3
:1018F000013B86F8BB310423A3747CE7218BB4F849
:101900006C218A4203D05020FFF7BAFEEBE7217C1E
:1019100094F86E218A4206D0B1FA81F14920490932
:10192000FFF7AEFEDFE7142286F8BB211C4A934284
:10193000BDDC762FA7D17320FFF798FE032300228A
:10194000C4F87451A37456E7732F9CD0D4F8741163
:10195000124B691A9942A0DC95E7D4F874310F4A0A
:10196000EB1A93428FDD7620FFF780FE02230022E0
:10197000C4F87451A3743EE700231A46A3743AE7EF
:10198000E08D01203C8F01201049012014490120E5
:10199000F0030120B95D0608C30501203F0D0300D7
:1019A0003F420F00334D2A23D4F878610DF1020233
:1019B00085F8D33120230DF10101304685F8D4316B
:1019C00012F09DF830B19DF801109DF8027051EAB7
:1019D000070339D1552385F8D531462385F8D6310B
:1019E000202301A9304685F8D73112F082F803464A
:1019F000214813B1BDF804209ABB20493EF0AEF94E
:101A0000B4F870711E4D87B30DF10301304612F02A
:101A100073F850B30DF106029DF80310304611F033
:101A2000D7FF10B3BDF806203B4616492846BA42F8
:101A30000CBF20222A223EF091F9B4F87231A4F8AA
:101A40007C3103B0BDE8F083304612F03DF83946F2
:101A500085F8D501304612F023F8037885F8D631A1
:101A6000BEE709493EF07AF9CAE7084928463EF040
:101A700075F9E2E7F0030120C8050120DB5D0608E7
:101A8000CC050120D35D06083A9D0608DA5D0608FC
:101A900038B50B680C460E4D5A1C20460A600522CC
:101AA0001A700B6895F8BC21591C21601A702368C4
:101AB00095F8BF21591C21601A70B5F8C2113DF08C
:101AC000C7F8236895F8C421591C21601A7038BDE5
:101AD000F00301202DE9F0472DED028BFFF7B0F95F
:101AE000C8B31E4B93F9BC01012834DD93F8F241D1
:101AF00015461B4F8E1E02EB44089FED1A8A4FF0CD
:101B00003209454504D12046BDEC028BBDE8F08783
:101B100037F802ABB2EE040A07EE90AA26F802AF3D
:101B2000F8EEE70A60EE880A4AF06EF8BCEEC00AEA
:101B3000BAF10E0F10EE103A9BB209D91933B3FB6C
:101B4000F9F39BB203EB830303EB83035B009BB2CC
:101B500025F8023BD5E70024D5E700BFF0030120BC
:101B60005E8F0120CDCCCC3D38B50D46FFF768F92E
:101B7000044638B10C4890F8BF31DB0704D5B0F803
:101B8000C0012880204638BD084A00F5FA7010F9D7
:101B9000373C92F8302093FBF2F102FB1132013115
:101BA000013211F029FFECE7F0030120E08D012064
:101BB00038B5134C94F8353094F834209A4219D043
:101BC00004EBC3030F49D3E90E200023984212DC33
:101BD00093780D4A5B08C4F890011370FBF7C4FFBB
:101BE00094F8353006210133B3FBF1F201FB1233D7
:101BF00084F8353038BDD55C013301F8015BE5E789
:101C0000E08D0120E252012010530120AA4B1B78E5
:101C10002DE9F04F81468BB0002B40F0B680A74EE7
:101C2000D6F87851002D00F0B080A54AD2F8F841DE
:101C300004F0F021B1F1E02F6CD1C2F8F831D6F800
:101C40009421944266D004930DF11008C8F8043032
:101C50000DF11C0EA8F808309A4BC6F894419A88EA
:101C60001F78ADF8142093F801C01A7A93F802A0F7
:101C70008DF810708DF811C08DF812A08DF8182015
:101C800098E80700AEE803008F49AEF80020C4F3DF
:101C90004252895CC4F303428F4202F101021F46A3
:101CA00001D1944508D028468DF81C108DF81D20D0
:101CB00011F0A2FEADF82000284604F0070B12F048
:101CC000EEF8032833D0042835D000239A4501A923
:101CD000284618BF8DF81E3011F008FF48B1019B4F
:101CE000C4F3001103F001038B4202D0284611F027
:101CF000ADFF0A2207A940464BF098F950B19DF874
:101D00001E30BDF81C20BB70BDF820303A80BB806F
:101D10003EF0F8FA96F898A104AFDFF8A8B196F86B
:101D20009831032B7BD8DFE803F00A3376A3674BA7
:101D300013F80B30CAE7664B13F80B30C6E7394689
:101D4000284611F0D9FE044658B107A8FFF718FC41
:101D50009DF81E109DF810308B4260D0284612F07E
:101D600001F896F89831013303F0030386F89831AF
:101D70000CB99A45D3D196F81631DB0700D524B1BA
:101D80002B68494628461B6898470BB0BDE8F08F82
:101D900001A8FFF7F5FB96F816819DF8044008F0BE
:101DA0000108ECB1B8F1000F39D13A460DF1030149
:101DB000284611F0A4FE044688B307A8FFF7E0FB0D
:101DC0009DF81C109DF803309DF81D208B4203D117
:101DD0009DF81030934222D0284611F0CDFFC0E785
:101DE000B8F1000FBDD13946284611F082FE0446F5
:101DF000A8B107A8FFF7C4FBBDF82010BDF810304C
:101E00008B420CD086F89981284686F89A812B68F7
:101E10009B699847A5E796F81631D80701D50024A5
:101E20009FE707A9284611F061FE04460028F6D076
:101E30001E201FF091FE96F89B3180468342EED023
:101E400086F89B0160B1BBF80630002BE7D1079BF9
:101E5000D907E4D401212846444611F0F7FE80E773
:101E6000079BDA07DBD50146284611F0EFFE78E73D
:101E70003846FFF785FB07AB97E8070003C31A80D6
:101E80009DF810309BB10DF11D0207A9284611F0F5
:101E900036FE0DF11E01284611F02EFE0A2207A97A
:101EA00038464BF0C3F8041E18BF012459E708A9AF
:101EB000284611F01EFEECE726530120E08D01209C
:101EC000F0030120D8520120285E06081C5E060897
:101ED000105E0608FD292DE9F041044684B000F0AB
:101EE000D880F02900F0BC80EF2900F02B814AB1A6
:101EF0000346861803AD002003F8010B9E4205F847
:101F0000010BF9D19B4B0B2003F1090501E013F8FC
:101F1000010F814200F0C280AB42F8D14B1E832BEF
:101F200000F29280DFE813F01E01340184003E01CC
:101F3000AA01B001450150015C01900090006201CE
:101F4000620162017801780178015C0190009000E3
:101F500082018A0190009000900090009000900013
:101F600090009000900090009000900090009000F1
:101F700090009000900090009000900090009000E1
:101F800090009000900090009000900090009000D1
:101F900090009000900090009000900090009000C1
:101FA00090009000900090009F01900090009000A1
:101FB00090009000900090009000900090009000A1
:101FC0009000900090009000900090009000900091
:101FD0009000900090009000900090009000900081
:101FE0009000900090009000900090009000900071
:101FF0009000900090009000900090009000900061
:102000009000900090009000900090009000900050
:102010009000900090009000900090009000900040
:10202000900090009000900090009000190119011C
:10203000514B93F8AB11002900F05D81019223F020
:1020400035FB019AADF80C003AB103AB224413F80A
:10205000011B04F8011BA242F9D104B0BDE8F081D4
:1020600003214FF00508454FB8440025013701E032
:1020700017F8011B0846FFF7E5F8064660193246D7
:10208000FFF728FF7019B845C5B2F1D104B0BDE81B
:10209000F0810B214FF00408394FE5E7364BD3F8B8
:1020A000100180060CD4002AD7D003AB224413F8C9
:1020B000011B04F8011B9442F9D104B0BDE8F08182
:1020C00093F89C01870742D52E4D287D052834BF03
:1020D00002260326142917D97C39C8B20628E2D86B
:1020E0000629E0D801A050F821F000BFCF22010856
:1020F000CF220108B9220108A7200108DF22010828
:10210000D9220108E52201080929CCD90A390A296E
:10211000C9D801A757F821F09F220108EB22010836
:10212000A7200108A7200108A7200108A72001086F
:10213000A7200108A7200108A7200108B122010853
:10214000CF2201080C214FF006080F4F8CE70D4BF2
:102150000B29187DA7D10126C8E00C4BD3F8C0305D
:10216000039371E70192FFF745F8019AADF80C006F
:102170006AE700BFEC5D0608E08D0120005E0608FE
:10218000085E0608F0510120F85D0608243A012097
:10219000684BD3ED767AFDEEE77A17EE903AADF81C
:1021A0000C3051E7019223F081FA019AADF80C004E
:1021B0004AE7604D95F81631DE0700F1A580B5F8C5
:1021C000E831ADF80C303FE75B4B5C49B3F90430C4
:1021D00081FB0301DB17C3EBA103ADF80C3033E740
:1021E000544BB3F80432ADF80C302DE70C39544B96
:1021F0009FED547AC9B2D3ED9C7A03EB810367EE6D
:10220000877A93EDAE7A67EE877AFDEEE77A17EE7E
:10221000903AADF80C3017E70F39474B33F81130CF
:1022200003EB83035B00ADF80C300DE7414B93F8F3
:10223000163103F00103ADF80C3005E7424B198865
:10224000CD0556BFCB43032303F0010311F0440F28
:1022500018BF042311F0020F18BF072311F4806F79
:1022600018BF0923ADE70192FEF7C4FF374B019A6F
:10227000D3F8C83043EAC0400390E5E62D4BD3F8CD
:10228000F831ADF80C30DFE62A4BB3F8E81100293D
:1022900034D0019223F022FA019A80B2D2E62B8A3E
:1022A00003EB830303EB83039B00ADF80C30FAE6EA
:1022B000EB89ADF80C30F6E6EB89254903EBC30357
:1022C0009B00A1FB03135B09ADF80C30EBE6B3F800
:1022D0009E31ADF80C30E6E66B680393E3E62B68BD
:1022E0000393E0E6AB680393DDE6F6B28DF80C608D
:1022F0008DF80D00D7E6B3F8C401A3E6D3F80002C9
:1023000080F3100080B29DE6019221F05BF8D5EDDC
:10231000767A019AFCEEE77A17EE903A9BB20028A3
:102320007FF44FAF0B49096811F0100F18BF00235D
:1023300047E700BFE08D0120A05201206766666676
:10234000844B002000007A44C4520120243A01202A
:102350001F85EB51D8510120014B1B681B6A1847A0
:10236000F44A0120024B186808B183691847704786
:10237000F44A0120024B186808B1436918477047B6
:10238000F44A012010B5074C606D40B131F0EAF815
:1023900094F8513013B180F00100C0B210BD01209B
:1023A00010BD00BFEC1E01200368042201F01F01D4
:1023B000186A02FA01F120EA010010B418621A6AE0
:1023C0000A4C114319625A6C42F400425A649A68EA
:1023D0001440062C06D0B4F5803F03D01A6842F0B2
:1023E00001021A6000205DF8044B704707000100ED
:1023F000B1F5805FF0B400F0D4802AD8102900F045
:10240000F580B1F5807F4ED1046A166924F480749A
:1024100057689A4B0462016A446821F40071C569E7
:1024200041EA0621964E2B40156821F48071B04296
:1024300045EA030541EA072173D0924B984270D0D8
:10244000D26800234460C561C26301621846F0BCD3
:102450007047B1F5803F00F08180B1F5801F48D111
:10246000046A156924F480145668874B0462016A73
:10247000446D21F400112340146841EA0551804D58
:1024800043EA042421F48011A84241EA06515DD0B8
:102490007C4B98425AD0D26800234465C2650162E1
:1024A0001846F0BC7047012923D1046A166924F04C
:1024B00001045768714B0462016A446821F002010B
:1024C000856931436E4E2B40156821F00101B04201
:1024D00045EA030541EA07010FD06A4B98420CD048
:1024E000D268002344608561426301621846F0BCF3
:1024F00070470123F0BC18467047D2E9056321F00C
:10250000080124F4807441EA86011C439668D3696B
:1025100021F0040124F4007441EA860144EA4304F2
:10252000DEE7D2E9056321F4006124F4805441EA36
:102530008621966844EA0314D36921F4806124F467
:10254000005441EA862144EA431479E743689569D7
:1025500023F4802343EA852343609CE7046A1569DA
:1025600024F480345668494B0462016A446D21F4B6
:1025700000312340146841EA0541414D1C4321F4D8
:102580008031A84241EA064155D03E4B984252D094
:10259000D26800234465846D826501621846F0BCF0
:1025A0007047046A166924F480545768384B0462F3
:1025B000016A456821F40051C46941EA0631304E90
:1025C0002340146821F48051B04243EA042441EAD4
:1025D000073138D02B4B984235D0D2680023456064
:1025E000C461026401621846F0BC7047046A16694F
:1025F00024F010045768264B0462016A446821F0F5
:102600002001856941EA06111D4E2B40156821F015
:102610001001B04243EA052541EA071119D0194BD0
:10262000984216D0D26800234460856182630162BB
:102630001846F0BC70474368956923F4803343EA39
:1026400005234360A4E725F48045936945EA831593
:10265000C3E7D2E9056321F0800124F4806441EAF4
:102660008611966844EA8304D36921F0400124F47A
:10267000006441EA861144EAC304D3E78CFFFEFFFD
:102680000000014000040140FF8FFFFE8FFFFEFFAE
:10269000FF8CFFFE70B4344CB0F1804F0368A0EBA8
:1026A0000404B4FA84F44FEA541406D02CB92F4D24
:1026B0002F4A904218BFA8421DD12E4A23F0700322
:1026C0004D68821A2B43B2FA82F2520923F4407306
:1026D000D1E902652B430D880360C66285623CB96F
:1026E00032B9436943F0010370BC43610020704775
:1026F0000B7C0363F5E702F58062904220D002F57F
:10270000784290421CD01C4A1C4DA84218BF9042EF
:102710000CBF0122002224D0194EA5F59635A842FF
:1027200018BFB042D2D0174A90421AD002F5806248
:10273000904216D08C680A880360C4628262D0E737
:102740000C4A23F07003104D821A4E68A842B2FA68
:1027500082F243EA06034FEA5212B7D0002AB5D1FB
:10276000D1E70022B2E700BF0000014000040040B2
:1027700000080040000401400040014000440140C6
:1027800000480140001C0040000C00402DE9F04FC3
:10279000002383B0DFF810820D68DFF810E203E059
:1027A0000133102B00F0B88001229A4032EA050470
:1027B00005EA020CF4D14C6824F01007022F40F017
:1027C000AE80DF0803F0070A4FF00F0B0E6900EB35
:1027D00087074FEA8A0AD7F820900BFA0AFB06FA15
:1027E0000AF64FEA430A29EA0B094FF0030B46EABF
:1027F00009090BFA0AF604EA0B0BC7F820906FEAF6
:10280000060907680BFA0AFB27EA06064BEA0606E2
:1028100006608768C4F3001607EA090BCF689E407C
:1028200007FA0AF747EA0B078760476827EA0202B8
:1028300016434660C668E7008A6806EA090902FA94
:102840000AF242EA0902C260AAD5D8F8447023F01D
:10285000030903F003020F2647F4804709F180497A
:102860009200C8F8447009F59C39D8F8447006FA0B
:1028700002FA07F480470197444F019EB842D9F805
:10288000086026EA0A061AD007F58067B8425ED0CB
:102890003F4FB84260D03F4FB84262D03E4FB8423F
:1028A00064D03E4FB84266D03D4FB84268D03D4FED
:1028B000B8420CBF0727082707FA02F21643C9F8E7
:1028C00008606FEA0C07DEF80020E60303F101035D
:1028D00054BF3A404CEA0202CEF80020A203DEF8D0
:1028E000046054BF3E404CEA0606E202CEF80460A3
:1028F000DEF8086054BF3E404CEA0606A402CEF85B
:102900000860DEF80C2054BF3A404CEA0202102B5B
:10291000CEF80C207FF448AF03B0BDE8F08F4FEA4B
:10292000430A4FF00309D0F800B0013F04EA09065A
:1029300009FA0AF9012F2BEA090B06FA0AF66FEADF
:10294000090946EA0B0606603FF674AF61E7012706
:1029500007FA02F21643B2E7022707FA02F2164319
:10296000ADE7032707FA02F21643A8E7042707FAA0
:1029700002F21643A3E7052707FA02F216439EE781
:10298000062707FA02F2164399E700BF000002404B
:1029900000080240000C02400010024000140240F7
:1029A00000180240001C024000380240003C014078
:1029B00030B40023154C0168C36725680B681B07FA
:1029C00009D4002220231446436780F870208367CF
:1029D000204630BC7047CB6913F40013F1D1226854
:1029E000521BB2F1007FF6D30A682025032422F49B
:1029F000D0720A608A6822F001028A60456780F816
:102A000070308567204630BC704700BFF833012026
:102A1000436ADA0710B406D50168846A4A6822F46A
:102A2000003222434A609C0706D50168C46A4A689E
:102A300022F4803222434A60590706D50168046BAC
:102A40004A6822F4802222434A601A0706D50168A8
:102A5000446B4A6822F4004222434A60DC0606D5F1
:102A60000168846B8A6822F4805222438A60990646
:102A700006D50168C46B8A6822F4005222438A603A
:102A80005A060AD50168046C4A68B4F5801F22F41E
:102A9000801242EA04024A600BD01B0606D5026887
:102AA000816C536823F400230B4353605DF8044B9F
:102AB00070474A68446C22F4C00222434A60ECE743
:102AC000754B002108222DE9F0411D6882B0804637
:102AD0000191D0E9166334689A40224204D001681B
:102AE0000F68780700F18A8001229A40224204D0C0
:102AF000D8F800104969090678D404229A40224285
:102B000004D0D8F8001009688F0767D410229A40C3
:102B1000224204D0D8F800100F68380749D4202288
:102B20009A40224217D0D8F800100C68E00612D55F
:102B3000B26098F83520052A73D00B6813F4802F03
:102B40000B6800F09080190340F19B80D8F83C306E
:102B50000BB140469847D8F854303BB3D8F85430BE
:102B6000DA071BD5D8F8002005214C4B88F8351022
:102B7000A3FB0535136823F00103AD0A136002E0DF
:102B80001368DB0704D5019B0133AB420193F7D9EE
:102B90000022012388F8342088F83530D8F84C30EA
:102BA00023B1404602B0BDE8F041184702B0BDE88D
:102BB000F081B2600A6812F4802F0A682AD1D70522
:102BC00003D40A6822F008020A60D8F84020002ADC
:102BD000A5D040469047D8F85C30A0E7B260D8F85E
:102BE000542042F00402C8F854208FE7B260D8F8AD
:102BF000542042F00202C8F854207EE70F6827F004
:102C000004070F60B260D8F8542042F00102C8F8FF
:102C1000542069E71203D8D5D8F84820002AD8D123
:102C20007DE70A68D8F8404022F016020A604A6937
:102C300022F080024A6154B30A6822F008020A6056
:102C40003F220024012102FA03F3D8F85020B36098
:102C500088F8344088F83510002AA7D0404602B0E2
:102C6000BDE8F041104713F480737FF46FAF0A683A
:102C7000012422F010020A6088F8343088F83540C8
:102C800064E7D8F84430002B7FF463AF63E7D8F8EB
:102C90004820002AD0D1D3E7F42B0120B5814E1B68
:102CA00090F835200346022A03D0802201205A657D
:102CB000704702680521002083F83510136823F05F
:102CC00001031360704700BF70B5324A002590F8C9
:102CD0004130044680F84250283BC2624585426C30
:102CE000022B41EA020141642BD80321FDF788FE43
:102CF0002822294B80F8412043630563226813682A
:102D000013F4804312D01368A06B23F48043136044
:102D1000B0B1224A0023026584F84030FFF7C0FFBB
:102D200070B1A06BBDE87040036D1847116811F4D5
:102D3000004114D194F84130602B24D084F8401025
:102D400070BD0721FDF75CFE90F84130602B02D08A
:102D5000202380F84130002323636363CEE71168AA
:102D6000E06B21F4004111600028E9D00B4A0265B4
:102D700084F84030FFF794FF0028E1D0E06BBDE815
:102D80007040036D1847202384F8401084F84130C8
:102D900070BD00BF0000FFFF8D2E01088D0A0108E5
:102DA0000368202270B51E680D46DA6107210446CB
:102DB000FDF726FE03683348596841F40041596025
:102DC0005A6802405A609A69910701D500229A62B6
:102DD0009A69D20703D49A6942F001029A61700499
:102DE0002BD5A26B1AB11268526892B262856A073B
:102DF00009D55A6A25F00405636A1A70636A228D40
:102E0000013363624ABB638D9BB21BB1636C43F0B9
:102E1000040363640023236384F84230666C6363B5
:102E200016BBE36A184DAB420DD194F84130202314
:102E300084F8406084F8413070BD3104D7D5E26B2E
:102E4000002AD0D1D3E72046FDF75AFE2023E562C1
:102E500084F8406084F8413070BD638D013A013BD5
:102E600022859BB26385CEE7616C2046FFF72CFF7D
:102E700094F84130282BDFD129462046BDE8704028
:102E8000FDF712BE00E800FE0000FFFFF8B590F865
:102E90004030C66A012B00F0848017460123CA0621
:102EA00004460D4680F8403020D5FB061ED5438DE4
:102EB0009BB2002B62D190F84130B6F1007FDBB2BB
:102EC00002D1282B00F0848094F841301021292B66
:102ED0002368D96102D116F5803F68D1AA0601D5D1
:102EE000BB0659D4002084F84000F8BD680710D410
:102EF0002A072ED53B072CD594F8413003F0280340
:102F0000282B61D0216808200023C86184F8403054
:102F1000E4E77907ECD5638D9BB27BB1216825F09E
:102F20000405636A496A1970638D606A218D013BEB
:102F300001309BB20139606263852185638D9BB24C
:102F4000002BCBD116F5803FC8D02046FDF7D8FD29
:102F5000C4E7A807C2D5B907C0D5638D9BB213B328
:102F6000606A236810F8016B218D9E62638D0139C0
:102F70006062013B21859BB26385AFE70368102146
:102F8000D961436C43F00403436436F08073A5D1E8
:102F9000416CFFF799FEA1E729462046FFF700FFA5
:102FA000A0E70220F8BD36F0807397D1CDE799698C
:102FB0008A0701D5002199629969CE07C5D499691C
:102FC00041F001019961C0E72046FDF73BFD85E72F
:102FD000FDF76AFD82E700BF38B520220368204D67
:102FE0000024DA615A682A401E4D5A600463446323
:102FF000CC06C56205D51022DA61426C42F00402AB
:1030000042649A69910701D500229A629A69D207AF
:1030100003D49A6942F001029A610321FDF7F0FCA2
:10302000436C90F84120602A0CD01A1E18BF012270
:1030300043B990F84130212B08D090F84130222B31
:1030400004D038BD416CBDE838403DE6202380F80F
:10305000402080F8413090F8423080F8422038BD5E
:1030600000E800FE0000FFFF38B590F8403004464D
:10307000C06A012B71D0012384F84030CB0615D5EE
:10308000D50613D5D30BC2F3803543EA9232D2076B
:1030900029D5E26B5AB3DB0729D513685B6833BBCC
:1030A000A36B53B34DB31B685B6826E00B0707D4D3
:1030B000880601D5930612D4002084F8400038BD5C
:1030C0001507F5D594F8413003F02803282B46D096
:1030D000236808220020DA6184F84000EFE72046E8
:1030E000FFF75EFEE8E723681022DA61E4E7A36BEE
:1030F00023B31DB31B685B6803BB94F84130282BD6
:1031000002D1B0F1007F2ED094F841301022292B4B
:103110002368DA61D0D110F5803FCDD09A6991074C
:1031200001D500229A629A69D20703D49A6942F0C3
:1031300001029A612046FDF7E3FCBDE723681022F7
:10314000DA61636C43F00403636430F08073B3D1DD
:10315000616C2046FFF7B8FDAEE7022038BD20467F
:10316000FDF770FCA8E72046FDF79EFCA4E700BF32
:10317000F8B590F84030012B7BD00123CD060446F2
:1031800080F8403023D5D00621D510222368616B0A
:103190004548DA61626C814242F00402626466D0A2
:1031A000424A914263D0F4211A680A431A609A692C
:1031B000910701D500229A629A69D20703D49A69CD
:1031C00042F001029A61002084F84000F8BD0B062D
:1031D00031D5570643D523681A6822F040021A6099
:1031E000628D92B2002A46D05868618DC0F3090002
:1031F0008AB2FF2A4BD8628DE56A91B215F5803FFD
:103200002185CDB24BD0E76A2D045A68284E324052
:1032100002433A432A435A60628D521A92B262853F
:1032200094F84120222A1A680CBF42F4004242F46A
:1032300080421A60C7E74D0611D550060FD5638D41
:103240009BB2FBB923685A689101BCD4E26A12F5BB
:10325000803F13D15A6842F480425A60B3E78B062C
:10326000B1D59206AFD52046FFF7B6FEABE7602199
:103270009AE70220F8BD5B689E0103D42046FDF763
:1032800063FCA0E740212046FFF71EFD9BE7FF22DD
:103290004FF47F054FF0807711462285B5E74FF058
:1032A00000772D04B1E700BF6930010871310108D2
:1032B000009C00FC90F84030012B00F09C80012322
:1032C0002DE9F041044680F84030C8060D4690468E
:1032D0001BD512F0100F18D023681021D961616C32
:1032E00041F0040161649969890701D5002199625F
:1032F0009969CA0764D5AB0602D518F0200F71D1C1
:10330000002084F84000BDE8F0816B0712D4AF07BD
:1033100024D518F0020F21D0606A236810F8016BE1
:10332000218D9E62638D01396062013B21859BB2D4
:103330006385E0E718F0040FE9D0216825F0040563
:10334000636A496A1970638D606A218D013B01309F
:103350009BB20139606263852185CCE72E0615D4C6
:103360006906C8D518F0400FC5D0638D9BB2002BFD
:1033700033D1236859688A01BDD4E16A11F5803FD1
:1033800027D1596841F480415960B4E718F0400FE3
:10339000B1D0638D9BB2C3B1238DB3B920684168AE
:1033A000638DC1F309019BB2FF2B26D94368FF2728
:1033B000204E27853340204E19430E4346609AE73E
:1033C000996941F00101996195E723685B6898016B
:1033D00003D42046FDF7B8FB8DE740212046FFF7D8
:1033E00073FC88E720462946FFF7F6FD002084F8A5
:1033F0004000BDE8F08102207047638DE66A9BB211
:1034000016F5803F23850AD0E76ADBB24668094A91
:1034100016403E4346EA0343194341606BE7466862
:10342000DBB2044F3E40314341EA034343F00073B3
:10343000436060E7009C00FC0000FF01F0B404461C
:1034400090F834000128A66D38D0012594F8350095
:10345000A84284F8345005D00023022084F8343088
:10346000F0BC704725680227002084F83570A768F3
:1034700060652868402F20F4802028606B601AD097
:10348000A960EA60E16D3F23226C8B40B3602B683A
:1034900043F016032B606B6943F080036B611AB134
:1034A0002B6843F008032B602B68002043F00103D6
:1034B0002B60F0BC7047AA60E960E3E70220F0BC33
:1034C000704700BFF0B490F83530022B37D0036856
:1034D00000221D492126DCB21D68103C25F00105A3
:1034E0005F2CA1FB04711D60184F4FEA11111A6087
:1034F0005A609A60DA601A618CBFA2F58062144A41
:103500005E6188BF1A407D5C98BF1A404FF03F0152
:103510004FF0000388BF0432C565A9401C46826590
:103520009160436580F8343080F83530C0E90F335E
:10353000C0E91133C0E913332046F0BC7047DCB258
:103540002046F0BC704700BFABAAAAAA8CD80508D9
:1035500000FCFFFF0246F0B4494C2068002A56D018
:1035600002231168002582F8353082F834500B6848
:1035700023F001030B6003E023681B1A052B3ED8E0
:103580000B68DD07F8D4D2E90130D56803430F6832
:10359000D2E904402B432343146AD2E9066503436E
:1035A0003848334338402B43556A2343042D40EABF
:1035B00003002FD008604B6923F007031D43CBB2F3
:1035C00031484D61103B314CA0FB03505F2B304B19
:1035D0004FF001054FEA101003EA01034FF03F01DD
:1035E000205C4FF0000488BF04338140D065204642
:1035F00093659960546582F83550F0BC7047032399
:1036000020211846516582F83530F0BC7047012002
:10361000F0BC7047D2E90B74936A3C4320430860C6
:103620004D6925F007051D4345F00405002FC6D060
:103630007EB1B6F5005F12D0022B03D9032BBED1A9
:10364000FB01BCD5012340211846516582F8353075
:10365000D3E7012B10D033F00203B0D1F0E7032BF6
:10366000ADD801A050F823F04536010841360108D5
:103670004536010879360108B7F1C07F9FD1E1E7EF
:10368000F83301203F8010E0ABAAAAAA8CD8050825
:1036900000FCFFFF0023C0E90033C0E90233C0E9AA
:1036A0000433C0E90633C0E90833C0E90A33C0E98E
:1036B0000C338363704700BF1F4BF0B4595C044662
:1036C000D2E90236451810693343566967580343F7
:1036D00090693343D6690343906A3343174E0343DB
:1036E0003E40D06A3343635090B16E69176B26F049
:1036F0000706536B3843976B30436861605820F07E
:10370000C07018436050635823F4C0033B436350B8
:10371000566800201368EE60AB60094E6B681E406F
:10372000D2E908321E436E60635823F0F05313430E
:103730006350F0BC704700BFE05D06081F80FCFFCF
:103740000000FFFF30B4614C0346614A655C0C1E0B
:1037500018BF0124821A405918BF012220F001002D
:10376000585192B98CB95B4A0021212011605160F7
:103770009160D160116150615A5922F0F0525A5152
:103780003F2200209A6030BC70475348181A18BF77
:10379000012014B908B9514AE6E74C1E18BF0124AC
:1037A0001ABB14BB4E4A0020212410605060906068
:1037B000D060106154615A5922F0F0525A510129D7
:1037C0000DD0022915D0032924D0042927D005299A
:1037D00014D006292BD0072935D00120D3E74FF488
:1037E0007462002030BC9A60704760B95CB93D4A91
:1037F000D9E74FF47C1200209A60C4E74FF474625A
:103800000020DA60BFE78C1E18BF01245AB954B9F2
:10381000354AC8E74FF0746200209A60B3E73F2250
:103820000020DA60AFE738B934B9304ABBE74FF46B
:103830007C120020DA60A6E7CC1E18BF01243AB93A
:1038400034B92B4AAFE74FF074620020DA609AE790
:1038500010B90CB9274AA6E70C1F18BF012412B9EA
:103860000CB9254A9FE710B90CB9244A9BE74C1FB5
:1038700018BF012412B90CB9214A94E710B90CB948
:10388000204A90E78C1F18BF012412B90CB91E4AB8
:1038900089E710B90CB91D4A85E70D4A934203D157
:1038A000072901D11A4A7EE71A4A00202124106014
:1038B00050609060D060106154615A5922F0F0520B
:1038C0005A5100297FF47BAF5AE700BFE05D06083C
:1038D0000060024010600240006402401064024038
:1038E0002860024028640240406002404064024078
:1038F00058600240586402407060024070640240A8
:103900008860024088640240A0600240A0640240D7
:10391000B8600240B86402402DE9F8433C4E337D64
:10392000012B6DD0012380460F463375F7F718FA47
:10393000054600285FD14FF0FF333B60D8F80030D8
:10394000012B3DD0D8E901934B444B4553D9314C21
:103950002DE0022B0CBF4FF400734FF4407322692B
:1039600022F440722261226913432361236923F008
:10397000F8032361236943EAC90343F00203236187
:10398000236943F480332361BFF34F8FF7F7E8F9DE
:10399000236923F07A032361002835D1D8F8083051
:1039A00009F10109D8F8042013444B4523D998F8AC
:1039B0000C30002BD3D0012BCBD14FF48073CEE74A
:1039C000144CD8F80C3022691B0222F440729BB2CE
:1039D0002261226942F0040222612269134343F406
:1039E00080332361BFF34F8FF7F7BAF92369054698
:1039F00023F004032361002328463375BDE8F883D0
:103A000002252846BDE8F8830546C7F80090F2E78E
:103A1000B8490120003C02400B4B01E0013B10D0B3
:103A20000269002AFADA0369074A43F001030361D5
:103A300001E0013A05D0036913F00103F9D11846FA
:103A400070470320704700BF400D0300144B10B4B3
:103A5000046C9C421AD800F53060002301290361F0
:103A6000036943F400230361036943F0180303610E
:103A7000036943F0C043036104D14261036843F02A
:103A80008023036000205DF8044B7047D0F8003BB2
:103A900000F53060002BE0DA00205DF8044B704741
:103AA0000A30544F4B78012BF0B50D7826D000F535
:103AB0003060404C404B00EB45104D690669344086
:103AC00004610469234003618B6805B14B6104699B
:103AD000C3F31203012A44F400240461046943EA95
:103AE0000403036105D0036843F00443036000202E
:103AF000F0BDCB68002BF6D04361F4E74B6993B37C
:103B000000F510642B4FD1F808C004EB45142A4E81
:103B10006345D4F810E00EEA07072761276906EA33
:103B200007062661266938D946F40026C1F814C074
:103B3000CCF31203012A2661266943EA06032361B6
:103B400026D0BCF1000F08D005F00F020125D0F8F7
:103B5000343895401D43C0F834582368002043F0A2
:103B600004432360F0BD00F51060134EA3F500235D
:103B7000012A00EB4514206906EA00062661206947
:103B800040F400202061206903EA00032361E4D1AE
:103B90000B69002BE1D06361DFE746F40026C3F335
:103BA0001203012A2661266943EA06032361CBD169
:103BB000EEE700BF0000F8FFFFFF07E02DE9F0434C
:103BC0004D780F78012D4DD000F530636F4E4C6964
:103BD00003EB47136E4D1F693E401E611E69354061
:103BE0001D616CB38D68012A6A4E2C441F6904F173
:103BF000FF34B4FBF5F41FFA84FC06EAC44405FB69
:103C00000CF544EA0704C5F312051C611C6945EA7A
:103C100004051D6121D0CA78012A0AD1D0F80828EC
:103C200012F4807F1A680CBF42F0005242F08052BA
:103C30001A601A6842F004421A600020BDE8F0835E
:103C40008C68012A1D69C4F3120444EA05041C614E
:103C50001C6944F400241C61DDD1CA68002ADAD052
:103C60005A61D8E74B6900F51064002B37D104EB9B
:103C70004714474E454D012AD4F810C00CEA0606F9
:103C80002661266946F400262661266905EA0605AE
:103C90002561CE7872D0012E59D1D0F8085815F48C
:103CA000807F25680CBF45F0005545F080552560A4
:103CB000256845F004452560002ABED19BB2033338
:103CC0009C08BAD0CA6800F5805302EB840403EB69
:103CD000073352F8041BA2421960FAD1ADE704EB96
:103CE0004714D1F808E0DFF8A490C3F31206D4F823
:103CF000108003EB0E0C08EA09090CF1FF3CDFF819
:103D00009080C4F81090D4F81090BCFBFEFE09EA35
:103D10000808DFF880C0C4F810800CEACE4CD4F854
:103D200010E04CEA0E0CC4F810C0D4F810C046EAFB
:103D30000C062661CE78012E10D0012A22D007F081
:103D40000F03D0F834789D403D43C0F834582368C1
:103D5000002043F004432360BDE8F0832569012A75
:103D600025F0C0452561256945F00055256194D1B0
:103D70000D69002D91D0164665618CE70D69002D07
:103D800089D0F9E70D69002DF6D1E0E70000F8FFD2
:103D9000FFFF07E00000F81F70B41D4E056803E048
:103DA0003468A41AA14226D3AB6913F02003F7D0DC
:103DB00010222023EA61EB61AB699A0701D5002349
:103DC000AB62AB69DB0703D4AB6943F00103AB61C2
:103DD0006B6800220F4C202123406B60436C80F8FD
:103DE000402043F00403436480F8411080F84220EF
:103DF000012070BC7047426C202180F840300A439B
:103E0000426480F8411080F84230012070BC704755
:103E1000F833012000E800FE2DE9F041DFF854807E
:103E200004460E4615460AE09B69DB0602D5FFF7FD
:103E3000B3FFE0B9D8F800305B1BB34209D8236860
:103E40002A46314620469F69BF07EDD50020BDE8D0
:103E5000F081636C2021002201200B4384F8402074
:103E6000636484F8411084F84220BDE8F0810120A9
:103E7000BDE8F081F8330120F0B484460568049F62
:103E8000104E03E03468E41B9C420AD8AC6931EA66
:103E900004000CBF012400249442F3D00020F0BCA5
:103EA0007047DCF844302021002201200B438CF8BD
:103EB0004020CCF844308CF841108CF84220F0BC03
:103EC000704700BFF833012003689A69196810B47D
:103ED000D4052FD50C061FD5416C4FF4807441F0EA
:103EE000010141645105DC6129D5416C4FF48064C6
:103EF000920541F008014164DC6106D5426C4FF443
:103F0000007142F002024264D961416C11F00B0F62
:103F10000CD15DF8044B70475405F6D49405F4D5E4
:103F20000906EBD4416C11F00B0FF2D05DF8044B95
:103F3000FEF7CABE5405F1D50906D6D4E5E79205C9
:103F4000DCD4E2E70268436B9169126803B1184759
:103F5000704700BFF0B490F841200346002A40D0DB
:103F60002420DC68D3E9002183F84100012C10688B
:103F700021F0706120F0010010601161916821F45E
:103F800000419160996828D041F40441022C91606D
:103F900002D14FF40061516051680020134C20267B
:103FA0009F690C43D3E9041554602943DC69D56843
:103FB00041EA07211F6A25F400453C43D560D160E2
:103FC0001460116841F001011160586483F8416088
:103FD000186383F84200F0BC704741F400419160DF
:103FE000DAE702F0FF0180F84010B9E70080000234
:103FF000F8B501F00F05012600271C21C5EBC5040B
:1040000001FB050100EB84043C31A264236584F8C4
:104010003C50676584F83D600369B34208BFE264C1
:10402000DAB200681DB9FFF73DFD0020F8BDFFF7CB
:10403000C5FD0020F8BD00BF2DE9F0410A46D0F8CB
:10404000A05200270B4E044685F838222F7205F542
:104050000B720D238121C5F82C62D0F8A802FFF75E
:10406000C7FF05F5037220461F230121BDE8F0417B
:10407000F9F7B4BE555342532DE9F047137882B097
:10408000914604468A465A2B5CD8DFE813F0D000EC
:104090005B005B0080005B005B005B005B005B0023
:1040A0005B005B005B005B005B005B005B005B0038
:1040B0005B00B5005B005B005B005B005B005B00CE
:1040C0005B00AB0177005B005B0077005B005B008F
:1040D0005B005B00CE015B00F8015B005B003D0113
:1040E0005B00E2005B005B005B005B002A015B00A1
:1040F0005B005B005B005B005B005B005B005B00E8
:104100005B005B005B005B005B005B005B005B00D7
:104110005B005B005B005B005B005B005B005B00C7
:104120005B005B005B005B005B005B005B005B00B7
:104130005B005B005B005B005B005B005B005B00A7
:104140005B001902D0F8A0120524002091F85D321E
:104150005A1C01EBC303D2B283F83C4283F84002FD
:10416000042A15BF4FF0FF354FF0FF3581F85D226F
:1041700081F85D02284602B0BDE8F087D0F8A03291
:10418000002005465881284602B0BDE8F087D0F8E7
:10419000A042002104F10B0304F11D0003F8011FEC
:1041A0008342FBD1702094F85C320C25207394F884
:1041B0005D02E574984213D004EBC300013390F81C
:1041C0003C52DBB2A573042B90F84152257690F84F
:1041D000400218BF84F85C32607608BF84F85C1235
:1041E0001223638199F80430122B98BF6381002554
:1041F000284602B0BDE8F08799F80130D0F8A00257
:10420000DB0740F18081072100F1120300F10B056B
:1042100083224181C3F10604D44900E0127A03F8F5
:104220000129E218AB4211FA82F2F7D1DFE7D0F8A8
:10423000A062D6F81472002F40F02582D0F8A43284
:1042400008469B6898470546002840F052827081D6
:1042500090E7D0F8A062357A002D40F0898196F978
:104260001832002BC0F26E81D0F8A43208469B6849
:1042700098470746002840F07B82D4F8A432504685
:10428000DB6898470546002840F05F82D9F80210A5
:10429000D4F8A00209BAD0F86072C6F86412B9F86E
:1042A00007305BBA9BB21944C6F86832B94200F2D3
:1042B0007082B6F85E12D6F8142203FB01F3934223
:1042C00040F09781B3F5007F4FF00101204606F1E1
:1042D0000C0228BF4FF4007331729BB2F9F77EFDD8
:1042E00048E799F80150D0F8A03215F0020040F0EC
:1042F0001A82D3F86012D3E9992422448A4200F248
:10430000E7810546588135E7D0F8A08298F8086023
:10431000002E40F0298198F91832002B80F2C681D6
:10432000D0F8A43208469B6898470546002840F01C
:104330004282D9F80200D4F8A06200BAD6F86072BE
:10434000C8F86402B9F807305BBA9BB21844C8F8E1
:104350006832B84200F2F680B8F85E22022003FB11
:1043600002F3D8F8142288F808009A4240F0EA8054
:10437000B6F85E324FF4007CD6F8687206F10C0590
:10438000D4F8A422504607FB03F72946A8F80AC030
:104390006745D2F81080D6F8642228BF6746B7FB7D
:1043A000F3F39BB2C0470028C0F259812A463B462E
:1043B000D4F8A8028121FFF71BFEB6F85E52D6F8AA
:1043C0003432B7FBF5F5D6E99920DF1B2A44451BAB
:1043D000C6F83472C6E99925002D7FF408AF03238F
:1043E0003372C7E6D0F8A072082000225F4E07F1B2
:1043F0001303788107F10B05C3F1070000E0127C7D
:1044000003F80129C2189D4216FA82F2F7D1D4F8B6
:10441000A4325046DB68984700283FF4E8AEBB7BE7
:10442000002563F07F03BB73A4E6D0F8A0620025EB
:1044300006F10B0306F1170203F8015F9342FBD16B
:10444000D4F8A43250460DF1020201A95B689847E6
:10445000002840F0DE80019B0821BDF802200220E8
:10446000013BF17352BA0C211C0EF374F2821A0C48
:104470001B0A34747274B374B0827181B7E6D0F8D9
:10448000A0620846D4F8A43206F25E2206F518713E
:104490005B6898470546002840F0CE80D6F8603229
:1044A0000821B6F85E22013B308252BA7181180EA3
:1044B000F373190C72821B0A30737173B37359E66C
:1044C000D0F8A07208200022284E07F1130378814B
:1044D00007F10B05C3F1070000E0127E03F8012984
:1044E000C218AB4216FA82F2F7D1D4F8A432504681
:1044F000DB68984700283FF47AAEFB7B002563F029
:104500007F03FB7336E6D4F8A44201EBC10199F8AE
:104510000430E46904EB810422790532934228BF18
:1045200013464381002B3FF462AE013B9AB2531C09
:104530000C322344024413F8011D9C4202F8011975
:10454000F9D154E696F85D3205211A460133DBB203
:1045500006EBC202042B82F8405282F83C1200F0B3
:10456000A28086F85D3242E6464601E78CD805080F
:10457000B6F85E5206F10C08D6F868720846D4F810
:10458000A432414607FB05F7D6F86422D3F814900D
:10459000B7F5007F28BF4FF40077B7FBF5F39BB268
:1045A000C8470028C0F22A81B6F85E02D6F8343235
:1045B000B7FBF0F1D6E99925DB1B0A446D1AC6F862
:1045C0003432C6E9992525B920462946FFF734FD3E
:1045D000D0E505FB00F3424620460121B3F5007FFC
:1045E0004FF0000528BF4FF400739BB2F9F7F6FBBC
:1045F000C0E590F85D3205215A1C00EBC303D2B22E
:1046000083F8405283F83C12042A39D080F85D22A6
:10461000EDE5D4F8A022022092F85D32591C02EB9D
:10462000C303C9B283F8405283F83C02042900F066
:10463000D68082F85D12DAE5D4F8A02202200025A7
:1046400092F85D32591C02EBC303C9B283F83C02F5
:1046500083F840520429ECD182F85D528AE5D4F8FF
:10466000A0220420002592F85D32591C02EBC303FE
:10467000C9B283F83C0283F840528142D9D1EBE7BA
:1046800080F85D5276E596F85D32052100251A46E0
:104690000133DBB206EBC202042B82F83C1282F833
:1046A00040527FF45EAF86F85D5263E598F85D3264
:1046B00005211A460133DBB208EBC202042B82F853
:1046C000406282F83C1200F08D8088F85D328EE501
:1046D00093F85D22052411460132D2B203EBC101E9
:1046E000042A81F8400281F83C427FD083F85D22A1
:1046F0007DE5D4F8A0220220002592F85D3219460B
:104700000133DBB202EBC101042B81F8407281F866
:104710003C0218BF82F85D324FF0050308BF82F8F3
:104720005D72337226E593F85D220520002511465F
:104730000132D2B203EBC101042A81F83C0281F8B4
:104740004052D3D183F85D5214E5D4F8A022022060
:1047500092F85D3219460133DBB202EBC101042B42
:1047600081F8407281F83C0244D082F85D323EE527
:10477000D4F8A022022092F85D3219460133DBB250
:1047800002EBC101042B81F8405281F83C02ECD1CC
:1047900062E790F85D3205211A460133DBB200EB87
:1047A000C202042B82F8405282F83C123FF468AFF8
:1047B00080F85D321BE5D4F8A022022092F85D3229
:1047C00019460133DBB202EBC101042B81F84062D0
:1047D00081F83C02C9D1354682F85D62CAE482F8AC
:1047E0005D5204E5354688F85D62C3E4054683F80A
:1047F0005D02BFE43D4682F85D72BBE4D4F8A022BE
:104800000420002592F85D3219460133DBB202EB39
:10481000C101834281F83C0281F84052A5D11BE7D7
:10482000D0F8A01210B50B7A022B07D0033B012B56
:1048300002D80021FFF700FC002010BD01F21B226E
:1048400091F819120446FFF717FC0028F4DA204605
:104850000121FFF7F1FBEFE7F8B5D0F8A0420546DC
:10486000267A5EB1012E07D104F21B2294F81912A8
:10487000FFF702FC00282FDB0020F8BDD0F8A8329B
:10488000D4F81012D3F83032D4F814221F2BC4E914
:104890008C1208D12D4BD4F80C229A4203D194F8F3
:1048A000191201291DD994F85D32002105205A1CE6
:1048B00004EBC303D2B283F83C0283F84012022314
:1048C000042A2846637214BF84F85D2284F85D12BE
:1048D000FCF7F0FC0020F8BD28460121FFF7ACFBF7
:1048E000CAE794F81A32013B0F2BDCD804F21B22E2
:1048F000FFF7C2FB0028237A1DDB013B022BBBD94B
:104900006189F1B1D5F8A07204F10C020420D7F846
:104910003432D7F814425B1A87F83862A1423872F1
:10492000D5F8A802C7F834320B4628BF23468121A8
:10493000FFF75EFBA0E7052BCED02846FCF7BAFCBC
:104940009AE72846FFF778FB96E700BF55534243A6
:1049500070B5D0F89062E6B101EB810500EB8505FA
:10496000EB695BB1D0F8A802C1EBC10400EB840491
:10497000626CB3FBF2F402FB14341CB10020C6F8E5
:10498000140270BD23462246EC61FFF731FB20463E
:1049900070BD022070BD00BF002310B504241A466C
:1049A0001946C0F86C42D0F8A802FFF721FB00209E
:1049B00010BD00BF70B5054641B9D0F86C320C4649
:1049C000032B10D0052B1FD0002070BDD0F88C32E7
:1049D0009B6933B190F87422032A02D198470020D2
:1049E00070BD022070BDD0E953639E4212D8D0F84A
:1049F0008C321B6923B190F87422032A00D19847A6
:104A00002846FFF7C9FFDFE7C5F86C12F9F772FA1D
:104A1000204670BDF61AB342C0F84C6128BF334639
:104A20009BB2F9F7DBF9204670BD00BF10B5134605
:104A300002240A460021C0F86C42C0E90733D0F8CE
:104A4000A802FFF7D5FA002010BD00BFF0B5002383
:104A500083B00E460446ADF806300B78D0F8A0724D
:104A600013F0600522D0202D19D14A78FE2A11D0EA
:104A7000FF2A14D14A8892B9CD8885B91B060ED475
:104A80004FF4807107F503721F2339810121F9F773
:104A9000A5F908E04D8815B9CE88012E73D02046BF
:104AA0000225F9F783FA284603B0F0BD4B780B2BAB
:104AB000F5D801A252F823F0F74A01081F4B01086C
:104AC0009F4A01089F4A01089F4A01089F4A01081E
:104AD0009F4A01089F4A01089F4A01089F4A01080E
:104AE0000D4B0108E94A010890F87432032BD6D126
:104AF0008B787B60D7E790F87422032ACFD102220B
:104B00000DF106011D46FFF791FFCCE790F87432D6
:104B1000032BC4D1391D0122FFF788FFC3E70979B0
:104B2000D0F8A802FCF728F83179D4F8A802FCF7ED
:104B300055F8B38896F9042003F00F03002A4FF0CC
:104B4000000203EB830304EB83032ADBC3F8442155
:104B5000237C9BBB4FF40073022201212046F9F70E
:104B60002FFA0123C4F85831D4F8A0727B7A022BB3
:104B700032D03279D20996D0012B94D0204601212F
:104B8000FFF75AFA8FE71A0689D5D0F8A4329B6945
:104B9000984703463246204639463B60FFF746FFBA
:104BA00081E79A61237C83B94FF40073022281214B
:104BB0002046F9F705FA0123E362D5E740230222F4
:104BC00001212046F9F7FCF9CBE74023022281219D
:104BD0002046F9F7F5F9EEE720468121F9F78AF941
:104BE00000237B725FE700BF10B50C7882B0002312
:104BF000D0F8982214F06004ADF8063016D0202CBE
:104C00000ED14B78023B092B0AD8DFE803F0333989
:104C10000909090909093F2F90F87432032B5AD06A
:104C20000224F9F7C3F9204602B010BD4B780B2BD4
:104C3000F6D80FF2080C5CF823F000BFC14C010855
:104C4000214C0108214C0108214C0108214C01088C
:104C5000214C0108974C0108214C0108214C010806
:104C6000214C0108194C0108B34C01088B78002431
:104C70001360D8E7111D01220024FFF7D7FED2E709
:104C8000114601220024FFF7D1FECCE74B88002417
:104C90001B0A5360C7E74B881B0A222B1FD0212B0E
:104CA000BED1CA881149092A28BF0922FFF7BEFED2
:104CB000B9E790F87432032BB2D18B789360B2E7E6
:104CC00090F87422032AABD102220DF106011C4692
:104CD000FFF7ACFEA7E702F108010122E6E7CA8868
:104CE0000349362A28BF3622E0E700BF2406012008
:104CF000EC0501202DE9F0410A7884B000270D462B
:104D000012F060060446D0F890328DF80D70ADF8C0
:104D10000E7016D0202E1AD1CE8806B3120643D5B7
:104D200019460193D4F89432324668783E46D3F857
:104D30000880C047019BEA8820461946FFF776FEA7
:104D400009E04B780A2B20D00B2B28D08BB12046C2
:104D50000226F9F72BF9304604B0BDE8F081D0F80F
:104D60009432324648789B689847304604B0BDE894
:104D7000F08190F87432032B29D002262046F9F7EF
:104D800015F9304604B0BDE8F08190F87432032B79
:104D9000F3D101220DF10D01FFF748FEDBE790F89A
:104DA0007432032BD7D0E8E74A78032583F80162F1
:104DB000394683F800221A46C0F848613346C0F8E5
:104DC0004C613E46C0F86C52F9F708F8C3E702227E
:104DD0000DF10E01FFF72AFEBDE700BF2DE9F043FC
:104DE0000D784FF0010883B0044680F8805205F03A
:104DF0001F0C4F7800F5207EC44580F88172CB7877
:104E00008E7806EB0326B6B2A0F882624A790B7957
:104E100003EB02239BB2A0F8843291F807908A79C1
:104E2000C0F86C8202EB092292B2A0F88622C0F888
:104E300070220DD0BCF1020F3ED0BCF1000F19D092
:104E400005F08001F9F756F8002003B0BDE8F083C3
:104E500005F06002402A67D06A0665D580212046A9
:104E6000F9F748F820460021F9F744F8002003B08C
:104E7000BDE8F08305F06005202D6FD0402D6DD08A
:104E8000002DEBD1092FE9D801A151F827F000BF7F
:104E9000A94F0108D74F01085D4E0108F54F0108E1
:104EA0005D4E010805500108655001085D4E01087E
:104EB00091500108714F010805F06005202D4DD07B
:104EC000402D4BD0002DC9D1012FD9B200F0048163
:104ED000032F00F0EF80002FC0D190F87422022A37
:104EE00000F0CC81032AB9D113F0800F01F00F0339
:104EF00003EB830300EB830340F0D881D3F8443104
:104F0000002BABD001F07F03142202FB030202F559
:104F1000A072002B40F00D82002313601146204642
:104F20000222FFF783FD8FE794F87422013A022AE8
:104F300094D8DBB2032B91D8D4F88C32714620463A
:104F40009B689847B4F88632002B7FF47DAF002829
:104F50007FF47AAF2046FFF71FFD75E7D4F88C3257
:104F6000714620469B689847002003B0BDE8F08357
:104F7000F1B2C14D012985F806123FF66FAF90F8E6
:104F80007432022B00F0BE81032B00F0A981802136
:104F9000F8F7B0FF00212046F8F7ACFF95F80612AD
:104FA0002046FBF7B5FC4FE790F87432013B022B2B
:104FB0003FF654AF022A7FF451AF0122D0F87C3281
:104FC000C2600BB10323C360022204F10C0120462E
:104FD000FFF72CFD38E790F87432013B022B3FF6C7
:104FE0003DAF012E7FF430AF0023C0F87C32FFF7D5
:104FF000D3FC29E7012E7FF427AFC0F87C62FFF7CE
:10500000CBFC21E713437FF429AF7F2E3FF626AF79
:1050100090F87432032B3FF421AFF1B2D0F8A832EC
:1050200080F8761293F8BC23012A11D01A68002068
:1050300083F83810D2F8001821F4FE61C2F8001885
:10504000D2F8001841EA0611C2F8001883F8BC0330
:105050002046FFF7A1FC002E00F07C81022384F89B
:105060007432F1E6330A013B062B3FF6F7AE01A29C
:1050700052F823F0F5510108DB510108C95101082C
:105080005D4E01085D4E0108B35101086D510108E4
:10509000012A7FF4E3AE90F87432022B00F2FF8015
:1050A000002B3FF4DBAE0023014641F8083FFFF739
:1050B000BDFCC9E690F87432022B00F0D380032BBC
:1050C0007FF4CCAE4F063FF445AF56EA02037FF4BF
:1050D00041AFF8F70FFF3DE790F87422022A00F085
:1050E000C180032A7FF4BAAE002E7FF4ADAE48062D
:1050F0003FF430AFD4F8A80201F00F0142689142AA
:105100003FF628AF13F0800F4FF01C0340F02681CC
:1051100003FB01020025134602F5FE7283F8FD51E0
:1051200000231170937090F8BC33012B3FF412AF41
:105130000121036880F8BC1355781178012D0CBF4C
:1051400003F5106303F5306303EB4113196821F491
:1051500000111960D278023A012A03D81A6842F085
:1051600080521A60002380F8BC33F3E6037C002BE6
:105170007FF474AED0F88C320DF106001B6B9847AB
:1051800007234370BDF806306BB1B4F88622002ABD
:105190003FF4E0AE9A420146204628BF1A46ADF8D9
:1051A0000620FFF743FCB4F88632002B7FF44CAEA8
:1051B000D0E6037C002B7FF451AED0F88C320DF199
:1051C00006005B6B9847DDE7F6B2052E3FF646AE6C
:1051D000DFE806F0302820184038037C002B40F030
:1051E0009F80D0F88C320DF106009B6A984702230D
:1051F0004370C7E7D0F888320DF10601007C1B68C8
:105200009847BFE7D0F888320DF10601007C1B6992
:105210009847B7E7D0F888320DF10601007CDB68CB
:105220009847AFE7D0F888320DF10601007C9B6803
:105230009847A7E7D0F888320DF10601007C5B683B
:1052400098479FE7D0F888320DF10601007C9B69F2
:10525000984797E7D0F888320DF10601007C5B692A
:1052600098478FE74D063FF4F9ADF8F743FE204627
:105270008021F8F73FFEE7E5E08D01204A067FF444
:10528000EDAD1B064FF000034FF002024CBF00F1E2
:10529000140100F5A0710B60FFF7C8FBD4E5032BE8
:1052A0007FF4DCAD011DFFF7C1FBCDE59B69002B51
:1052B0003FF4D4AD01F07F035A1C02EB820200EBF5
:1052C0008202002B3FF428AED0F8A8121C2000FB6D
:1052D000031393F83E30002B3AD0012313601DE6F0
:1052E00079B3416801293FF435AEC9B2FBF710FB31
:1052F00095F8061220466160FBF712FB02287FF446
:1053000029AEABE500293FF425AE0121032341601E
:1053100080F87432FBF704FB02287FF41BAE9DE596
:10532000D0F88C320DF10600DB6A984702234370F7
:1053300028E7D0F8A8321C2000FB013393F8FE3197
:10534000C9E70223416080F87432FBF7E1FA01E615
:105350001360E3E5012384F8743275E503FB010271
:10536000012513463C3283F83D50D9E603682DE908
:10537000F04F13F0010785B000F0F080C44A13F439
:105380000025916821F400019160C46A9168B4FA23
:1053900084FE41EA04014FEA5E1E916000F0E38062
:1053A000BB49446BD1F88C20B4F5801F22F4401225
:1053B00042EA0402C1F88C2000F0B681B4FA84F409
:1053C00013F480124FEA5414019240F0D2809906EF
:1053D00000F1E480DE060CD5AD49D1F88C2022F036
:1053E0008072C1F88C20D1F88C20066B3243C1F852
:1053F0008C20590408D5A649C66DD1F8902022F416
:1054000040323243C1F890201A0408D5A049066EF4
:10541000D1F8902022F440223243C1F89020DE03DC
:1054200008D59B49466ED1F8902022F440123243B1
:10543000C1F89020590608D59549C66BD1F890203F
:1054400022F003023243C1F890201A0608D5904991
:10545000066CD1F8902022F00C023243C1F8902063
:10546000DE0508D58A49466CD1F8902022F030023A
:105470003243C1F89020990508D58549866CD1F84A
:10548000902022F0C0023243C1F890205A0508D57E
:105490007F49C66CD1F8902022F440723243C1F8A3
:1054A00090201E0508D57A49066DD1F8902022F487
:1054B00040623243C1F89020D90408D57449466D42
:1054C000D1F8902022F440523243C1F890209A043F
:1054D00008D56F49866DD1F8902022F440423243BE
:1054E000C1F8902013F4001C0ED06949D0F87480E4
:1054F000D1F89020B8F1006F22F0006208BF0124BB
:1055000042EA0802C1F890205E0309D5DFF88081E5
:10551000C26ED8F8901021F040710A43C8F890206C
:10552000190209D5DFF86881826FD8F8901021F050
:1055300080510A43C8F890205A0100F18E80B3F1DF
:10554000007F00F09980BEF1000F40F09580012CA3
:1055500000F0F180002005B0BDE8F08F13F40025C5
:10556000BE467FF41DAF2C4613F4801201923FF427
:105570002EAFDFF81CC1816BDCF88C20B1F5800FF9
:1055800022F4400242EA0102CCF88C2000F0D080E4
:10559000002908BF012499067FF51CAFDFF8F080D1
:1055A0003C4AD8F840903C49944649F08059C8F8A4
:1055B0004090D8F8408008F08058CDF80C80DDF895
:1055C0000C80D2F8008048F48078C2F80080D1F8CE
:1055D000008005E00A68A2EB0802642A00F2A080BD
:1055E000DCF80020D205F5D5DFF8A480D8F87020CB
:1055F00012F4407C826A02F4407919D0E14517D058
:10560000D8F870C0D8F870A02CF4407C4AF4803AE6
:10561000C8F870A0D8F870A02AF4803AC8F870A032
:10562000C8F870C0D8F870C01CF0010F40F00581B8
:10563000B9F5407F00F0EE80DFF854C0DCF80810C8
:1056400021F4F811CCF808101149C2F30B02D1F87B
:1056500070C042EA0C020A67BCE6DFF83480B3F19E
:10566000007FC26FD8F8901021F0005142EA010289
:10567000C8F890207FF467AF054A0749D2F8008048
:10568000964628F08068C2F80080D1F800800AE0D1
:105690000038024000700040F83301200A68A2EB95
:1056A0000802642A3CD8DEF800201601F6D46FB157
:1056B000C26A5AB98268DEF884704668120707F039
:1056C000706742EA86123A43CEF88420002D40F0FB
:1056D0008380019A22B1826BB2F5800F00F0818045
:1056E0009A010AD5C36842681B06876843EA821399
:1056F0005B4A43EA0773C2F88430594B1F681A4665
:1057000047F080671F600F6803E00B68DB1B642BAA
:1057100006D813681B01F8D5012C7FF41BAF0AE0F3
:10572000032005B0BDE8F08F00244FF0010E1BE709
:105730004FF0010E4BE64A4B4A491C681A4624F0CA
:1057400080541C600C6803E00B681B1B642BE7D8BB
:1057500013689E00F8D4002D6BD1019BC3B1836BFD
:10576000B3B93F4A4369D2F8884005691B0604F47F
:10577000403443EA85132343C2F88830D2F88C3092
:10578000046A23F4F853013C43EA0423C2F88C3042
:10579000BCF1000F10D0436FB3F1006F0CD18369DF
:1057A0002F4C00691B04D4F8882043EA801302F0D0
:1057B00070621343C4F88830294B18681A4640F0C9
:1057C00080501860086803E00B681B1A642BA7D888
:1057D00013689B00F8D5BDE6426BB2F5801F7FF4DD
:1057E00078AFDFF87CE0C268DEF8847046681206A5
:1057F00007F0E04842EA861242EA0802CEF8842026
:10580000DEF88C70C26927F01F07013A3A43CEF8E0
:105810008C2065E7DFF84880DFF84CC0D8F8081026
:1058200002EA0C0C21F4F81141EA0C01C8F8081046
:105830000AE7436B002B94D08FE7D1F800B041F218
:10584000883A06E0D1F800C0ACEB0B0CD4453FF62B
:1058500067AFD8F870C01CF0020FF3D0E8E600BFC5
:1058600000380240F8330120FFFCFF0F054A064BC9
:1058700092680649C2F382220868134493F82030E4
:10588000D8407047003802408CD80508F42B01201E
:10589000134908B58B6803F00C03042B1DD0082BAB
:1058A00019D14A684B68496802F03F0213F480033B
:1058B000C1F388111ABF0B4800230B48A1FB00015C
:1058C00045F042F9064B5B68C3F3014301335B00CB
:1058D000B0FBF3F008BD044808BD024808BD00BF96
:1058E0000038024000127A000024F400F8B50446A3
:1058F0008368B849E669E768B74DD0E904201A43E0
:10590000236802431868AB4201EA000142EA06023A
:1059100042EA0102A1691A605868226A20F44050E4
:1059200042EA010240EA07005860996821F43061B8
:1059300042EA01029A605FD0A84A93421CD0A84A6A
:10594000934200F00881A74A934200F01281A64AD0
:10595000934200F08B80A54A934200F0A380A44AB2
:10596000934200F05381A34A934200F02081002328
:105970000120C4E91833F8BD9F4BA04AD3F89030FA
:1059800003F00C03134493F82C30B6F5004F17D0F6
:10599000082BECD801A151F823F000BFD55A01081B
:1059A000155A0108BB5A01086F5901088F5A01089E
:1059B0006F5901086F5901086F590108455A0108CC
:1059C000082B06D8DFE803F0BBA79E059205050566
:1059D000890001200023A3F110014FF6EF729142DC
:1059E000C5D823F00F02C3F3420321681343CB60F1
:1059F0000023C4E91833F8BD7F4B804AD3F89030B8
:105A000003F00303013B022B40F29C80B6F5004FEC
:105A100000F0818078497A4B89681B68C1F3423174
:105A200060680A4492F82020D34003EB5003B3FB94
:105A3000F0F39BB2A3F110020DE0302B97D1B6F535
:105A4000004F4AD06268530803F50043B3FBF2F3FA
:105A50009BB2A3F110024FF6EF718A4287D82268F9
:105A60000020D3600023C4E91833F8BD624BD3F89B
:105A7000903003F44073B3F5007F1BD066D833B386
:105A8000B3F5807F7FF473AFB6F5004F2ED0FFF7EC
:105A9000FFFE636800EB5300B0FBF3F39BB2A3F18E
:105AA0001002D8E7544BD3F8903003F44063B3F5B9
:105AB000006F70D1B6F5004F24D06268514B03EBF4
:105AC0005203B3FBF2F39BB2A3F11002C3E7B6F5A6
:105AD000004F34D0FFF7CAFEDBE7626800205308AE
:105AE00003F58033B3FBF2F39BB274E7FFF7D0FE0C
:105AF0006168034600204A0802EB4303B3FBF1F35D
:105B00009BB268E7626800203F4B03EB5203B3FB94
:105B1000F2F39BB25FE738490020394B89681D6872
:105B2000C1F3423166680A44730892F8202025FACE
:105B300002F203EB4203B3FBF6F39BB24BE7FFF732
:105B400095FED5E7134493F828301EE7B3F5407F60
:105B50003FF475AF0BE7284BD3F8903003F03003D8
:105B6000202BA7D03FF669AF002BB0D0102B8BD0E5
:105B7000FDE6214BD3F8903003F0C003802B99D081
:105B800005D8002BA3D0402B3FF47EAFEFE6C02B0F
:105B90003FF455AFEBE605D8D3B1B3F5806F3FF4D2
:105BA00073AFE4E6B3F5406F3FF449AFDFE6124B65
:105BB000D3F8903003F44043B3F5004F3FF47AAF8D
:105BC0003BD8002B83D0B3F5804F3FF45DAFCEE6DA
:105BD0000A4A1BE7F369FFEF001001400044004050
:105BE00000480040004C00400050004000140140BC
:105BF00000780040007C0040003802408CD8050846
:105C0000F42B01200024F4000048E8010D4BD3F8E8
:105C1000903003F44053B3F5005F3FF44BAF07D827
:105C2000002B3FF454AFB3F5805F3FF42DAF9EE6F9
:105C3000B3F5405F3FF403AF99E6B3F5404F3FF44F
:105C4000FEAE94E600380240002807DB00F01F019A
:105C500001234009024A8B4042F82030704700BFC0
:105C600000E100E0034A0130116813685B1A8342C7
:105C7000FBD37047F833012001F01F01036A10B411
:105C800001248A408C4023EA04035DF8044B03623C
:105C9000016A0A4302627047034690F83C000128FB
:105CA00000F0C6800220F0B4012483F83D0083F8A0
:105CB0003C40002A31D0042A73D0082A1A6800F028
:105CC0009580166AC86826F480560D684F688C68FF
:105CD000010316622D03D06989B2166A05F42045C6
:105CE00020F4407026F4204640EA0720354320F493
:105CF00070400143D1611562D06920F44060D061E9
:105D0000D16941EA0421D16100220121104683F8C2
:105D10003D1083F83C20F0BC70471A68DFF814C1CE
:105D2000166A62450C6826F001064D68C86816625E
:105D30009769166A1DD0B2F1804F1AD0ACF57C4C31
:105D4000624516D00CF5806C624512D00CF5806C63
:105D500062450ED00CF5784C62450AD00CF5705CAB
:105D6000624506D0ACF5943C624502D047F001058F
:105D700002E027F003073D43000125F0F00526F07F
:105D80000A0604F00A04C0B28F68344328439061C5
:105D90001462906920F00C0090619169394391611F
:105DA000B2E71A68C868166A0D6826F010064F68D0
:105DB0008C68010316622D01906989B2166A05F09C
:105DC000A00520F4407026F0A00640EA07203543E5
:105DD00020F47040014391611562906920F44060A5
:105DE0009061916941EA042191618DE7176AC86861
:105DF00027F480770E684C688D68010117623602BF
:105E0000D069C9B2176A06F4206620F0030027F4AF
:105E1000206720433E4320F0F0000143D161166229
:105E2000D06920F00C00D061D1692943D1616BE7C2
:105E300002207047000001400368012201F01F01A9
:105E4000186A02FA01F120EA010010B418620F4C3E
:105E50001A6AA34241EA0201196212D00C4A934223
:105E60000FD099680B4A0A40062A06D0B2F5803F47
:105E700003D01A6842F001021A6000205DF8044B5A
:105E800070475A6C42F400425A64EAE7000001404D
:105E90000004014007000100F0B490F83D30002BF1
:105EA00066D0026802233B49B2F1804F80F83D3052
:105EB000A2EB01011368B1FA81F14FEA51113BD015
:105EC000002939D1344D354CA24218BFAA4233D0F3
:105ED000334F05F50065D71BAA42B7FA87F74FEA9B
:105EE00057174AD0002F48D12E4F2F4CA24218BF2F
:105EF000BA420CBF012700274AD02C4DA4F5963496
:105F0000A24218BFAA4220D004F58064A2423FD02A
:105F100004F58064A2423BD0816923F08003C46809
:105F20000B4341681360D46291620123536180F88E
:105F30003D300020F0BC7047194F23F07003856896
:105F4000D71B2B43B7FA87F77F09046923F4407303
:105F500085692343C668446823F080032B4313609C
:105F6000D662946209B9002FDFD043691363DCE77E
:105F700003F0FF0280F83C2093E70D4C23F0700300
:105F80008568A24243EA0503DFD0002FDDD1ABE7ED
:105F90000027DAE70000014000040040000800404C
:105FA000000401400040014000440140004801401D
:105FB000000C004010B4016802240B4A034680F82C
:105FC0003D4088680240062A06D0B2F5803F03D0E3
:105FD0000A6842F001020A600122002083F83D2095
:105FE0005DF8044B704700BF070001000B4B93F8AE
:105FF0001621D20703D5012283F80722704793F8B0
:1060000007224AB9D3F8783133B1054B1A781044D6
:106010005A78114418705970704700BFE08D012004
:10602000D852012040F0080210B50D4C84F84122EE
:1060300094F9BC21022A06DD420704D583071CBF60
:10604000012384F8C43105210648FAF761FF0621CF
:1060500084F842020348BDE81040FAF741BF00BF90
:10606000F00301202D06012010B5FAF7E9FEA8B3D0
:106070001B4C94F9BC31012B30DD59B3022B2DD0D0
:1060800094F8C4319BB971B180230521154884F877
:106090004732FAF73DFF062184F848021148BDE86F
:1060A0001040FAF71DBF0420BDE81040BAE70029F0
:1060B00014BF0020042094F8BF311A0748BF40F0F5
:1060C00002005B0701D411B108B940F00100BDE83E
:1060D0001040A7E7022BD3D10420ECE710BD00BF8E
:1060E000F003012033060120F8B5224C030A0546CF
:1060F000062104F2492784F84E0284F84D323846CE
:10610000FAF706FF94F8BF3184F84F02DB072AD470
:10611000B4F8C021AA4226D1174D41F26F71D4F8CC
:10612000493205F50276C5F80832C3B2304685F823
:106130000E324FF6FF738A4218BF01230621134423
:10614000C3F3072285F80D3285F80C22FAF7E0FE3A
:10615000072185F80E023046FAF7C2FE052104F544
:106160001470FAF7BDFE07210448BDE8F840FAF7BD
:10617000B7BE00BFF0030120E08D012039060120E9
:1061800008B5FAF75DFE48B1A1F59C53083BB3F59D
:106190007A7F03D20846BDE80840A5E708BD2DE98F
:1061A000F0476A4E3368002B3AD0694D694C05F5CB
:1061B000DE77306827F086FD002833D1664B1988DA
:1061C0001D46092909D95F8864227A43B2FBF1F29E
:1061D000452A40F39E811880588094F84932012B5B
:1061E00000F0C281022B00F0DD8133B905215B484C
:1061F000FAF776FE012384F84932594B1D68594B52
:106200001B78002B00F0D881574B1B68EB1A782BBA
:1062100040F2D281D4F89001F7F7A6FCC4F84C52B2
:10622000BDE8F087306827F045FD94F80F328046CE
:10623000052BBED8DFE803F00309151B3543AA2858
:10624000B7D1012384F80F32B3E7552817BF424A6C
:106250000223938801331CBF9380002384F80F32FC
:10626000A7E7032384F8100284F80F32A1E713286C
:1062700084F81102C4F82C0207DD374AD3880133B1
:10628000D380002384F80F3293E718B9052384F8EC
:106290000F328EE70023C4F83032042384F80F3223
:1062A00087E7D4F83032E218013382F81202D4F8CA
:1062B0002C22C4F8303293427FF47BAFE6E7D4F867
:1062C0002C322A4803F1020A4FFA8AF1FAF720FE2B
:1062D000804594F8109240F0148126201BF03CFC7D
:1062E000204B48B100221A701B4A53880133538057
:1062F000002384F80F325CE71A784A4519D100224E
:106300001A7009F1FF33102B00F2F680DFE813F06A
:1063100030008D008D00DE008D00F400F400F400EC
:106320003000F400F400F400F400F400F400F40091
:106330003000B9F1090F02D0B9F1110F01D1012AD2
:10634000DDD0054A538901335381DAE7D452012065
:10635000F0030120E08D01200253012040060120BE
:10636000A82A01201053012014530120F08F01208E
:10637000BAF1060F59DDB9F1010F06D0B9F1090FD5
:106380000CBF4FF002094FF0030994F8150294F87E
:10639000161294F8142241EA002194F912E294F9B9
:1063A00014C2900709B294F8133285F8BC9185F8AD
:1063B000BDE185F8BFC1A5F8C01106D512F00C0FDC
:1063C00014BF0122002285F8C421B9F1030F12D1B4
:1063D000BAF1090F29DD94F918220020082AA8BF74
:1063E000082222EAE27285F8F22143B201309A4291
:1063F0005ADC94F817320020D4F81CA09BB2024655
:106400005245904658DB7C4B85F8BE011B78232B08
:106410000BD109EB8903794A03EB8303A2F802E06D
:1064200091800CEB8303D08013800A227449754855
:1064300046F0FCFD10B1002384F83E32704B3A6800
:106440001A607A685A603A891A8194F83E3233BBEE
:1064500095F8C4316C4A002B117814BF0223012334
:1064600084F8401284F83E3295F8BF3113F00103EE
:1064700018BFB1FA81F3517818BF5B0984F8411253
:106480009188D8B29278A4F8421284F83F0284F836
:10649000442213B109B1A4F8461284F848020EF060
:1064A0004FF80EF04DF81FE704EB4308234493F830
:1064B0001A32A8F87E3198E7013204EB480852B24C
:1064C000B8F82080984508BF104699E7BAF1040F44
:1064D000ABDD94F8122294F8133243EA02235904F4
:1064E0001AB204D5C3F30D03A5F8C2319DE7002A03
:1064F000F8DBA5F8C03198E7444A938901339381CA
:10650000F2E619F0010F01BF404A138901331381EC
:10651000EEE63F4BD3F85822B3F85C12012A1AD1A9
:1065200041F25632914203D14FF0FF32C3F8582264
:10653000D3F85822306802EB820202EB820201EBB0
:10654000420189B2A3F85C1203681B6998470023D3
:106550002B806B8041E60132EAD1B1F5965F04BF32
:106560000122C3F85822E3E7294D95F9BC61002EBA
:106570003FF443AE022E11D14FF48040FFF7B4FD3B
:1065800084F8496295F9BC31012B7FF736AE95F856
:10659000BF31C3F3400385F8C4312EE6032384F8EA
:1065A0004932EFE71A4BB3F8C231002B3FF425AE66
:1065B000032384F8493220E694F8342094F83530E7
:1065C0009A4204D0FBF7F4FAC4F84C5228E6D4F807
:1065D0004C32EB1AB3F57A7FBFF422AE0D4B1B6839
:1065E000ED1A952D7FF61CAE05210B48FAF778FCC5
:1065F000BDE8F047FBF7DCBA10490120144901203F
:1066000014900120AC050120D85201200253012032
:10661000F00301201453012040060120104BD3F851
:10662000780110B5D8B10F4C217841B162780DF0E6
:10663000E3F9A388834216BF01210021A080E288EC
:106640005AB141F288339342B8BF13469A4204D0FC
:10665000E380BDE8104039F055BE0029F9D110BDE6
:10666000E08D0120D85201200023014410B410F81D
:10667000014B0822634013F0800F4FEA4304234686
:1066800016BF84F00703E3B2DBB2013AF3D18842CC
:10669000EDD118465DF8044B704700BF30B54FF49C
:1066A000806085B021F0E4FD48B3164C0023012141
:1066B0004FF4E13294F8505290F904009D42019158
:1066C00000924FF4806118BF08250F4A029521F00F
:1066D0002EFE206700384FF0FF0318BF012084F81A
:1066E0008C3084F89C3084F8AC3084F8BC3084F86A
:1066F000CC3084F8DC3084F8EC3084F8FC3005B021
:1067000030BD00BFE08D0120C5110108364B1B686C
:1067100013F0006359D0354B2DE9F0471F78B8428C
:106720004ED3FF2853D1DFF8D8A09AF8CC31002BF4
:1067300043D0DFF8D0800022C8E99522C8F85C2257
:10674000A8F86022002F4BD008F18C0310461446A5
:1067500011461546164603EB0719B3F802E010334D
:1067600033F804CC714413F810EC624413F90FCCE5
:10677000764509B212B238BF7646654553F80CEC3F
:10678000B8BF654653F808CC994574446044E4D1D9
:1067900088F8546288F8555291FBF7F192FBF7F2B2
:1067A000C8E99640124B0020A8F856121B78A8F8AA
:1067B0006022092B8AF8CC010CD00E48BDE8F08786
:1067C0000D4A02EB0010BDE8F08718467047002024
:1067D000BDE8F08798F85422084B0648DA80F2E7C3
:1067E0003A463946DEE700BFD85101207007002045
:1067F00010490120349001206C8E012014490120A1
:10680000F0030120E08D012070B40478A51E15F07E
:10681000FF061DD0451E02464FF6FF73354401E0CA
:1068200012F8014F1B1BAA429BB2F9D11C0A084463
:1068300010F8012CA24205BF10F8020CDBB20020B8
:10684000C01A08BFB0FA80F070BC08BF400970479A
:10685000FF244FF6FF73EAE72DE9F8434378434CF2
:10686000190703F00F0594F8642200D072B10021DB
:10687000AA4284F8681204D94FF000084046BDE8E7
:10688000F883AA1AD1B20E29F6D803E084F864522C
:1068900084F86822224492F8AC110029ECD003F06D
:1068A000F003802B40D0902B49D0A02BE4D1084698
:1068B00065F05F05FAF7C6FC02462D48131D84F803
:1068C000695284F86832FBF705FB94F86882B8F1E6
:1068D000000FD1D0A8F1020313F0FF0641D0254AE2
:1068E0004FF6FF71901912F8015B491B904289B273
:1068F000F9D15FFA81F90D0A4BB11E4FFE1817F856
:10690000011BD4F88C0227F003FABE42F7D14946A6
:10691000D4F88C0227F0FCF9D4F88C02294627F031
:10692000F7F94046BDE8F883042365F07F050226A9
:10693000984684F8683284F869523346CFE70846AF
:1069400065F06F05FAF77EFC0426062284F86B02D8
:10695000334684F86952904684F86A1284F86822B3
:10696000BDE7FF254FF00208A946C5E7E08D0120ED
:106970004A90012048900120C21D2DE9F04F02F4F9
:10698000FC7285B0524C064600AFD4F89032ADEBA5
:10699000020D04F5287A89460DEB0002E8465345BE
:1069A000FA602FD094F8E0130DF1010C94F8E10394
:1069B00001F00F0ED4F894520131C7F808C04EEA26
:1069C000401E07F1080084F8E0138DF800E0ED1A8E
:1069D000A2EB0C0B1946AB4544DD2A4638F0F4F81F
:1069E000D4F89022B96840462A44C4F890A2A1EB9A
:1069F0000801C4F89422C9B2C84700201437BD4624
:106A0000BDE8F08F94F8E05394F8E10305F00F012E
:106A1000B4F99AC2013541EA4011BCF1000F84F883
:106A2000E05341F01001D4F89452C9B2A5EB0A0B1F
:106A3000B8BF41F08001012888F8001022D1BBF1D5
:106A4000FE0F38DD07F10800FF2594F8982208F1C1
:106A500003031FFA8BF1786088F8015088F8022050
:106A6000BB6020E05A4638F0AFF8D4F89032404688
:106A700031465B44C4F89032C84701201437BD4604
:106A8000BDE8F08F07F1080094F89C2208F102039A
:106A9000B4F89812786088F80120BB6038F0D8F814
:106AA0001FFA8BF1786838F0D3F87868D7E902C21A
:106AB000D4E9A4358BE794F8981208F1030C07F198
:106AC000080088F801B088F80210C7F808C07EE70F
:106AD000E08D012010B5062982B004464FF0320344
:106AE0000A460DF1010028BF062221468DF800302C
:106AF00046F052FA024B68461B68984702B010BD38
:106B0000189201205E2810B50ED05D2804D00B4BE2
:106B1000BDE810405B681847084C63689847636895
:106B20003D20BDE810401847044C5D20636898473D
:106B300063683E20BDE81040184700BF189201204E
:106B400070B5084E05460C465E2073689847284687
:106B500073689847E0B2FFF7D5FFC4F30720BDE89C
:106B60007040CFE7189201200368002B2DE9F04117
:106B7000B8BF5B423A4F04463A4DA7FB03013A4E79
:106B8000890DB27905FB0135C5EB0515AD0087FB15
:106B90000537EB17C3EBA757002A55D101EB81014D
:106BA00001EB810107EB810109B2DFF8B880132006
:106BB000FFF7C6FF1B2008FB07552C4FE91787FB83
:106BC0000535C1EBA511264D09B2FFF7B9FF2368C2
:106BD0002320002BB4BF53214E21FFF7B1FF636880
:106BE000B279002BB8BF5B42A5FB0301890D08FBFE
:106BF0000138C8EB08184FEA880885FB08354FEACA
:106C0000E873C3EBA5552ABB01EB810101EB8101C0
:106C100005EB810109B21220FFF792FF114B1349D6
:106C20001A2003FB058581FB0531ED17C5EBA1118A
:106C300009B2FFF785FF63682220002BBDE8F04111
:106C4000B4BF572145217BE7C1EB011107EB81015F
:106C500009B2AAE7C1EB011105EB810109B2DAE73C
:106C60006BCA5F6B806967FF808F0120D34D621014
:106C700000234FF4167140F2D932018142814380E2
:106C80008380838130B4022515240580847130BC53
:106C90007047084B5A881B88801A9B1AC00090FBCB
:106CA000F3F00628A8BF062020EAE070C0F19600A5
:106CB000C0B27047BC8F0120094B03EB4002118921
:106CC000084A127802EAD122520707D0D3F884206A
:106CD000511CC3F88410134483F88800704700BF28
:106CE0001892012050060120164B426810B51B78FF
:106CF00003F00303032B21D1134B1B88DBB1134992
:106D00000A24134BB1F90410B3F9C63091FBF4F126
:106D10005B1A4FF4B4711B0103F5B9531433B3FB81
:106D2000F1F3C3F1080303F00F03603313704368FA
:106D300000225A7010BD05231370F8E72D2313703D
:106D4000F5E700BF7C8F01207E8F0120A05201203B
:106D500018920120436872221A70732243685A7095
:106D6000742243689A7000224368DA7070470F4BB0
:106D70000A214268B3F9043093FBF1F31B014FF48D
:106D8000B47103F5B9531433B3FBF1F310B503F049
:106D90000F03074C1919E35813604B6853600B7AC3
:106DA0001372002243685A7210BD00BFA052012026
:106DB000E4630608044B93F8CD3013F0FD0F14BFC5
:106DC0009E209D20704700BF18920120094B93F828
:106DD000CD3013F0FD0F06D142F210735843064B2D
:106DE00090FBF3F07047242358434FF47A7390FBE1
:106DF000F3F070471892012040D20600064B07EED0
:106E0000900A93F8CD30B8EEE70A1BB9DFED037AAC
:106E100020EE270A704700BF1892012048F9514020
:106E2000104B10B593F83421012A10D1D3F8382132
:106E3000811A00290BDD0221B3F82E4183F83411A9
:106E40000949B1FBF4F142B10A44C3F8382193F87F
:106E50003401013818BF012010BD0844C3F83801BF
:106E6000F5E700BF1892012040420F00831E00F199
:106E70007A02EA2123F8021F9342FBD14E2243F605
:106E80004913C280CE224385CD23028123228380F1
:106E9000A0F87220A0F87830704700BF30B400BB73
:106EA0001D48B0F83C3103F00103C3B990F84041EC
:106EB000ACB11A4A02F1F00502E00133A3420ED050
:106EC00052F8041B4904F8D590F82C1200EB81010C
:106ED000D1F8C41145F823100133A342F0D130BCDE
:106EE00070470D48B0F83C31032B4FEA530408D9E2
:106EF0000D6804F001030A4AA0F83C412A440A60E4
:106F0000D3E70A6848F20504054BA0F83C41134456
:106F100030BC0B60704700BF189201205C930120C9
:106F2000A08601002DE9F04100283AD12D4A92F8BF
:106F3000400180B32C4A00242C4B92F804E092F9D3
:106F400005C003EB8000CEF1FF07AEF17F0692F99A
:106F5000068003F1F002FFB2F6B203E0834202F1D1
:106F6000040218D053F8041B8904F7D5E1B2A1EB51
:106F70000C0181EAE175A5EBE175012D0DDC71B124
:106F8000414514BF394631468342D17004F10104B2
:106F900002F10402E6D1BDE8F0810821F4E7714670
:106FA000F2E7114B1A79F02A09D802F10F000D4AC5
:106FB0001871086844F21A1303440B60B7E7094AD2
:106FC0007F2593F9054092F842011D71844298791A
:106FD00001DA002C02DA4042C0B2987120445871A4
:106FE000E7E700BF18920120500601205C930120C2
:106FF000F0B5384E78B196F8B432002B46D0013B4C
:10700000354ADBB286F8B4321378DB0741D4334B10
:107010000A681A440A6096F84041B4B3304B002520
:107020002D4F03EB840403F1F00003E09C4200F1D8
:1070300004002AD053F8041BC1F30322062AF5D119
:1070400097F800C0EA431CF0010F02F001020DD0D6
:1070500096F8B42296F843E102EB050CBCFBFEF275
:107060000EFB12C2012ACCBF002201220135002AE8
:10707000DCD0C1F383419C4200F1040006EB8101A6
:10708000D1F8C42140F8042CD4D1F0BD96F8433196
:10709000B5E7D6EDB17A6420124BFDEEE77A124DDA
:1070A000124C17EE902AA2F57A7200FB02F283FBD3
:1070B0000230D317C3EBA01303EB4303C3EB03135B
:1070C00085FB0302DB17C3EB6213053394FBF3F379
:1070D0009EE700BF18920120F68E0120400D0300AC
:1070E0005C930120D34D62101F85EB5140420F008D
:1070F000F0B4524C002864D194F8000300285CD00E
:107100004F4BB3EE097AD3ED007AF4EEC77AF1EE85
:1071100010FA54DCBBEE097AF4EEC77AF1EE10FAFD
:107120004CBF08270027B3EE097AD3ED017AF4EEBD
:10713000C77AF1EE10FA6FDD47F0010794F840517D
:10714000002D3AD03F4ADFF80CC102EB850502F171
:10715000F00011E094F90363B142ACBF02210021B9
:1071600094F90463B34218DB41F004010F421CD1CF
:10717000954200F1040020D052F8043BD903F7D522
:1071800003F00F0194F90263C3F30313B142E1DC8E
:1071900094F904630121B342E6DA94F90563B3423A
:1071A000D8BF41F008010F42E2D0DCF80C30954224
:1071B00000F1040040F8043CDED1F0BC7047042725
:1071C000B1E794F801338BB31D4B1F4ED3ED007A1A
:1071D00093ED017AF0EEE77A1C4DB0EEC77A0A68BB
:1071E00094F80003C7FE877AFDEEE77A80F001008D
:1071F00017EE903A84F80003193B03EB4303C3EB0B
:10720000031386FB0376DB17C3EBE6130533B5FBED
:10721000F3F31A440A6071E7BBEE097AF4EEC77A19
:10722000F1EE10FA48BF47F0020787E70A68084BFB
:1072300094F8000313440B6060E700BF189201202C
:10724000AC8F01205C930120353AFC4440420F0092
:10725000400D0300FCD80508F0B40D4F97F84061CD
:10726000A6B107F5A272054607F50D77002302E0E7
:107270000133B3420AD052F8044B35EA0400F7D187
:10728000086847F823000133B342F4D1F0BC7047DB
:1072900018920120294B30B460B9294A127DBAB93D
:1072A00093F82D322749203301EB83014FF4A0607E
:1072B00030BCD1E793F80603E0B10138204A83F8E7
:1072C00006030C68204820440860127D002AE7D09D
:1072D0001E4A12689106E3D51D4A93F806131278E8
:1072E00092071AD511BB93F82F321649203301EBC0
:1072F0008301DBE7124A93F80743157DA54205D8C1
:10730000042483F8070383F80643DAE701340120F5
:1073100083F8074383F80603D3E70029C0D193F825
:107320002E320849203301EB8301BFE793F82B325B
:107330000449203301EB8301B8E700BF1892012014
:10734000F05101205C930120801A0600F08E01208C
:107350007C8F01201D4A10B448B91D4C92F80803D7
:107360000B6823440B6098B15DF8044B704792F8AA
:10737000093303B3012B16D092F808030B68154CA0
:1073800080F00100234482F808030B600028EBD151
:1073900092F82B324FF440700F4920335DF8044BC4
:1073A00001EB830158E792F808030C4C80F00100D0
:1073B00082F80803D4E708680124054B82F80843E3
:1073C00003445DF8044B0B60704700BF1892012026
:1073D00040420F0048E801005C93012020A1070013
:1073E0003F4A10B4B0B992F80A336BB192F80B135C
:1073F0008A081341DB070AD501F00101032A06D8E8
:10740000DFE802F0534B433B92F811335BBB5DF86E
:10741000044B704792F80B33013303F00F0382F8EB
:107420000B3333B192F80A330C682E4820440860BD
:10743000DBE72D4882F80A33437A002B46D12B48EC
:10744000C07818B143F0040382F80A332848007862
:10745000C00732D592F810030028E5D043F00803A6
:1074600082F80A33E0E792F81E33224901EB8301E8
:107470004FF400305DF8044BEEE61E4B03F1300292
:10748000002914BF19461146F2E71B4B03F11802FD
:1074900000290CBF19461146EAE7164B03F1080212
:1074A000002914BF19461146E2E7124B03F11802F6
:1074B000002914BF19461146DAE7D2F80C03002858
:1074C000C8D043F0010382F80A33C3E792F80933C6
:1074D000002BB4D00220034682F80A03AFE700BFB6
:1074E00018920120A0860100BC8F0120F88E012097
:1074F000F68E0120FCD805080CD9050870B432219D
:10750000022640F203154FF4FA7446F201420023BA
:10751000C6708580C48001814281038070BC704741
:10752000F8B5224C94F82013621892F82423002A0C
:107530003AD000231E4D4A1C0133A5FB02614908C5
:1075400001EBC101511A621892F824230AB1092BE8
:10755000F1D1CBB284F8203302680C260025571CE9
:10756000076001EB41071670026801EB8701561CAA
:10757000066015700D2205680E4E6F1C31440760C1
:107580002B7037F021FB94F820130120084B0A18C8
:107590002144A3FB025381F82403C34003EBC3033C
:1075A000D31A84F82033F8BD0B46D5E71892012092
:1075B000398EE33848950120024B0146D3F8A803E1
:1075C00026F0A6BB1892012008B5044BD3F8AC03F3
:1075D00026F078FBB0FA80F0400908BD189201202F
:1075E000044B93F831310BB11EF060B8024B188890
:1075F000704700BF18920120A48F0120084B07EEAE
:10760000900A93F8CD304BB9F8EEE77A9FED057A02
:107610009FED050AA7EE870A44F04CBA704700BFF9
:10762000189201206766E63F0000004210B5184C32
:10763000A379CBB194F82230C0B2DFED166A07EE21
:10764000903A154BF8EEE77A03EB8000838986EEDB
:10765000A77A07EE903AF8EEE77A67EE277AFDEE22
:10766000E77A17EE900A10BD0C4B1B6813F000630D
:107670000CD0C0B2FFF74AF86423808910FB03F0F6
:1076800094F822305B0890FBF3F0ECE71846EAE749
:10769000D4490120000048434C4E0020D85101201D
:1076A00008B5FFF7C3FF3C2390FBF3F008BD0328A8
:1076B00011D8DFE800F00A0C0206084BD3F8B40337
:1076C0007047074B1B78DB0701D426F003B9034B47
:1076D000D3F8B00370470020704700BF1892012014
:1076E000F68E0120F0B52B4F0E462B4A83B03B6837
:1076F0002A4D82FB0312DC17B5F8DC33C4EBA2047D
:107700003F89A4B2A3420CD1D5F8E0332449F31A3F
:10771000B5F8E4238B4298BFBA4214BF012300237B
:1077200034D0036834210022019003F1010CC0F829
:1077300000C019702146036803F1010CC0F800C0B5
:107740001A7037F085FA3946019837F081FA47F612
:10775000FF71019837F07CFA47F6FF71019837F016
:1077600077FA47F6FF71019837F072FA47F6FF7122
:10777000019837F06DFA01980221F5F765FC0123B5
:10778000A5F8DC43A5F8E473C5F8E063184603B038
:10779000F0BD00BFD88F0120676666661892012091
:1077A00080841E0002680E2170B5561C7F250024BF
:1077B000066015700268551C05601470F5F744FCEE
:1077C000012070BD2DE9F0416A4F84B06A4D044636
:1077D000D7F800800E4640460CF061FB85F8E603C2
:1077E000B8F1000F0AD00DF1090202A940460CF0D1
:1077F00086F9002840F08D8095F8E60300231946AD
:10780000ADF808308DF80A30431E0022FF208DF8B5
:107810000C10DBB2ADF80E208DF80B00FD2B04D957
:107820000023184604B0BDE8F0819DF80830042B11
:1078300000F09480052B00F09780032B00F09680D9
:10784000022B00F08A80012B00F092809DF8093015
:107850000DF10E023868013B9DF80A108DF80930D1
:107860000CF0B6F895F8E633032B74D0042B0CD14A
:10787000424A9DF80A000121002301E012F8011F8D
:1078800081426ED20133082BF8D1D5F8E8230DF1EF
:107890000808029B3A4F9A4250D023680D210022DB
:1078A000581C2060204619702368591C21601A70EA
:1078B00023689DF80820591C21601A7023689DF8E0
:1078C0000920591C21601A7023689DF80C20591C4E
:1078D00021601A7023689DF80A20591C21601A70D3
:1078E000BDF80E1037F0B4F923689DF80B20204640
:1078F000591C216007211A70F5F7A6FB0123C5F872
:10790000F06398E8030087E80300184604B0BDE878
:10791000F08101A940460CF0E9F800283FF46CAF73
:1079200040460DF10A010CF0E7F800283FF464AF7F
:10793000019995F8E60301F0010165E77A68D8F846
:1079400004309A42A9D1D5F8F0330E4AF31A934283
:107950007FF666AFA1E70C4A8BE703228DF808207B
:1079600074E78DF80A3090E70122F7E70222F5E785
:107970000422F3E7588F012018920120105E0608B8
:107980000096012080841E001C5E0608C74B1B6801
:107990002DE9F04F814613F0800083B000F078812C
:1079A000C34B187810F0020000F07281DFF820A3BA
:1079B0009AF81430052B40F27281DAF80030BD4C91
:1079C000002B0093BC48B8BF5B42BC49A4FB0352E8
:1079D000920D00FB023302EB8202C3EB031302EBB6
:1079E00082029B0084FB0354DD17C5EBA45500FB0A
:1079F000053305EB820581FB0321ADB2DB17C3EB39
:107A0000A111C5B10020AE4F0446A7FB053CC3B28F
:107A10002E4601304FEADC0C9A00092E0CEB8C0349
:107A2000A5EB43031FFA8CF59BB203FA02F344EA79
:107A30000304EAD8250489B2C1B10020A04F04464E
:107A4000A7FB013CC3B20E4601304FEADC0C9A00A2
:107A5000092E0CEB8C03A1EB43031FFA8CF19BB2B4
:107A600003FA02F344EA0304EAD82543DAF804B03F
:107A7000904C8BEAEB739048904AA3EBEB73A4FB1A
:107A80000361890D00FB013301EB8101C3EB03139B
:107A900001EB81019B0084FB0364DE17C6EBA45657
:107AA00000FB063306EB810682FB0312B6B2DB173E
:107AB000C3EBA212CEB10021814F0846A7FB063EC0
:107AC000CBB2344601314FEADE0E4FEA830C092C6B
:107AD0000EEB8E03A6EB43031FFA8EF69BB203FA5E
:107AE0000CF340EA0300E9D8060492B2CAB10021BF
:107AF000734F0846A7FB023ECBB2144601314FEA52
:107B0000DE0E4FEA830C092C0EEB8E03A2EB43032F
:107B10001FFA8EF29BB203FA0CF340EA0300E9D895
:107B20000643DAF80830664A002B18460193B8BFBE
:107B30005842644C6449A2FB0030030AA4FB03438F
:107B4000DB0901FB03F1C1EBD00189B2C1B1002413
:107B500096462746AEFB013CE3B20A4601344FEAA3
:107B6000DC0C9800092A0CEB8C03A1EB43031FFAF1
:107B70008CF19BB203FA00F347EA0307EAD8B9B2E3
:107B8000BAF81080B8F1000F1AD00024DFF830E105
:107B90002746AEFB083CE3B2424601344FEADC0C18
:107BA0009800092A0CEB8C03A8EB43031FFA8CF80E
:107BB0009BB203FA00F347EA0307EAD81FFA87F8F3
:107BC000BAF812303E4AA2FB0307FF08632F28BF12
:107BD0006327092B67D94FF0000C92466046AAFB39
:107BE000073E5FFA8CF33A460CF1010C4FEADE0EC9
:107BF0009C00092A0EEB8E03A7EB43031FFA8EF7B6
:107C00009BB203FA04F340EA0300E8D8C4B2009B35
:107C1000019A002BCCBF39233823BBF1000F4FEA68
:107C2000226738DD27F07F07284A3B43934543F01E
:107C30000207C8BF43F00607D9F80030162000221B
:107C400003F1010CC9F800C018704846D9F800309B
:107C500003F1010CC9F800C01A7036F0F9FF29468B
:107C6000484636F0DFFF3146484636F0DBFF4846EF
:107C7000414636F0EDFFD9F8003001201A18C9F856
:107C800000201C70D9F800301A18C9F800201F70A5
:107C900003B0BDE8F08F27F07F071F43CCE700203B
:107CA00003B0BDE8F08F0024B1E700BFD851012038
:107CB0007C8F01206BCA5F6B806967FFD34D6210B8
:107CC000CDCCCCCCC55A7C0AA0860100FFC99A3B1A
:107CD000F0510120AE4B1B682DE9F047064613F02A
:107CE000800084B000F0A180AA4B187810F0020048
:107CF00000F09B80DFF8B4E29EF81410052940F2F2
:107D00009980632900F29480002089B2A24F044632
:107D1000A7FB013CC3B20D4601304FEADC0C9A00D0
:107D2000092D0CEB8C03A1EB43031FFA8CF19BB2E2
:107D300003FA02F344EA0304EAD8E4B2DEF80830B6
:107D4000964AD91782FB0323C1EB633399B200290A
:107D500000F019810025DFF840C22846ACFB01384D
:107D6000EBB20F4601354FEAD8089A00092F08EB0D
:107D70008803A1EB43031FFA88F19BB203FA02F3D5
:107D800040EA0300EAD8C7B2BEF80E304FF4F365FC
:107D9000834942F20F7005FB03F5A1FB0535C5F3DE
:107DA0008F1585424AD8D5B10021DFF8ECE10846AD
:107DB000AEFB0538CBB2AC4601314FEAD8089A0089
:107DC000BCF1090F08EB8803A5EB43031FFA88F504
:107DD0009BB203FA02F340EA0300E9D885B2714B83
:107DE000D3E9FE2313433ED14FF0FF3833682946D1
:107DF000172000225D1C35601870304633685D1C0A
:107E000035601A7036F024FF4146304636F00AFFDE
:107E10003368304606215A1C32601C7033685A1C85
:107E200032601F70F5F710F9012004B0BDE8F0874B
:107E3000992483E7002004B0BDE8F0870021DFF833
:107E400058C10D46ACFB0032D20802EB8203A0EB16
:107E5000430390B29BB28B400431102945EA0305DD
:107E6000F0D1ADB2BBE701A837F0C2F99DF8081018
:107E7000002900F08A800020DFF81CE18046AEFB7C
:107E80000139C3B28C4601304FEAD9099A00BCF1DE
:107E9000090F09EB8903A1EB43031FFA89F19BB298
:107EA00003FA02F348EA0308E9D84FEA08289DF8E4
:107EB0000920E2B10021DFF8E0E00846AEFB023A1B
:107EC000CBB2944601314FEADA0A4FEA8309BCF19A
:107ED000090F0AEB8A03A2EB43031FFA8AF29BB253
:107EE00003FA09F340EA0300E8D848EA00089DF8DD
:107EF0000A204FEA0828E2B10021DFF89CE008469A
:107F0000AEFB023ACBB2944601314FEADA0A4FEAAD
:107F10008309BCF1090F0AEB8A03A2EB43031FFAA2
:107F20008AF29BB203FA09F340EA0300E8D848EA70
:107F30000008BDF80C304FEA08181B4A632BA2FB5F
:107F400003124FEA52127FF651AF0021DFF848E0EA
:107F50000846AEFB023ACBB2944601314FEADA0A48
:107F60004FEA8309BCF1090F0AEB8A03A2EB430332
:107F70001FFA8AF29BB203FA09F340EA0300E8D839
:107F800048EA000832E70F46FEE688468FE700BF62
:107F9000D85101207C8F0120CDCCCCCC89B5F814F0
:107FA000D34D6210189201201F85EB51F051012032
:107FB000F8B53B4B054601687E27B3F9003400262F
:107FC000384A481C03EBC3032860FF2082FB0342AE
:107FD000DC170F702B68C4EB62045A1C20342A6033
:107FE000A4B21E70FEF792FB2F4B00284DD01B78D9
:107FF000B0F90C1023BBA1F57A722C4B9A4246D8EB
:108000002B48B0FBF1F189B2284636F0FDFD294B33
:10801000DB7A7BB11DF04AFB0146284636F0F4FDC1
:108020002146284636F0F0FD28460821F5F70CF8E1
:108030000120F8BD204B2846198836F0E5FDEFE712
:108040001E4B1E78002ED6D000231D4800EB830265
:1080500001339289B3421144F8DB1A4B07EE901AB0
:108060009FED196A93F82230F8EE676A07EE103A2E
:10807000B8EEC77AC6EE077A67EEA67AFCEEE77A24
:1080800017EE901AB1FBF6F1B5E71B7813B94EF66F
:108090009C21B9E7094B1E78002EF8D00146D3E7A2
:1080A00018920120676666660C15002017839303FB
:1080B00000879303808F0120A48F01207007002088
:1080C0004C4E0020D449012000004843244A00239C
:1080D0004361D2F8DC1041F45C5130B541F02C0121
:1080E0000124C2F8DC104471D2F8D41004FA03F56C
:1080F0000133112B41EA0501F8D121F4F0314FF49D
:1081000020634FF0A064C2F8D4105022C38040F620
:10811000012314490381144BA0F856206FF07E42CE
:108120000360142303718023037642F61403038251
:108130004FF6FF73438303F58C03C36140F20123C1
:10814000C0E9161203840023084A80F8223080F820
:10815000333080F84430A0F86830C0E9184230BDB0
:1081600018920120C4FF00FF98086400180B0C004F
:1081700008B5A0F101030228B3FA83F34FEA5313C1
:1081800001D0184608BD0F2019F05CFC28B9054B3A
:108190001B7803F00103184608BD0F20BDE8084016
:1081A00019F0DABCF68E012038B505468022002190
:1081B00005F1800444F062FF00213822204644F09B
:1081C0005DFF00230B4951F8232044F8232001339D
:1081D0000E2BF8D11E22084905F1C00044F0DCFE48
:1081E0000B22064905F1E40044F0D6FE032385F88E
:1081F000EF3038BDFCD8050834D9050854D9050836
:10820000034B01220349B3F90830406837F0A6BD9B
:1082100050060120D45D060837B504462A4800EB15
:108220004303B3F8CE5005F00F0049B1022804F122
:1082300001011DD8002814BF9C239B2323700C46EA
:108240000AB3C5F30315FFF732FA204B3C21012D89
:10825000B0FBF3F3B3FBF1F201FB123315D0022DA7
:1082600023D01B49204603B0BDE8304037F076BD2F
:10827000032806D1174B1B7803F00103653BDBB2E3
:10828000DCE72023DAE71546DDE742F210716425CA
:10829000B0FBF1F1B1FBF5F005FB10100E490090B9
:1082A000204637F05BFD03B030BD0C490A25B0FB1A
:1082B000F1F1B1FBF5F005FB1010094900902046E3
:1082C00037F04CFDEFE700BF1892012040420F004D
:1082D0002E5E0608F68E0120385E0608A086010094
:1082E000475E0608037801224068053B114693E784
:1082F0001D4B1E499A68B1F8C83007EE902A9FEDD1
:108300001C7A4068F8EEE76A07EE903AF8EEE77AF2
:1083100067EE877AF4EEE76AF1EE10FA02D81549B3
:1083200037F01CBD934202DA134937F017BD9B1A90
:10833000124A07EE903AB8EEE77AD1EDEC7A3C219A
:10834000F8EE677A67EE277A87EEA67AFDEEC77AAF
:1083500017EE903AB3FBF2F3B3FBF1F201FB1233E9
:10836000074937F0FBBC00BFD88F012018920120CD
:10837000CDCCCC3D565E06085C5E060840420F0040
:108380002E5E0608064B07491A88074B40681B6893
:10839000534342F2107293FBF2F237F0DFBC00BF9E
:1083A000A48F0120625E0608D88F0120054A064985
:1083B00092F8053492F8042401334068013237F012
:1083C000CDBC00BF18920120675E06080B4B0A2245
:1083D0004FF4B4714068B3F9043093FBF2F31A011F
:1083E00002F5B9521432B2FBF1F2C2F108020449AB
:1083F00002F00F02603237F0B1BC00BFA052012082
:108400006D5E0608034A072303499268406837F007
:10841000A5BC00BFD88F0120745E060807B5144ABA
:10842000406892F81414B2F81634012909D1009367
:10843000104992F818347B2237F090FC03B05DF8B5
:1084400004FB022906D17B220B4903B05DF804EB43
:1084500037F084BC0A220949534340F2FF32B3FB90
:10846000F2F39BB27B22092B28BF0923EDE700BF63
:10847000189201207A5E06082F5F0608845E0608BF
:1084800013B54468FEF796FC0F4B02461B789B071A
:1084900012D50E4B93F823140D4B59B19889FEF762
:1084A00095FC0C49034600922046702237F056FC9A
:1084B00002B010BDD889F2E700902D237022064942
:1084C000204637F04BFCF3E77C8F01201892012007
:1084D000F0510120E25E06088A5E06082DE9F041AF
:1084E000404F86B090F800C006463C78BCF1170FAC
:1084F000416890F803E00CBF4FF098084FF08908EE
:1085000014F0040405D0BCF1170F374B0CBF5C68A6
:108510001C6884EAE473354DBEF1010F01F10100DE
:10852000A3EBE473B3FBF5F205FB123345D0BEF1C8
:10853000020F46D181F800803C21BCF1170F01FBEE
:1085400003F3B3FBF5FE05FB1E3301FB03F3B3FBA3
:10855000F5F105FB1135264BB5FBF3F528D1002CC1
:10856000B4BF572345230593222302912149CDE926
:1085700003532723CDE900E3082337F0EFFB3378DB
:108580001D495A0903F01F0301EB8201012202FA7F
:1085900003F33A78D1F8280402F00602042A0CBF4B
:1085A000034320EA0303C1F8283406B0BDE8F08194
:1085B000002CB4BF53234E23D5E74FF47A75B3FB99
:1085C000F5F3002C81F8008002DA2D24881C4C7011
:1085D0000A4C0B49BEF1000F08BF214637F0BEFB25
:1085E000CDE700BF7C8F0120F051012080969800DC
:1085F00040420F00A15E060818920120915E060815
:10860000995E06080D4B1B681B0137B514D50C4C41
:108610004568D4F8303493F90100FEF7EFFF94F881
:10862000CD2003460749002A28460CBF0D220E2202
:1086300000927A2237F092FB03B030BDD85101206E
:1086400018920120B75E0608034B0449D3F834247E
:10865000406837F083BB00BF18920120C05E060857
:10866000044B1B78DB0703D40349406837F076BB23
:10867000704700BFF68E0120C45E060807B5094AA0
:108680000949B2F906300193B2F904300093B2F906
:108690000230B2F90020406837F060FB03B05DF8AB
:1086A00004FB00BF14490120CD5E060837B50A4C13
:1086B0004568B4F90004FEF7A1FF94F8CD20034605
:1086C0000649002A28460CBF0D220E2200927A226B
:1086D00037F044FB03B030BD18920120E15E06087C
:1086E000084BD3F84424002A0ADD074B03EB82032E
:1086F0001A6E2AB1054B0649DB68406837F02EBB7D
:10870000704700BF18920120FCD8050850060120D0
:10871000EA5E06081FB59388029393780193537815
:10872000009313780A46034937F018FB05B05DF84B
:1087300004FB00BFF25E0608034B0449D3F848244B
:1087400040681432E6E700BF18920120055F060872
:10875000034B0449D3F8482440680832DAE700BFE5
:1087600018920120095F0608034B0449D3F84824F6
:1087700040680E32CEE700BF189201200D5F060858
:108780002DE9F0472DED028B82B0924607460C464C
:108790009DF8302099469DF83480002B52D0022B52
:1087A00014BF0A25642507EE905AF8EEE77A27EE03
:1087B000808A002A48D0B0EE480A43F07BF907EEE1
:1087C000900AF8EEE77AF0EEE77AFDEEE77A17EE38
:1087D000906AB6FBF5F205FB12660CB13C70012401
:1087E000B5EEC08AF1EE10FA05D552EA060302D0C2
:1087F0002D233B5501349AF800103819144B0029E9
:1088000014BF5146194637F0A9FA2518B9F1000FDF
:108810000AD04A460F49684637F0A0FA781932461E
:10882000694637F09BFA0544B8F1000F02D007F80B
:1088300005800135002328467B5502B0BDEC028B34
:10884000BDE8F0870125AEE7F0EE487ABBE700BF50
:10885000115F0608165F06081A4B1A6812F0200FFF
:1088600002F0040313B5446825D0174A1278920722
:1088700021D5164BB3F90000FEF7C0FADFED147AEC
:10888000144B204620EE270A134A93F8CD30B5EE5C
:10889000C00AB0EEC00AF1EE10FA4CBF7621752185
:1088A000002B0CBF99239F23019301230093FFF713
:1088B00067FF02B010BD002BDBD12D222270426871
:1088C0005370F6E7F08E01207C8F0120E48F0120A9
:1088D0000AD7233C1892012092AC06081FB5184B0A
:1088E0009FED187A1B88184A07EE903A9FED170AF9
:1088F00092F80923F8EEE77A4468F4EEC77A27EE97
:10890000800AF1EE10FAACBF01230223022A14D030
:108910008DED030A02931CF0C9FEFEF7BAF9029B23
:1089200001469DED030A01220620CDE90020084AF8
:108930002046FFF725FF04B010BD9721F3E700BFE5
:10894000A48F012000007A44189201200AD7233C0A
:1089500092AC0608114BB3F84C34B3F57A7F07B5E7
:10896000406806D201220E4903B05DF804EB37F0EF
:10897000F5B907EE903A572200239FED0A0AF8EE68
:10898000E77ACDE90032012327EE800A064A19462C
:10899000FFF7F6FE03B05DF804FB00BF189201205C
:1089A0001E5F06086F12833A92AC060873B5194E23
:1089B0000546406896F86834052B07D01F231E2211
:1089C000154902B0BDE8704037F0C8B9134C1E22FB
:1089D0001349237D00931F2337F0C0F996F8223105
:1089E000ABB16B6820220021DFED0E7A1A54638A46
:1089F000441C686800EE103A01230B4A2044B8EE8C
:108A0000C00ACDE9003120EE270AFFF7B9FE02B017
:108A100070BD00BF18920120265F0608F0510120AA
:108A20002D5F06080AD7233C92AC060807B5012340
:108A300047220649CDE90032054A91ED000A00219E
:108A40004068FFF79DFE03B05DF804FB88960120A7
:108A500092AC06080B4BDFED0C7A93ED000A9A23DB
:108A6000B8EEC00A07B520EE270A0021074AB0EE8B
:108A7000C00ACDE9001302234068FFF781FE03B06E
:108A80005DF804FBD88F01200AD7233C355F060828
:108A900013B504461CF00AFE0E4B00EE100A646883
:108AA00093F80933022B13D0FEF7F3F80146B8EE22
:108AB000C00ADFED097A00230622204620EE270AAD
:108AC000CDE900320223054AFFF75AFE02B010BD7D
:108AD0009721ECE7189201200AD7233C92AC0608B4
:108AE00013B50378134A1A2BDFED137A134C0CBF1E
:108AF000B2F90220B2F900201A2B4FF0010300EE68
:108B0000102A0CBF152114210022B8EEC00ACDE9AD
:108B1000003220EE270A0A4A4068B5EEC00AB0EEDD
:108B2000C00AF1EE10FA48BF2246FFF729FE02B054
:108B300010BD00BFA0520120CDCCCC3D395F06084E
:108B40003F5F0608194B37B51A68446812F0200FCA
:108B500002F0040320D0164A127892071CD5154A59
:108B6000C17892F8CD30D2F87404002B0CBF0F25D9
:108B70000C25FEF743F90123DFED0F7A2046009321
:108B8000CB1A20EE270A0D4A18BF01237F21019539
:108B9000FFF7F6FD03B030BD002BE0D17F222D2181
:108BA00022704268517042689370F3E7F08E0120A2
:108BB0007C8F0120189201200AD7233C92AC060832
:108BC00013B5044608461146FEF718F9164B93F8FC
:108BD000CD30002B0BBF4FF4A5534FF47A737E2298
:108BE0007D2207EE903A0CBF0F230C23F8EEE77AB4
:108BF000F4EEC07AF1EE10FA13DC80EE270AF2EE02
:108C0000047AB4EEE70AF1EE10FAACBF01230223B6
:108C10000192002220460092044AFFF7B1FD02B003
:108C200010BD1A460023F3E71892012092AC060803
:108C30000C4B10B41B78446803F00303032B06D1DC
:108C4000094B204611225DF8044B1988B8E711231F
:108C50002D22237043685A70002243689A705DF891
:108C6000044B70477C8F01207E8F0120094B4068A8
:108C70001B7803F00303032B07D1074B7122D3F8B2
:108C800078146423B1FBF3F19AE72D237122034991
:108C900037F064B87C8F0120189201208C5E0608A2
:108CA000224B1B885A0510B5446805D5204620493B
:108CB000BDE8104044F0C0BA180505D520461D494E
:108CC000BDE8104044F0B8BA590605D520461A4907
:108CD000BDE8104044F0B0BADA0705D52046174980
:108CE000BDE8104044F0A8BA9B0705D520461449BA
:108CF000BDE8104044F0A0BA252018F02DFF28B19F
:108D000020461049BDE8104044F096BA0E4B93F847
:108D10007C342BB120460D49BDE8104044F08CBA9C
:108D200020460B49BDE8104044F086BAC4520120E9
:108D3000455F06084A5F06084F5F0608545F06084D
:108D4000595F06085E5F060818920120635F0608F7
:108D5000685F0608074B93ED6E7AD3ED6B7AB4EE3D
:108D6000E77AF1EE10FA03DD0349406844F064BA93
:108D7000704700BF083100206D5F060810B50C4633
:108D8000A0B9174A174892F87D142368034423605A
:108D900001B110BD92F82B324FF48060124920339C
:108DA000BDE8104001EB8301FEF756BA11F046FF13
:108DB000322808DD206801210A4B094A034482F861
:108DC0007D14236010BD064A142892F87D14C8BF94
:108DD000064881F00101D8BF054882F87D14D4E728
:108DE0001892012040420F005C93012020A107004F
:108DF00048E8010010B504461AF0C6FF04220346F5
:108E000002496068BDE8104036F0A8BFD45D06088E
:108E10002B4BF0B51C6887B02A4E074620463178A8
:108E20000AF052FE7178054620460AF039FE00220B
:108E300003460592B2788DF813206CB1039005A912
:108E400020460AF053FE327A039B2AB10DF113013A
:108E500020460AF051FE039B9DF81310ECB1E1B1DE
:108E6000194A1268914218DC184A02EB8102D2F8C2
:108E700080442620039318F06FFE0599039B70B978
:108E800011F0010F14BF502200228907786808D51D
:108E90000F4936F063FF07B0F0BD0E4CE9E74422FE
:108EA000F3E732B10C49CDE900422A4636F056FFCD
:108EB000F1E72A460949009436F050FFEBE700BF7E
:108EC000588F0120D8520120FC8D012018920120DA
:108ED000705F0608CD650608785F0608845F06089F
:108EE000F8B50446417882782C48237890F8E95008
:108EF000302B2B4B05F1FF354FEA85052B4448D12C
:108F000093F8E85093F8E96000EB85054FF47A7721
:108F100000EB86004FF0030CD5EDAE7A40F2CF7532
:108F2000FDEEE77A17EE903AD0EDAE7AAB42FDEE69
:108F3000E77AA8BF2B4617EE900AB3F57A7FB8BF41
:108F40004FF47A73A842A3F57A73A8BF2846C3EBFF
:108F50000313B842B3FBF7F3C3F10E03B8BF3846AF
:108F6000DBB2A0F57A70B3FBFCFCC0EBC00062443E
:108F70000CEB4C0ED2B2A3EB0E03B0FBF7F70833A9
:108F800039442046DBB2C9B2F4F7E2FD0023237373
:108F9000F8BD93F8EA5093F8EB60B5E7189201201A
:108FA000FCD805082DE9F04790F80290044690F8A7
:108FB0000180002609F10207FFB2002508EB060A2E
:108FC000032E1BD108F10301022DC9B20ED10B23D0
:108FD0003A462046F4F7BCFD0135052DF0D10136A7
:108FE000072EEAD100232373BDE8F08709EB0502C1
:108FF00016232046D2B2F4F7ABFDEDE7022DEBD1FC
:1090000017233A465FFA8AF12046F4F7A1FDE3E719
:1090100070B504466FF00205A278132361782046EC
:1090200052FA85F2EEB207390135D2B2C9B2F4F77D
:109030008FFDA27861781323324420460731D2B2E3
:10904000C9B2F4F785FD042DE6D161780323A27837
:1090500020460639C9B2F4F77BFD61780223A27875
:1090600006312046C9B2F4F773FD0023237370BDA7
:109070002D492DE9F84391F8D830054691F8D920CB
:1090800091F8E71003EB830302EB820227480029E3
:109090004FEA43034FEA4202B0F9004014BF4FF0D9
